:1000000000800020BD010000CDA3000091A30000EE
:1000100091A3000091A3000091A3000091A3000010
:1000200091A3000091A3000091A30000CDA30000C4
:10003000CDA3000091A30000CDA3000081A3000088
:10004000CDA30000CDA30000CDA30000CDA30000F0
:10005000CDA30000CDA30000CDA30000CDA30000E0
:10006000CDA30000CDA30000CDA30000CDA30000D0
:10007000CDA30000CDA30000CDA30000CDA30000C0
:10008000CDA30000CDA30000CDA30000CDA30000B0
:10009000CDA30000CDA30000CDA30000CDA30000A0
:1000A000DD9D0000CDA30000CDA30000CDA3000086
:1000B000CDA30000CDA30000CDA30000CDA3000080
:1000C000CDA30000CDA30000CDA30000CDA3000070
:1000D000CDA30000CDA30000CDA30000CDA3000060
:1000E000CDA30000CDA30000CDA30000CDA3000050
:1000F000CDA3000069AE0000CDA300003DCB000001
:10010000CDA30000B9D00000CDA30000CDA3000016
:10011000CDA30000CDA30000CDA30000CDA300001F
:10012000CDA30000CDA30000CDA30000CDA300000F
:10013000CDA30000CDA30000CDA30000CDA30000FF
:10014000CDA30000CDA30000CDA30000CDA30000EF
:10015000CDA30000CDA30000CDA30000CDA30000DF
:10016000CDA3000051B10000CDA30000CDA300003D
:10017000CDA30000CDA30000CDA30000CDA30000BF
:10018000CDA30000CDA30000CDA30000CDA30000AF
:10019000CDA3000069710000CDA30000CDA3000035
:1001A000CDA30000CDA30000CDA30000CDA300008F
:1001B000CDA30000CDA300005DBE0000574B4CF264
:1001C000205210B51A804DF628121A8000BF00BFC9
:1001D0000AF000F9524B4FF010621A60514A9A60CF
:1001E000514ADA60A3F53043203B1A6812F480725A
:1001F00004D14E490A604FF4A8521A604C4B1A7849
:10020000110703D51A7842F008021A70494B4A4C7C
:100210004A482A221A704A4A00239918A14203D256
:10022000195899500433F8E7464B474900228B424E
:1002300002D243F8042BFAE74448454900235A58B0
:100240001A500433B3F5DE7FF9D1424B424A802184
:1002500003F8011B9342FBD1404B3C4A1A60404BD0
:100260008A221A70A3F5805324225A70A0221A7091
:100270009A799207FCD59A79D406FCD4394A9379B5
:1002800003F00C03082B374BF9D103221A714022DB
:100290005A719A799006FCD5324A9179314B4906C8
:1002A000FBD5314A314911600221516020221A7078
:1002B0009A7902F00C020C2AFAD12D4B2D4A1A60C1
:1002C0002D4B2E4A1A6000225A60072243F8042C54
:1002D0002B4AC3F80C2D62B60AF066FA134B1B6862
:1002E000DA0705D527480AF025F9274B274A1A606F
:1002F000274B1B785B0609D5234C244A236893427D
:1003000004D120480AF016F9002323600EF03EF9CC
:100310000AF066F80CF096F8FEE700BF0E200540E4
:1003200030800440823F04000100002B14D00340C1
:1003300002D0074000E0074080AFFF1F500E0100D1
:100340006097FF1F80AFFF1F9CDEFF1F0092FF1F03
:100350000000000000E400E05FE400E008ED00E0E1
:100360000050064000400640448004400000030165
:1003700004800440C010050014E000E0FF76010096
:1003800000002020648D9E5B1CE00340A5C3945AAE
:1003900000F00740FFFFFFFFFFFFFFFFFFFFFFFF32
:1003A000FFFFFFFFFFFFFFFFFFFFFFFFFFFFFFFF5D
:1003B000FFFFFFFFFFFFFFFFFFFFFFFFFFFFFFFF4D
:1003C000FFFFFFFFFFFFFFFFFFFFFFFFFFFFFFFF3D
:1003D000FFFFFFFFFFFFFFFFFFFFFFFFFFFFFFFF2D
:1003E000FFFFFFFFFFFFFFFFFFFFFFFFFFFFFFFF1D
:1003F000FFFFFFFFFFFFFFFFFFFFFFFFFFFFFFFF0D
:10040000FFFFFFFFFFFFFFFFFFFFFFFFDEF9FFFF23
:1004100010B5054C237833B9044B13B10448AFF33E
:1004200000800123237010BD80AFFF1F000000007B
:10043000500E010008B5064B1BB106480649AFF344
:1004400000800648036813B1054B03B1984708BD07
:1004500000000000500E010084AFFF1F80AFFF1F9F
:100460000000000038B5074C074DC4F8B05204F541
:10047000327008F0CFFC204640F8185B08F0CAFC48
:1004800038BD00BF84C0FF1FA009010070B5084E31
:1004900006F62804A6F52676064D44F8185C204694
:1004A00008F0B8FCA4F52C74B442F6D170BD00BFBE
:1004B0003CB2FF1FA009010008B5224B1B7813B105
:1004C000012B13D008BD204B1968204B1B68194421
:1004D0001F4B19601F4806F035FE0122194B1A7098
:1004E0001D4814211D4A06F033FF08BD184B1A6839
:1004F000164909680A441A60194B1B7823B1194B35
:100500001B689A4204DA0AE0164B1B689A4206DC22
:10051000144B1A680E4B1A6002220A4B1A700D48CF
:100520000B4B196806F00EFE064B1B78012B05D10C
:1005300009481421094A06F00BFF08BD0022014BAF
:100540001A7008BDAAB0FF1F549AFF1FA4B0FF1F66
:10055000E0AFFF1FD0C6FF1F0CB1FF1FB9040000A2
:1005600034CBFF1FB0A4FF1F00B583B0374B1B78FF
:1005700043B10022364B1A703648374B196806F0E3
:1005800001FF5FE0354B1B78012B1AD013B1022B12
:1005900036D057E0324B18780AF000F8002851D1D5
:1005A000304B1B680093009A2F4B1A602948142186
:1005B0002E4A06F0CDFE284B18600122274B1A70F8
:1005C00040E0274B187809F0E9FF58BB244B5B78D3
:1005D00063B327E01F481421244A06F0B9FE1E4BDE
:1005E00018602FE001221A4B1A7002221B4B1A705E
:1005F000184864211D4A06F0ABFE174B186021E035
:10060000174B187809F0CAFF012803D10022104BBC
:100610001A7017E00F486421144A06F099FE0E4B39
:1006200018600FE000220A4B1A700BE00D4B1B689C
:100630000193019A0C4B1B68D21A40F2DB539A4289
:10064000C8D9CFE703B05DF804FB00BF5BBFFF1F55
:10065000B8C6FF1F0CB1FF1F04BEFF1FE4C5FF1F7C
:1006600068C9FF1F50DBFF1FF8CAFF1F69050000A4
:100670000F4B03604172026100230372C36039B102
:100680001946026942F823100133427A9A42F8DC93
:10069000084B1A680AB9186004E053690BB11A468E
:1006A000FBE75061002343618380C380704700BF34
:1006B00080FB0000E0DCFF1F144B03600423437247
:1006C00000F12803036100230372C3601946026925
:1006D00042F823100133427A9342F8DB0C4B1A683C
:1006E0000AB9186004E053690BB11A46FBE7506180
:1006F000002343618380C380064B03604FF4803343
:100700008361C36103624362704700BF80FB0000E6
:10071000E0DCFF1F8009010010B504460F4B0360A9
:100720000023437203610372C3600D4B1A680AB958
:10073000186004E053690BB11A46FBE754610023CB
:100740006361A380E3802046064B40F8183B08F025
:1007500051FB204607F062F9204610BD80FB0000E7
:10076000E0DCFF1FA009010010B5124B5B7B13B941
:10077000114B5B7B4BB1114B5B7B33B1104B5B7B04
:100780001BB101220F4B1A7010BD00220D4B1A70C5
:100790000D4B1B7863B10D4C20460BF03BFC2368DE
:1007A0005B6820460A492622984720460BF032FC17
:1007B00010BD00BF1CA4FF1F349AFF1F34A4FF1FED
:1007C00010A3FF1FE8CAFF1F339AFF1F14DDFF1F8E
:1007D000A0FB000010B5174B5B7B9BB10122164BB1
:1007E0001A70164B1B781BB3154C23685B682046A8
:1007F00014491C22984720460BF00CFC20460BF0B5
:1008000009FC10BD00220C4B1A700C4B1B787BB1FD
:100810000B4C20460BF0FEFB23685B6820460A4920
:100820002E22984720460BF0F5FB20460BF0F2FBFA
:1008300010BD00BFB4A4FF1F5ABFFF1F339AFF1F94
:1008400014DDFF1FC8FB0000E8FB0000F8B50746F9
:10085000224B1B78002B3FD0214803685B6821495D
:100860000E229847204A4FF42C7303FB07F3D41849
:1008700004F2832402F524761E44194D2B681B686C
:10088000284614F8011F9847B442F7D1144C236846
:100890005B682046154910229847204639460A22AF
:1008A00000230BF0C7FB23685B6820461049062233
:1008B00098474FF42C720C4B02FB07372046B7F8D1
:1008C000AA120BF0F3FB23685B682046094901225A
:1008D000984720460BF09EFBF8BD00BF339AFF1FE0
:1008E00014DDFF1F18FC000084C0FF1F28FC00005F
:1008F0003CFC000044FC0000F8B50746224B1B7886
:10090000002B3FD0214803685B6821490E2298479D
:10091000204A4FF42C7303FB07F3D41804F283240A
:1009200002F524761E44194D2B681B68284614F8DE
:10093000011F9847B442F7D1144C23685B682046E6
:1009400015490C229847204639460A2200230BF00D
:1009500071FB23685B6820461049062298474FF4D4
:100960002C720C4B02FB07372046B7F8AA120BF08B
:100970009DFB23685B682046094901229847204671
:100980000BF048FBF8BD00BF339AFF1F14DDFF1FBB
:1009900018FC00003CB2FF1F48FC00003CFC0000BB
:1009A00044FC0000F8B50746224B1B78002B3FD0D3
:1009B000214803685B6821490E229847204A4FF47A
:1009C0002C7303FB07F3D41804F2832402F5247676
:1009D0001E44194D2B681B68284614F8011F9847C0
:1009E000B442F7D1144C23685B68204615490C22A9
:1009F0009847204639460A2200230BF01BFB236848
:100A00005B6820461049062298474FF42C720C4B25
:100A100002FB07372046B7F8AA120BF047FB236802
:100A20005B68204609490122984720460BF0F2FAFC
:100A3000F8BD00BF339AFF1F14DDFF1F58FC0000F4
:100A40003CB2FF1F48FC00003CFC000044FC0000DE
:100A500038B50546124B1B7803B3124C23685B680C
:100A600020461149072298472046691C0BF01EFBBF
:100A700023685B6820460D490A2298470C4B03EB1C
:100A800005152046A9890BF011FB23685B682046F9
:100A900008490322984720460BF0BCFA38BD00BF36
:100AA000339AFF1F14DDFF1F68FC000070FC00007C
:100AB000ACB0FF1F7CFC000010B50446092804D828
:100AC000054803681B6830219847034821460A22DD
:100AD00000230BF0AFFA10BD14DDFF1FF8B5274B54
:100AE000A3FB00239B0B264DA5FB03246409C4EB49
:100AF0000414A3EB8404234BA3FB00239B09A5FB55
:100B000003256D09C5EB0515A3EB85054FF47A7236
:100B100002FB13000DF0C2FA1B490DF0C7FB06469D
:100B200000210DF0C1FC40B130464FF07C510DF07A
:100B300001FA0DF0CDFC074607E030464FF07C513E
:100B40000DF0F6F90DF0C4FC0746E0B2FFF7B4FF74
:100B50000E4C23680E4E5B682046314601229847B2
:100B6000E8B2FFF7A9FF23685B68204631460122FF
:100B70009847F8B2FFF7A0FFF8BD00BF73B2E74592
:100B800089888888D34D62100000204114DDFF1F42
:100B900080FC0000F8B53225094C0A4F0126236875
:100BA0005B6820463946324698476B1E13F0FF05B6
:100BB000F5D103480BF02EFA0AF0DAFFF8BD00BFBA
:100BC00014DDFF1F84FC000010B584B0164C2046D5
:100BD0000BF020FAFFF7DEFF23685B68204613491D
:100BE000122298472046124B19780A2200230BF054
:100BF00021FA20460BF00EFA23685B6820460D4967
:100C00001222984768460C490BF0F0FB20466946D3
:100C10000BF0DAF920460BF0FDF9FFF7BBFF684651
:100C20000BF098FB04B010BD14DDFF1F88FC000022
:100C3000CB9CFF1F9CFC0000B0FC0000F8B53225E7
:100C4000094C0A4F012623685B6820463946324624
:100C500098476B1E13F0FF05F5D103480BF0DAF946
:100C60000AF086FFF8BD00BF14DDFF1FA4FD0000E1
:100C700008B5034803685B6802490122984708BD2C
:100C800014DDFF1F7800010038B5054630B100249F
:100C9000FFF7EEFF0134E4B2AC42F9D138BD00BF3A
:100CA00070B506460024124D2B681B682846315D3E
:100CB000984701340D2CF7D10620FFF7E5FF737B31
:100CC00063B13069FFF70AFF0620FFF7DDFF084830
:100CD000317D0A2200230BF0ADF905E004480368DA
:100CE0005B6804490122984701480BF093F970BDF5
:100CF00014DDFF1F84FC000038B5154C20460BF0B6
:100D000089F9FFF747FF23685B68204611490F22E6
:100D1000984720460BF07EF9FFF73CFF23685B689D
:100D200020460D492822984720460BF073F9FFF71B
:100D300031FF0A4D2C1F05F50B7554F8040FFFF712
:100D4000AFFFAC42F9D102480BF064F938BD00BFE7
:100D500014DDFF1FC0FC0000D0FC0000D8C6FF1F40
:100D600008B530B1064803685B6806490322984716
:100D700008BD034803685B6803490222984708BD21
:100D800014DDFF1F0CFD000010FD000008B5FFF78B
:100D9000E7FF02480BF03EF908BD00BF14DDFF1F5E
:100DA00030B4002308481946012502241954C218FA
:100DB00051709170D57014710533962BF6D10022C5
:100DC000024B1A7030BC704738BEFF1F64C9FF1F4A
:100DD00038B5274C23685B68204626490722984788
:100DE00020460BF017F923685B68204622490F2242
:100DF0009847224D286822490DF0A4F90DF08EFB8A
:100E0000C1B220460A2200230BF014F920460BF051
:100E100001F923685B6820461A49102298476868E0
:100E200017490DF08FF90DF079FBC1B220460A2267
:100E300000230BF0FFF820460BF0ECF823685B680A
:100E40002046114916229847A8680D490DF07AF9F5
:100E50000DF064FBC1B220460A2200230BF0EAF831
:100E600020460BF0D7F820460BF0D4F838BD00BF71
:100E700014DDFF1F24FD00002CFD00004098FF1F23
:100E80000000C8423CFD000050FD00002DE9F84381
:100E90002A4C23685B68204629490F229847204640
:100EA0000BF0B8F800260125DFF8AC90DFF8AC8035
:100EB00023685B6820464946072298472046294612
:100EC0000BF0F4F823685B682046414605229847FA
:100ED0001C4F2046B95B0BF0E9F823685B6820469D
:100EE0001949052298473744204679880BF0DEF8E7
:100EF00023685B6820461549092298473879FFF72F
:100F00002FFF20460BF086F801351036072DCFD184
:100F10000A4C23685B6820460D49112298472046F9
:100F20000C4B19780A2200230BF084F820460BF0B2
:100F300071F820460BF06EF8BDE8F88314DDFF1F52
:100F400068FD0000ACB0FF1F80FD000088FD0000C0
:100F500094FD0000D79CFF1F68FC000078FD000096
:100F60002DE9F843002601251D4CDFF88490DFF8B9
:100F7000848023685B6820464946062298472046BD
:100F800029460BF093F823685B68204641460D2202
:100F90009847144F2046B95B0BF088F823685B68CC
:100FA00020461149102298473744204679880BF093
:100FB0007DF823685B6820460C491122984720463B
:100FC000B9880BF073F820460BF024F8013506368B
:100FD000042DCED102480BF01DF8BDE8F88300BF08
:100FE00014DDFF1F24BEFF1FC0FD0000D4FD000064
:100FF000A8FD0000B0FD000010B582B03C4C236895
:101000005B6820463B491822984720460BF002F8BF
:1010100023685B682046384921229847374B187867
:10102000FFF7B4FE23685B682046354925229847C0
:10103000344B1868B8B10DF02DF833490DF036F97E
:101040000CF064FC02460B460121009120460BF097
:1010500037F823685B6820462C49082298472046C9
:101060000AF0D8FF09E0224C23685B682046284933
:101070000322984720460AF0CDFF1D4803685B68AD
:10108000244918229847244B1B7853B1184C2368E5
:101090005B68204621490C22984720460AF0BAFF97
:1010A00009E0134C23685B6820461D4909229847D4
:1010B00020460AF0AFFF0E4C23685B6820461949B2
:1010C0000F2298472046184B19780A2200230AF06D
:1010D000B1FF23685B6820461449012298472046E7
:1010E0000AF098FF20460AF095FF02B010BD00BF3D
:1010F00014DDFF1FE8FD000004FE000000BEFF1F1E
:1011000028FE0000E4C9FF1F00606A4750FE00008F
:101110005CFE000060FE0000C89CFF1F7CFE00001B
:101120008CFE000098FE0000C99CFF1F20FD0000FF
:1011300038B53D4C23685B6820463C490E229847F1
:1011400020460AF067FF23685B6820463849102272
:101150009847384B1878FFF719FE23685B682046DC
:101160003549102298472046344B19880AF09EFFD3
:101170002368334D5B682046294603229847204662
:101180000AF048FF23685B6820462E4910229847E2
:1011900020462D4B19880AF089FF23685B6820469A
:1011A00029460322984720460AF034FF23685B68EB
:1011B000204626490C2298472046254B19780A22BA
:1011C00000230AF037FF23685B68204621490C2280
:1011D00098472046204B19680AF068FF23685B682F
:1011E00020461E490622984720461D4B19780A22A0
:1011F00000230AF01FFF23685B68204619490B2271
:1012000098472046184B19680AF050FF23685B681E
:10121000204616490422984720460AF0FBFE204645
:101220000AF0F8FE38BD00BF14DDFF1FA8FE000065
:10123000B8FE000034CBFF1FCCFE00009ACAFF1F8F
:101240007CFC0000E0FE000004CBFF1FF4FE000069
:10125000ACA4FF1F04FF0000549AFF1F14FF0000FE
:10126000329AFF1F1CFF0000B0A4FF1F28FF0000E0
:1012700070B50D4614460138072800F2F880DFE803
:1012800010F008000F0016001D0031005A009A00EF
:10129000C200774803685B6876490C22984770BDA6
:1012A000734803685B6874490B22984770BD7048A7
:1012B00003685B6871490D22984770BD6C4C2368C8
:1012C0005B6820466E4907229847204629460A2235
:1012D00000230AF0AFFE23685B68204669490522B7
:1012E000984770BD624E33685B68304666490C2291
:1012F0009847304629460A2200230AF09BFE022C1A
:101300000BD0032C10D0012C40F0B1803046336854
:101310005B685E490622984770BD554803685B6864
:101320005B490522984770BD514803685B6859497D
:101330000722984770BD4E4E33685B683046564969
:1013400006229847304629460A2200230AF072FEF8
:10135000013C052C00F28B80DFE804F0030A111831
:101360001F26434803685B684C490322984770BDB9
:101370003F4803685B684A490422984770BD3C486F
:1013800003685B6843490722984770BD3848036883
:101390005B6844490F22984770BD354803685B6815
:1013A00041491022984770BD314803685B683F4946
:1013B0000622984770BD2E4E33685B6830463C4924
:1013C0000B229847304629460A2200230AF032FEB3
:1013D000022C0AD0032C0FD0012C48D130463368A0
:1013E0005B6834490522984770BD214803685B68F3
:1013F00027490522984770BD1D4803685B682E4940
:101400000722984770BD1A4803685B682B490B2276
:101410009847012D164803685B680CBF2849294985
:1014200001229847013C082C21D8DFE804F0052070
:10143000202020200C131A000D4803685B68224905
:101440000A22984770BD0A4803685B681F490A2250
:10145000984770BD064803685B681D490E2298478F
:1014600070BD034803685B681A490C22984770BD39
:1014700014DDFF1F30FF000040FF00004CFF0000A4
:101480005CFF000064FF00006CFF00007CFF0000B8
:1014900084FF00008CFF0000A8FD000094FF000006
:1014A00098FF0000A0FF0000B0FF0000C4FF000094
:1014B000CCFF0000D8FF0000E0FF0000E8FF0000C4
:1014C000F4FF0000F8FF0000FCFF0000080001002E
:1014D00014000100240001002DE9F8435A4C236850
:1014E0005B68204659490D22984720460AF092FD34
:1014F000574D0126DFF89091DFF8908123685B68F3
:101500002046494608229847204631460AF0CEFD3B
:1015100023685B6820464146022298472F466B7D30
:1015200093B123685B6820464A49082298472046C1
:10153000697A0A2200230AF07DFD23685B68204651
:1015400045490B22984727E023685B6820464349BA
:1015500011229847AB7D012B0AD013B1022B0ED07C
:1015600014E023685B6820463D490422984713E055
:1015700023685B6820463B490C2298470CE02368AF
:101580005B68204638490D22984705E023685B6870
:101590002046364907229847FB792BB123685B68C0
:1015A000204633491322984720460AF033FD01367E
:1015B0001835062EA2D1244C20460AF02BFD2368B4
:1015C0005B6820462B491022984720460AF022FDEE
:1015D000294B1B78002B32D00025DFF8AC80274F39
:1015E00023685B68204641460822984705EB85033F
:1015F000FE182046F95C0A2200230AF01BFD23682E
:101600005B6820461E4905229847204671780A22C9
:1016100000230AF00FFD23685B6820461949032266
:101620009847B078F1783279FFF722FE20460AF029
:10163000F1FC0135EDB2104B1B78AB42D0D802481B
:101640000AF0E8FCBDE8F88314DDFF1F3400010058
:1016500068C9FF1F500001005C0001006800010024
:101660007C0001008400010094000100A40001003E
:10167000AC000100C000010064C9FF1F38BEFF1F9D
:10168000D4000100B8FC000044000100BC040100CB
:1016900070B5054610B1441EE4B200E000244B1EB4
:1016A000052B00F22581DFE813F0060028004A0030
:1016B0008800B200FF002C208E4B00FB043005F0A8
:1016C000E7FB8D4B1B78002B00F012818B4C2368BD
:1016D0005B6820468A4906229847204629460A2206
:1016E00000230AF0A7FC23685B6820468549032293
:1016F000984720460AF08EFC70BD2C207D4B00FBE5
:10170000043005F0CFFB7C4B1B78002B00F0F08001
:101710007A4C23685B682046794906229847204620
:1017200029460A2200230AF085FC23685B682046CC
:1017300075490422984720460AF06CFC70BD2C22A3
:101740006C4B02FB0434204605F05AFB6A4B1B78B5
:10175000002B00F0CD80204605F014FBB0B1674CA3
:1017600023685B682046664906229847204629463A
:101770000A2200230AF05EFC23685B682046634966
:101780000A22984720460AF045FC70BD5B4C23684E
:101790005B6820465A4906229847204629460A2275
:1017A00000230AF047FC23685B68204658490B2257
:1017B000984720460AF02EFC70BD564B6200111966
:1017C00003EB41010B462C204A4A00FB04204988C8
:1017D0009A8805F09FFB484B1B78002B00F088800F
:1017E000464C23685B6820464549062298472046B8
:1017F00029460A2200230AF01DFC23685B68204664
:1018000045490F22984720460AF004FC70BD2C265B
:10181000384B06FB0436304605F000FB18B1304665
:1018200005F02EFB0AE03B4B6200111903EB41016E
:101830000B46304649889A8805F06CFB2E4B1B7886
:10184000002B55D0304605F0E9FAB0B12B4C236897
:101850005B6820462A4906229847204629460A22E4
:1018600000230AF0E7FB23685B6820462A490F2221
:10187000984720460AF0CEFB70BD204C23685B6879
:1018800020461F4906229847204629460A2200235F
:101890000AF0D0FB23685B68204620490E22984757
:1018A00020460AF0B7FB70BD04EB44022C20114B1C
:1018B00000FB0430174B33F8121005F0DBFA0E4B27
:1018C0001B78ABB10D4C23685B6820460C4906229F
:1018D0009847204629460A2200230AF0ABFB2368DA
:1018E0005B6820460E490622984720460AF092FB84
:1018F00070BD00BFE8C5FF1F339AFF1F14DDFF1F37
:10190000A8FD0000DC000100E0000100E80001008B
:10191000F400010024BEFF1F0001010010010100BE
:10192000200101002DE9F843144E06F1080406F1E8
:1019300080094FF00208002540F2DC5714F8080C2B
:10194000414608F039FE04F8075C24F8067C24F8C8
:10195000047C04F8025C357204F8015C03237372A2
:1019600086F80A80F560A560257301236373A5736B
:10197000183618344C45E1D1BDE8F88368C9FF1F1B
:1019800010B50F4C20780F49042208F055FE207E38
:101990000D49042208F050FE94F830000B4904224F
:1019A00008F04AFE94F848000949042208F044FE71
:1019B00094F860000749042208F03EFE10BD00BF05
:1019C00068C9FF1F891A0000951A0000A11A0000BB
:1019D000AD1A0000B91A000008B5134B1878222878
:1019E00028BFFF2008F05CFD0F4B187E222828BF7F
:1019F000FF2008F055FD0C4B93F83000222828BF3B
:101A0000FF2008F04DFD084B93F84800222828BF1E
:101A1000FF2008F045FD044B93F86000222828BF02
:101A2000FF2008F03DFD08BD68C9FF1F70B50446E2
:101A300008F082FE054604EB4402114B03EBC2039F
:101A40009B79DBB90E4B13F8320008F0A7FD50B1BB
:101A500004EB44020A4B03EBC203DD6074B90122BC
:101A6000084B1A7070BD064B6200101903EBC000E2
:101A7000C668AE1B8680C5600122827170BD00BF42
:101A800068C9FF1F5BBFFF1F08B50020FFF7CEFF2F
:101A900008BD00BF08B50120FFF7C8FF08BD00BFA3
:101AA00008B50220FFF7C2FF08BD00BF08B503203C
:101AB000FFF7BCFF08BD00BF08B50420FFF7B6FF65
:101AC00008BD00BF10B5104B1B78012B03D073B1BC
:101AD000022B04D012E00D4805F0DAF90EE00B4CB1
:101AE000204605F0DFF9204605F036FA06E0074CFF
:101AF000204605F0D7F9204605F026FA024B1A7861
:101B0000034B1A7010BD00BFE0C9FF1F2CBFFF1FA1
:101B100019C0FF1F2DE9F04182B0234B1B680093D1
:101B2000009A224B1B68D31A642B3AD91E4B1B68B0
:101B30000193019A1D4B1A6008F0FEFD4FF08042A0
:101B40001B4B1A6072B61B4E06F1100233468836E4
:101B50000024194D4FF00208A4461969411AA94200
:101B600009D90134E4B212F80F1C012904BF02F8AC
:101B70000F8C83F814C018321833B242EDD162B61C
:101B80004FF080420D4B1A60052C02D102220C4B03
:101B90001A700B4B1A780B4B1B789A4201D0FFF747
:101BA00091FF02B0BDE8F08150DBFF1FACBDFF1F0D
:101BB00088E100E068C9FF1FA086010008E100E09D
:101BC000E0C9FF1F19C0FF1F2DE9F00F82B080464A
:101BD00000EB40025D4B03EBC2035F8893F8099072
:101BE000C7F57A75002DB8BF6D424E46B9F1010FA9
:101BF0004BDD0022012342F20F719446A9F1020449
:101C0000DFF858B1DFF858A15148CDF80480042C12
:101C10002FD8DFE804F0030C151D26004D491144B0
:101C2000B1F90210C91B0029B8BF494221E04A4955
:101C30001144B1F90210C91B0029B8BF494218E08C
:101C40008118B1F90210C91B0029B8BF494210E040
:101C50000AEB0201B1F90210C91B0029B8BF4942C1
:101C600007E00BEB0201B1F90210C91B0029B8BF54
:101C70004942A942BCBF5FFA83FC0D4601330232E0
:101C8000B342C4DBDDF8048001E04FF0000C0CF13E
:101C9000010C5FFA8CF008EB48082C4B03EBC808EA
:101CA00098F80730002B4DD0A9F10209B9F1040FC3
:101CB00048D8DFE809F003080E182200012814BFF5
:101CC000012002203EE0012825D0032808BF012082
:101CD00038E0012821D0022821D0032821D004286F
:101CE00008BF01202EE001281DD002281DD00428A5
:101CF0001DD0052808BF012024E0012819D00228A2
:101D000019D0032819D0042819D0052819D006287D
:101D100008BF012016E0032014E0042012E0032095
:101D200010E002200EE005200CE004200AE0022072
:101D300008E0062006E0052004E0042002E003207D
:101D400000E0022002B0BDE8F00F704768C9FF1F35
:101D50009006010088FB00008CFB000094FB000053
:101D60009806010042780378134482781344C278BD
:101D70001344007903F07F03984214BF0020012030
:101D8000704700BF08B50138052820D8DFE800F00B
:101D900003070C11161B0E4808F062FD08BD44F63F
:101DA000206008F05DFD08BD42F2107008F058FD9B
:101DB00008BD41F2883008F053FD08BD40F2836051
:101DC00008F04EFD08BD40F6055008F049FD08BD7D
:101DD0008038010008B50648064B196805F0B2F9CD
:101DE0000548064B1988064A05F0B2FA08BD00BF3F
:101DF000D0C6FF1F549AFF1F0CB1FF1F9ACAFF1FC6
:101E0000B904000010B51E4B1B78DBB11D4B1868E0
:101E10001D4B1B68C01A0CF041F904461B4B188877
:101E20000CF038F91A490CF041FA014620460CF042
:101E30003DFA4FF07C510CF07DF80CF049FB154B4E
:101E4000186010BD104B18680E4B1B68C01A0CF0C0
:101E500025F904460D4B18880CF01CF90C490CF0C0
:101E600025FA014620460CF021FA4FF07C510CF087
:101E700061F80CF02DFB4042064B186010BD00BF0E
:101E800034CBFF1FB0A4FF1F549AFF1F04CBFF1FCA
:101E90000000A041A4B0FF1F38B5254B18780CF006
:101EA000F9F824490CF044F823490CF04BF90546A5
:101EB000224B18780CF0EEF81E490CF039F81E4948
:101EC0000CF040F904461E4B1B78C3B128461D494F
:101ED0000CF030F84FF07C510CF02CF80CF0F8FAC4
:101EE000194B1860204619490CF024F84FF07C512A
:101EF0000CF020F80CF0ECFA154B186038BD2846B1
:101F000012490CF017F84FF07C510CF013F80CF05C
:101F1000DFFA0D4B186020460A490CF00BF84FF021
:101F20007C510CF007F80CF0D3FA094B186038BD5F
:101F3000ACA4FF1F0000C8420000A040329AFF1F5F
:101F400034CBFF1F00007A44549AFF1F0000FA446C
:101F5000B0A4FF1F70B5FEF723FF514B0021597548
:101F600001229A7583F87510022183F876104D4B83
:101F700019705A709A70597103209871D9719872BA
:101F8000DA7204251D735A73D873197405245C74AE
:101F90009974D974187558759C75D9751A765D76CB
:101FA0009A760724DC761A775A779D77D87783F864
:101FB000204083F8211083F822203B4B1C703B4AC1
:101FC00040F2DC5313804FF47A6151804FF4FA648D
:101FD000148241F28833538240F6B83010844FF4B3
:101FE000FA5555844FF47A7515865486A2F8400048
:101FF000A2F84210A2F8503041F27073A2F85230A9
:10200000131D02F1080102F16400002201F8042C02
:1020100001F8032C5A601A81103310318342F5D134
:102020001922234B1A70234B4FF07C521A605A60CE
:102030009A60214D01262E700522204B1A70204BEC
:102040001E225A809A801A801A815A81DA80DA8197
:102050001A829A8100241B4B1C701B4B1C701B4B5B
:102060001C70C8221A4B1A804FF44872194B1A8000
:102070006423194A1370194A13704FF4FA62184B0B
:102080001A604FF47A72174B1A60FFF705FFFFF7DB
:10209000B9FE154B1E70154A154B1A602C7070BD99
:1020A00068C9FF1F38BEFF1F64C9FF1FACB0FF1F08
:1020B000D79CFF1F4098FF1FC89CFF1FC99CFF1F94
:1020C00024BEFF1F70B0FF1F30C0FF1F34CBFF1FA7
:1020D0009ACAFF1F04CBFF1FACA4FF1F329AFF1F39
:1020E000549AFF1FB0A4FF1F00BEFF1FC0D4010001
:1020F000E4C9FF1F2DE9F04F85B0AA4FAA4EAB4DA2
:102100004FF05008CDF80080A94C04F1160301935C
:1021100038463146A74A2B4604F0E4FDCDF800804E
:1021200004F12E03019338463146A34A2B4604F0AE
:10213000D9FDCDF8008004F14603019338463146BD
:102140009E4A2B4604F0CEFDCDF8008004F15E03DC
:102150000193384631469A4A2B4604F0C3FDCDF828
:10216000008004F17603019338463146954A2B46A8
:1021700004F0B8FD04F17801234600209A7D02B1F5
:10218000587518338B42F9D1DFF818828E4F874E7D
:102190004FF05009CDF80090854DEB1D019340465E
:1021A00039468A4A334604F05DFDCDF8009005F1CA
:1021B0001F03019340463946854A334604F052FDD9
:1021C000CDF8009005F13703019340463946814A26
:1021D000334604F047FDCDF8009005F14F0301931D
:1021E000404639467C4A334604F03CFDCDF8009029
:1021F00005F16703019340463946784A334604F0B7
:1022000031FD6B7D53B1CDF8009005F109030193C9
:1022100040467349734A334604F064FD644B93F8B7
:102220002D304BB1502300936F4B01935D486C49A7
:102230006E4A5E4B04F056FD5D4B93F845304BB152
:10224000502300936A4B019356486549694A574B9E
:1022500004F048FD564B93F85D304BB1502300938A
:10226000654B01934F485E49644A504B04F03AFD78
:102270004F4B93F875304BB150230093604B019353
:10228000484857495F4A494B04F02CFDFEF788FD4A
:10229000A1460B254FF0010ADFF888B1DFF8048171
:1022A000594F4E4699F81530002B4AD099F809300D
:1022B000002B46D0002400230393601980B202A9AA
:1022C0000A2208F0DBF802465023009303AB019387
:1022D00040463946354B04F039FD68B34B4B1B780B
:1022E0001E2B29D84A4803EB8301421800F801A0AD
:1022F000611C51700398ABFB00C1490B5FFA81FE72
:1023000082F802E089B2DFF820C10CFB0101DFF89E
:102310001CC1ACFB01C1C1F347111171CEEB0E1E04
:1023200000EB0E1001EB810EC1EBCE0100EB810141
:10233000D1700133354A13700134E4B2737AA34289
:10234000B9D80AF1010A5FFA8AFA09F118090A35BF
:10235000ADB2BAF1060FA4D1124D2E4F134C502638
:102360000096DFF8CC80CDF80480284639462A4A0A
:10237000234604F0DBFC009608F102030193284693
:102380003946264A234604F0D1FC009608F104039E
:10239000019328463946224A234604F063FC0096FE
:1023A00048E000BF08CAFF1F2801010034C0FF1F1A
:1023B00068C9FF1F380101004401010050010100FC
:1023C0005C01010068010100740101008801010045
:1023D00094010100A0010100AC010100B80101005D
:1023E000C4010100D801010089C9FF1FE0010100FB
:1023F000A1C9FF1FE8010100B9C9FF1FF0010100D9
:10240000D1C9FF1FF80101000002010064C9FF1FCC
:1024100038BEFF1F1802010028020100300201002F
:10242000380201005917B7D1F0D8FFFF1F85EB51D3
:10243000ACB0FF1F08F11003019328463946A24AA9
:10244000234604F073FC009608F11203019328461A
:1024500039469E4A234604F069FC009608F11403AD
:102460000193284639469A4A234604F0FBFB00961E
:1024700008F12003019328463946964A234604F082
:1024800055FC009608F12203019328463946924AEA
:10249000234604F04BFC009608F1240301932846E0
:1024A00039468E4A234604F0DDFB009608F13003DE
:1024B0000193284639468A4A234604F037FC0096A1
:1024C00008F13203019328463946864A234604F030
:1024D0002DFC009608F13403019328463946824AC0
:1024E000234604F0BFFB009608F140030193284601
:1024F00039467E4A234604F019FC009608F142034F
:102500000193284639467A4A234604F00FFC009688
:1025100008F14403019328463946764A234604F0DD
:10252000A1FB009608EB0603019328463946724A40
:10253000234604F0FBFB009608F152030193284662
:1025400039466E4A234604F0F1FB009608F1540325
:102550000193284639466A4A234604F083FB0096D5
:10256000684B019328463946674A234604F0BAFB74
:1025700004ABFF2203F8042D00960193284663491B
:10258000634A234604F0AEFB9DF80C00FF2809D0F7
:102590006428A8BF64200BF07DFD5E490BF086FE29
:1025A0005D4B186004ABFF2203F8042D502200920B
:1025B00001935A4855495A4A5A4B04F093FB9DF8E7
:1025C0000C00FF2809D06428A8BF64200BF062FD2E
:1025D00050490BF06BFE504B586004ABFF2203F8E0
:1025E000042D5022009201934C4848494E4A4D4BCD
:1025F00004F078FB9DF80C00FF2809D06428A8BFE0
:1026000064200BF047FD43490BF050FE424B9860AD
:10261000FF238DF80C30414D444F424C502600961C
:10262000DFF82C81CDF8048028463946404A2346FD
:1026300004F07CFB009608F102030193284639461A
:102640003C4A234604F072FB009608F10403019310
:1026500028463946384A234604F068FB009608F1BC
:102660000603019328463946344A234604F05EFBAC
:10267000009608F10803019328463946304A23465C
:1026800004F054FB009608F10A03019328463946EA
:102690002C4A234604F04AFB009608F10C030193F0
:1026A00028463946284A234604F040FB009608F1A4
:1026B0000E03019328463946244A234604F036FB8C
:1026C000009608F1100345E04002010048020100B5
:1026D000500201005802010060020100680201007E
:1026E00070020100780201008002010088020100EE
:1026F0009002010098020100A0020100A80201005E
:10270000B0020100D79CFF1FB8020100C402010003
:10271000CC0201000000C8424098FF1F08CAFF1FFA
:10272000D402010034C0FF1FDC020100E4020100FA
:10273000EC020100F8020100040301001003010093
:102740001C030100280301003403010040030100C1
:1027500024BEFF1F019328463946444A234604F00D
:10276000E5FA434F0096434B019328463946424AC7
:10277000234604F077FA0096404B019328463946E9
:102780003F4A234604F06EFA3E4F00963E4B0193BB
:10279000284639463D4A234604F064FA00963C4BED
:1027A0000193284639463B4A234604F0BFFA009677
:1027B000394B019328463946384A234604F0B6FA85
:1027C0000096374B019328463946364A234604F093
:1027D00089FA0096344B019328463946334A2346FA
:1027E00004F080FAFFF758FBFFF70CFB3048314B41
:1027F000196804F0A7FC304F0096304B019328462F
:1028000039462F4A234604F02DFA00962D4B0193AA
:10281000284639462C4A234604F098FA2B4F009656
:102820002B4B0193284639462A4A234604F01AFACC
:102830000096294E019628463946284A234604F038
:1028400051FA30780BF026FC25490BF02FFD254975
:102850000BF078FC4FF07C510BF06CFB0BF038FE6A
:10286000214B187005B0BDE8F08F00BF4C0301008C
:102870005803010070B0FF1F6403010030C0FF1F48
:10288000700301007C03010034CBFF1F84030100AF
:102890009ACAFF1F9403010004CBFF1FA00301008D
:1028A000ACA4FF1FAC030100329AFF1FB803010064
:1028B000D0C6FF1FB0A4FF1FCC02010000BEFF1F47
:1028C000C4030100E4C9FF1FD0030100DC030100C1
:1028D000C89CFF1FE8030100C99CFF1FF80301000B
:1028E0000000C84200007F4301A4FF1F054B1B7876
:1028F0001BB90122034B1A7070470022014B1A705A
:10290000704700BF09BEFF1F2DE9F04F83B0054699
:10291000894617469846467B002E00F08480444B3B
:102920001878DFF824B18BF80000424C4FF42C7A71
:102930000AFB004005F088F89BF800C00AFB0C4E2B
:102940000EF521740FCD0FC495E8030084E8030051
:1029500001228EF89C228EF89D928EF8AE8247B1AD
:102960000CEB8C0C344800EBCC00344904F006FE30
:1029700008E00CEB8C0C304800EBCC003049012215
:1029800004F0FCFDDFF8C08098F80000294C4FF4FB
:102990002C7505FB00F02118084601F5217105F0A2
:1029A0007FF898F80000274B1B680093009B05FBFD
:1029B0000044C4F8A032B4F8AA320133A4F8AA3211
:1029C00084F8AC02FDF742FFFFF790FF5FB3184BAE
:1029D0001A78184B05FB023005F0ECFA054610B3E7
:1029E000134C237803EB8303134800EBC300134914
:1029F000002204F0C3FD2378124A12680192019A62
:102A00004FF42C700B4900FB031302F5C872C3F896
:102A1000A42203F52A71012283F8A822002283F858
:102A20009D228A712E46304603B0BDE8F08F00BF6C
:102A300009BEFF1F84C0FF1F20B0FF1F16B7030091
:102A40005D74D10550DBFF1F20BEFF1F08B50B468C
:102A500000210122FFF758FF08BD00BF08B50B4653
:102A600001210A46FFF750FF08BD00BF08B50B461D
:102A700000210A46FFF748FF08BD00BF00B583B03C
:102A8000074B1878074B1B78013B00930021FF226E
:102A90000B4609F051FCC0B203B05DF804FB00BF67
:102AA0001AC0FF1FACBFFF1F10B5064C204604F034
:102AB000CBFF04F52C7004F0C7FF0022024B1A7004
:102AC00010BD00BF84C0FF1F09BEFF1F08B50B4B20
:102AD0001B78012B11D10A4B1B6873B1094A11688D
:102AE000002903DD084804F0BFFC08BD064819466C
:102AF000064A04F02DFC034B186008BDA0C6FF1F5A
:102B0000E4C9FF1F30CBFF1F0CB1FF1FD52B000006
:102B100010B5074B1B78012B09D1064B1B6833B14D
:102B2000054C0648216804F02DFC0023236010BDED
:102B3000A0C6FF1FE4C9FF1F30CBFF1F0CB1FF1F52
:102B400010B5174A137817490B701070834225D0BF
:102B5000022B01D1FFF7DCFF114B1B78022B01D1B7
:102B6000FFF7B4FF0E4B1B78012B09D10E4C2368E5
:102B70005B6820460D490C229847204609F04AFA26
:102B8000074B1B78082B09D1074C23685B6820464C
:102B900007490F229847204609F03CFA10BD00BFB4
:102BA000E9CAFF1F19CBFF1F14DDFF1F0804010036
:102BB0001804010008B5054B1B782BB1044B1B789A
:102BC00013B90120FFF7BCFF08BD00BFE8CAFF1F13
:102BD000E9CAFF1F08B5044B1B7813F0F70F02D0AA
:102BE0000820FFF7ADFF08BDE9CAFF1F08B5194B64
:102BF0001870194B1B78012B0DD1184B1B783BB368
:102C0000174B1B7853B1174B1B783BB903281FD9BF
:102C1000FFF7D0FF08BD114B1B78CBB1114B1B78D0
:102C2000012B15D9082B13D028B1022B10D103206A
:102C3000FFF786FF08BD052B03D10720FFF780FFB4
:102C400008BD033BDBB2012B02D80620FFF778FF5B
:102C500008BD00BF1AC0FF1FA0C6FF1FE8CAFF1FA4
:102C600000BEFF1FE9CAFF1F2DE9F04F89B0804663
:102C70000591029203939DF848200492437B0193AF
:102C8000002B00F0BB805F4B1B78002B00F0AE8068
:102C90000024214622465C4F5A4D002A41D14FF470
:102CA0002C7303FB047393F89C32002B39D14FF43F
:102CB0002C7A0AFB04FA07EB0A09484604F0C4FE22
:102CC00009F52176C646BEE80F000FC69EE8030050
:102CD00086E803004FF0010B89F89CB2029A89F84C
:102CE0009D22039A89F89E22002289F89F22049B44
:102CF00089F8AE32484609F5217104F0D1FE434A05
:102D000013680693069BC9F8A032B9F8AA325B444F
:102D1000A9F8AA3289F8AC422046FDF7EDFD21461C
:102D20005A460134E4B22B78A342B6D8002A53D1D4
:102D3000344B1B78002B5CD00024334F314D002ADC
:102D400044D14FF42C7303FB047393F8980298F862
:102D5000143098423AD24FF42C7B0BFB04FB07EB68
:102D60000B06304604F070FE06F5217EC446BCE832
:102D70000F00AEE80F009CE803008EE803004FF060
:102D8000010A86F89CA2029A86F89D22039A86F888
:102D90009E22002286F89F22049B86F8AE3230469F
:102DA00006F5217104F07CFE184A13680793079B0F
:102DB000C6F8A032B6F8AA325344A6F8AA3286F86A
:102DC000AC422046FDF798FD214652460134E4B25C
:102DD0002B78A342B3D87AB14FF42C720A4B02FB82
:102DE0000131D1F8AA32059A136007E0002301935C
:102DF00004E00022019201E000230193019809B050
:102E0000BDE8F08FDCA2FF1F3CB2FF1F50DBFF1FAD
:102E100000B585B00023009303A91A46FFF724FFED
:102E200005B05DF804FB00BF00B585B0009103A9B3
:102E300000221346FFF718FF05B05DF804FB00BF42
:102E400000B585B00B460022009203A90122FFF7CE
:102E50000BFF05B05DF804FB10B582B0144600937B
:102E600001222346FFF700FF02B010BD00B583B07A
:102E7000009200221346FFF7F7FE03B05DF804FB53
:102E800038B504460D464FF42C70134B00FB04304C
:102E900004F0DAFD114B1B785BB955B14FF42C727D
:102EA0000D4B02FB043393F89C3213B12046FDF71F
:102EB00079FD4FF42C70084B00FB0430002380F8A0
:102EC0009C3280F89D3280F89E3280F89F3280F8E4
:102ED000AE3280F8A83238BD3CB2FF1FB8C6FF1F23
:102EE00038B500242546E0B22946FFF7C9FF013472
:102EF000042CF8D138BD00BFF8B50746094D0024B1
:102F0000E6B22B7E33B1284639460CF09BF908B95E
:102F1000F0B205E0013405F52C75042CF0D1FF204A
:102F200040B2F8BDC0B4FF1F08B5022808D003287E
:102F30000BD001280DD107480921FFF775FF08BD07
:102F400005480A21FFF770FF08BD04480B21FFF771
:102F50006BFF08BDE4A0FF1FFCA0FF1F14A1FF1F13
:102F600008B50248FFF754FF08BD00BF2CA1FF1FA2
:102F700008B50248FFF74CFF08BD00BF44A1FF1F82
:102F800008B50248FFF744FF08BD00BF5CA1FF1F62
:102F900008B50248FFF73CFF08BD00BF74A1FF1F42
:102FA00008B5022807D0032809D001280AD106480D
:102FB000FFF72EFF08BD0548FFF72AFF08BD0448AC
:102FC000FFF726FF08BD00BF8CA1FF1FA4A1FF1FB4
:102FD000BCA1FF1F08B50146012803D10348FFF734
:102FE00017FF08BD0148FFF72BFF08BDECA1FF1F2D
:102FF00008B50248FFF70CFF08BD00BF04A2FF1F81
:1030000008B518B10348FFF703FF08BD0248FFF7F2
:10301000FFFE08BD1CA2FF1F34A2FF1F2DE9F043D5
:1030200083B0F8B13F4B1B78002B78D13E4B93F81F
:10303000E5304BB13D483E490322FFF717FF68B129
:103040000122384B1A7009E03A48394900221346E8
:10305000FFF702FF10B10122324B1A700022364BEB
:103060001A705CE02F4B1B78002B58D0324B1B782A
:10307000002B54D12C4B93F81531002B45D02C4B01
:1030800093F902204FF42C702C4900FB0211B1F887
:10309000AA121B88994204D1284B00FB023004F08D
:1030A000D3FC4FF0010C244B83F800C0DFF8809074
:1030B00099F902E0214F4FF42C7808FB0EFE07EB44
:1030C0000E0606F521741E4D0FCD0FC495E80300C2
:1030D00084E8030086F89CC2002286F89D2204231F
:1030E00086F8AE32304606F5217104F0D9FC99F825
:1030F0000200144B1B680193019B42B208FB02774C
:10310000C7F8A032FDF7F8FB09E0094B98780021D9
:10311000FFF7B6FE0023034A1370074A137003B08B
:10312000BDE8F0839CC6FF1F349FFF1F0CA0FF1F4C
:1031300004BDFF1F24A0FF1FD0BEFF1F3CB2FF1F16
:103140003CA0FF1F50DBFF1F2DE9F04383B0F8B117
:103150003F4B5B78002B78D13E4B93F82D314BB130
:103160003D483E490522FFF781FE68B10122384BF8
:103170005A7009E03A48394900221346FFF76CFEBD
:1031800010B10122324B5A700022364B5A705CE06B
:103190002F4B5B78002B58D0324B5B78002B54D1EF
:1031A0002C4B93F85D31002B45D02C4B93F902202A
:1031B0004FF42C702C4900FB0211B1F8AA121B88A5
:1031C000994204D1284B00FB023004F03DFC4FF043
:1031D000010C244B83F801C0DFF8809099F902E0DC
:1031E000214F4FF42C7808FB0EFE07EB0E0606F578
:1031F00021741E4D0FCD0FC495E8030084E8030031
:1032000086F89CC2002286F89D22062386F8AE32FC
:10321000304606F5217104F043FC99F80200144B86
:103220001B680193019B42B208FB0277C7F8A032EA
:10323000FDF762FB09E0094B98780021FFF720FEBB
:103240000023034A5370074A537003B0BDE8F0836C
:103250009CC6FF1F349FFF1F54A0FF1F60C9FF1FA4
:103260006CA0FF1FD0BEFF1F3CB2FF1F84A0FF1F3A
:1032700050DBFF1F2DE9F04383B0F8B13F4B9B7843
:10328000002B78D13E4B93F875314BB13D483E4908
:103290000722FFF7EBFD68B10122384B9A7009E075
:1032A0003A48394900221346FFF7D6FD10B10122F2
:1032B000324B9A700022364B9A705CE02F4B9B7811
:1032C000002B58D0324B9B78002B54D12C4B93F8C9
:1032D000A531002B45D02C4B93F902204FF42C70D4
:1032E0002C4900FB0211B1F8AA121B88994204D1A3
:1032F000284B00FB023004F0A7FB4FF0010C244BDD
:1033000083F802C0DFF8809099F902E0214F4FF472
:103310002C7808FB0EFE07EB0E0606F521741E4DF9
:103320000FCD0FC495E8030084E8030086F89CC223
:10333000002286F89D22082386F8AE32304606F534
:10334000217104F0ADFB99F80200144B1B68019346
:10335000019B42B208FB0277C7F8A032FDF7CCFA16
:1033600009E0094B98780021FFF78AFD0023034A02
:103370009370074A937003B0BDE8F0839CC6FF1FAB
:10338000349FFF1F9CA0FF1F94BDFF1FB4A0FF1F11
:10339000D0BEFF1F3CB2FF1FCCA0FF1F50DBFF1FA2
:1033A00008B5022807D0032809D001280AD1084609
:1033B000FFF734FE08BD0846FFF7C6FE08BD084605
:1033C000FFF758FF08BD00BFF0B583B0002845D017
:1033D000644B1B78002B40F0C280634B1B78002BA2
:1033E00040F0B180614B93F85530002B00F0B18074
:1033F0005F4860490122FFF739FD002800F0AF80E7
:103400000122584B1A70AAE058485A490122FFF786
:103410002DFD002800F0A3800122524B1A709EE07F
:10342000524B93F86D3063B1534852490022134612
:10343000FFF712FD002800F092800122494B1A701C
:103440008DE04E484B4900221346FFF705FD00284A
:1034500000F085800122434B1A7080E0414B1B78BD
:10346000002B7CD0404B1B781BB9404B93F8853028
:1034700023B93E4B93F83D30002B5BD03D4B93F985
:1034800002204FF42C703E4900FB0211B1F8AA1241
:103490001B88994204D13A4B00FB023004F0D4FA65
:1034A000314B1B788BB1334B93F902204FF42C74C2
:1034B000334B04FB023404F52174324D0FCD0FC49D
:1034C00095E8030084E8030010E02A4B93F90220FA
:1034D0004FF42C742A4B04FB023404F521742A4D5A
:1034E0000FCD0FC495E8030084E80300214F97F93E
:1034F0000230234D4FF42C7606FB03F3E81801212C
:1035000080F89C12002480F89D4280F8AE4200F5BD
:10351000217104F0C5FAB8781C4B1B680193019B1C
:1035200042B206FB0255C5F8A0320E4B1C70FDF7E7
:10353000E3F914E00F4B98780121FFF7A1FC00227A
:10354000084B1A700BE0094B5B7B002B3FF479AF03
:103550005AE7064B5B7B002B3FF462AF54E703B0A6
:10356000F0BD00BF71B0FF1FA9BDFF1F349FFF1F3B
:103570007C9FFF1FB0BFFF1F949FFF1F4C9FFF1F2B
:103580003CB2FF1F649FFF1FAC9FFF1F50DBFF1F5C
:103590002DE9F04383B0F0B13A4B1B78002B6ED18C
:1035A000394B93F89D3053B1384839490222FFF71F
:1035B0005DFC002863D00122324B1A705FE0354871
:1035C000334900221346FFF747FC002857D0012259
:1035D0002C4B1A7053E02B4B1B78002B4FD02A4BEF
:1035E00093F8CD30002B42D0294B93F902204FF4B1
:1035F0002C70294900FB0211B1F8AA121B889942CC
:1036000004D1254B00FB023004F01EFADFF8809055
:1036100099F902E0204F4FF42C7808FB0EFE07EBDF
:103620000E0606F521741D4D0FCD0FC495E803005D
:1036300084E80300012286F89C22002486F89D423B
:1036400086F8AE42304606F5217104F029FA99F861
:103650000200134B1B680193019B42B208FB0277E7
:10366000C7F8A032074B1C70FDF746F907E0084B7E
:1036700098780121FFF704FC0022024B1A7003B076
:10368000BDE8F08318CBFF1F349FFF1FC49FFF1FAF
:1036900000BDFF1FDC9FFF1F3CB2FF1FF49FFF1FF9
:1036A00050DBFF1F08B568B10C4B1B786BB90C4899
:1036B0000C4900221346FFF7CFFB70B10122074BE4
:1036C0001A7008BD054B1B783BB1064B9878012159
:1036D000FFF7D6FB0022014B1A7008BD0ABEFF1F80
:1036E000D4A1FF1F28BFFF1F0139C9B2052909D87E
:1036F000090100EB800000EB8000400000F5FA704B
:10370000014B5852704700BFACB0FF1F0139C9B21E
:1037100005290AD8054B03EB011100EB800000EBF3
:103720008000400000F5FA7048807047ACB0FF1F81
:103730000139C9B2052909D8054B03EB0111003045
:1037400018BF012008710122024B1A70704700BF98
:10375000ACB0FF1F59BFFF1F08B5074B1B7853B90B
:10376000064840F6B831064A03F0F2FD054B1860F2
:103770000122014B1A7008BD9CAFFF1F0CB1FF1F47
:103780003138000008BDFF1F10B5154A00235371E2
:10379000537582F8253082F8353082F8453082F84A
:1037A0005530104A13701048104B196803F06EFE24
:1037B00020B10D480D4B196803F0E4FD0C4B1B784C
:1037C00063B10C4B1B784BB10B4C23685B682046F4
:1037D0000A490C229847204608F01CFC10BD00BF87
:1037E000ACB0FF1F9CAFFF1F0CB1FF1F08BDFF1F38
:1037F000339AFF1F59BFFF1F14DDFF1F280401006C
:1038000010B582B0084B1B6801930199074A00016B
:10381000131803F108049960105A598808F082FDC2
:10382000A08002B010BD00BF50DBFF1FACB0FF1F77
:103830002DE9F041164B1B783BB3164E002425466C
:10384000154F4FF00108E8B23B191A7942B15A7985
:1038500032B996F825231AB183F80580FFF7D0FF17
:10386000013510341836602CEDD10C4B1B7863B148
:103870000B4B1B784BB10B4C23685B6820460A4905
:103880000D229847204608F0C5FBBDE8F08100BF37
:103890009CAFFF1F349FFF1FACB0FF1F339AFF1F69
:1038A00059BFFF1F14DDFF1F3804010010B5044687
:1038B000094B03EB00135B796BB1213000EB400047
:1038C000064B03EBC000FFF7A3FA2046FFF798FF73
:1038D0002046FDF7BDF810BDACB0FF1F349FFF1FA1
:1038E00070B582B00B4D00240B4EE0B22B785BB16B
:1038F00033680193019AD5F80330D31AB5F807203D
:10390000934201D3FFF7D2FF01341035062CECD1DE
:1039100002B070BDB1B0FF1F50DBFF1FF0B583B028
:103920000446234B1B788B2B06D8591C204A117058
:10393000204A42F8230009E01F4D2B685B682846A7
:103940001E493C229847284608F064FB204605F0B3
:10395000DFF920B31A4D284604F076F828462146B0
:1039600004F09EF8174B1B680093009F154E2846E5
:1039700004F020FB18B1284604F032FB20612369D3
:103980008BB933680193019BDB1B052BEFD908E052
:10399000012565730A4804F057F8284606E0002020
:1039A00004E0002002E0322BF2D8002003B0F0BD8A
:1039B00098CAFF1FD8C6FF1F14DDFF1F480401006F
:1039C0003CB2FF1F50DBFF1F08B5FFF789FAFFF776
:1039D0006BF808BDF8B505460E4617461268A2B941
:1039E000002923DD00210C464FF0FF305A7B22B125
:1039F0006C503A6801323A6000E068500134183384
:103A00000431B442F2D13B689BB1304608F07EFCF1
:103A100055F82030B3F1FF3FF7D03A68013A3A60E9
:103A20004FF0FF3245F820201846F8BD4FF0FF3028
:103A3000F8BD4FF0FF30F8BD08B503480521034A33
:103A4000034BFFF7C7FF08BD6CC6FF1FB4C6FF1FBF
:103A500034A4FF1F2DE9F04F87B0704D05F5217498
:103A600005F2E476DFF8CC81DFF8CCA1DFF8CC9169
:103A70002746237E002B00F0C78094F82A30042BC1
:103A800000F2C280DFE803F08E032E4E7C00284651
:103A900004F090FA002800F0B780284604F092FA6B
:103AA0002369A3F5C8739842C0F0AE805C4B1B78C5
:103AB00053B15C4B5B7B3BB15A480021FEF7CEFF14
:103AC0000220FFF73DF89FE0FFF7B6FF00EB400054
:103AD000554B03EBC0000021FEF7C0FF0220FFF7AB
:103AE0002FF891E0284604F065FA002800F08C8059
:103AF000284604F067FA2369A3F5C8739842C0F01A
:103B00008380FEF7BBFF074600EB4000474B03EB0B
:103B1000C0000321FEF7A2FF454B1F700520FFF7F1
:103B20000FF871E099F80030052B6DD1FEF7A6FF74
:103B300083463F4B1B7883420BD000EB40003B4B4E
:103B400003EBC0000321FEF789FF394B83F800B077
:103B50005AE0284604F02EFA002855D1D8F8003053
:103B60000093009AE369D31A042B4DD928462146C5
:103B700003F096FFD8F800300193019BE36143E026
:103B8000284604F017FA00283ED1D8F800300293F6
:103B9000029AE369D31A042B36D9002323768AF8D4
:103BA000003031E0AB46284604F004FAA8B9D8F852
:103BB00000300393039AE369D31A042B0DD9637E73
:103BC0004BB12846214603F06BFFD8F80030049330
:103BD000049BE36101E000232376584604F0EAF9F0
:103BE00090B13B7E83B197F824306BB1D8F80030A8
:103BF0000593059A3B6A934206D0584603F024FF8A
:103C000000233B7687F8243005F52C7504F52C74D9
:103C1000B4427FF42DAF07B0BDE8F08F84C0FF1F22
:103C200031C0FF1F04A4FF1F34A4FF1F10A3FF1FF8
:103C300008BEFF1F50DBFF1FA9BDFF1FE9CAFF1F02
:103C400008B503480521034A034BFFF7C3FE08BD2F
:103C50001CCBFF1FF0C9FF1F589AFF1F08B5034870
:103C60000521034A034BFFF7B5FE08BD0CBEFF1F3D
:103C700038B2FF1FD89CFF1F08B5554B1B78013B7E
:103C8000072B00F2A480DFE803F004A24DA2A234C7
:103C9000709B504B1B78002B40F09980FEF704FF7F
:103CA0004D4B1B787BB14D4B5B7B23B14B480121C6
:103CB000FEF7DCFE16E04A4B5B7B9BB148480121D6
:103CC000FEF7D4FE0EE0464B5B7B23B14448012156
:103CD000FEF7CCFE06E0414B5B7B1BB13F48012168
:103CE000FEF7C4FE00223C4B1A700122394B1A70B9
:103CF00008BD3C4B1B783BB13B4B5B7B23B13A4847
:103D00000021FEF7ABFE09E0FFF796FE00EB400056
:103D1000364B03EBC0000021FEF7A0FE0220FEF7A9
:103D20000FFF08BDFFF78CFFC0B2314B187010F0C9
:103D3000800F0CD140B200EB40002E4B03EBC000D3
:103D40000221FEF783FE0420FEF7FAFE08BDFEF70F
:103D500095FE00EB4000284B03EBC0000321FEF76B
:103D60007DFE0520FEF7ECFE08BDFFF777FFC0B231
:103D7000224B187010F0800F09D140B200EB4000C8
:103D80001F4B03EBC0000121FEF760FE14E0154B52
:103D90001B783BB1144B5B7B23B113480021FEF72A
:103DA0005DFE09E0FFF748FE00EB40000F4B03EB20
:103DB000C0000021FEF752FE0220FEF7C1FE08BD42
:103DC00010480421FEF742FE0020FEF7B9FE08BDB0
:103DD000E9CAFF1FA9BDFF1F319AFF1F1CA4FF1FC7
:103DE000349AFF1F31C0FF1F04A4FF1F34A4FF1F1C
:103DF000A4A5FF1F589AFF1F10A3FF1FAFA4FF1F0A
:103E0000D89CFF1FB09CFF1F044B1B78022B0CBFDC
:103E100003220222014B1A70704700BFAEA4FF1F9D
:103E20002DE9F04F83B00546894617469846467BF4
:103E3000002E00F08980464B1878DFF82CB18BF803
:103E40000000444C4FF42C7A0AFB004003F0FCFDC8
:103E50009BF800C00AFB0C4E0EF521740FCD0FC469
:103E600095E8030084E8030001228EF89C228EF876
:103E70009D928EF8AE8257B1ACF1020C0CEB8C0C1B
:103E8000354800EBCC00354903F078FB0AE0ACF193
:103E9000020C0CEB8C0C304800EBCC0030490122BA
:103EA00003F06CFBDFF8C08098F80000294C4FF459
:103EB0002C7505FB00F02118084601F5217103F06F
:103EC000EFFD98F80000274B1B680093009B05FB53
:103ED0000044C4F8A032B4F8AA320133A4F8AA32DC
:103EE00084F8AC02FCF708FDFFF78EFF67B3184BB0
:103EF0001A78184B05FB023004F05CF8054618B33D
:103F0000134C2378023B03EB8303134800EBC300FD
:103F10001249002203F032FB2378124A1268019200
:103F2000019A4FF42C700B4900FB031302F5C87281
:103F3000C3F8A42203F52A71012283F8A8220022E3
:103F400083F89D228A712E46304603B0BDE8F08F7B
:103F5000AEA4FF1F3CB2FF1FC4BFFF1F16B7030074
:103F60005D74D10550DBFF1F309AFF1F08B50B466B
:103F700000210122FFF754FF08BD00BF08B50B4622
:103F800001210A46FFF74CFF08BD00BF08B50B46EC
:103F900000210A46FFF744FF08BD00BF054B18701B
:103FA00018B10122044B1A7070470022024B1A709C
:103FB000704700BF0CBDFF1F20BDFF1F00B583B0C1
:103FC000074B1878074B1B78013B00930021FF2219
:103FD0000B4608F0B1F9C0B203B05DF804FB00BFB6
:103FE0000CBDFF1F9DAFFF1F08B502200021FEF78B
:103FF00047FF03200021FEF743FF0222014B1A7006
:1040000008BD00BFAEA4FF1F08B51D4B1B78002BD9
:1040100035D01C4B1B7873BB1B4B1B787BB3022228
:104020001A4B1A70FFF7E0FF194B5B7B23B118485E
:104030000121FFF7ABFF09E0FFF7C0FF00EB4000F5
:10404000144B03EBC0000221FFF798FF01220D4B38
:104050001A7010E0104B5B7B23B10F480321FFF770
:1040600085FF04E0FFF7C0FF0422084B1A7000220E
:10407000044B1A7008BD044B1B78002BEAD008BD16
:104080005ABFFF1FA9B0FF1F20BDFF1FDCA2FF1FEB
:10409000F8A2FF1FB4A4FF1FE0A2FF1F2DE9F04FFD
:1040A00087B05C4B03F5AC6403F2E47503F52C6751
:1040B000DFF86891DFF868A1DFF86881264694F898
:1040C0009C22002A00F09B8094F8AE32032B00F271
:1040D0009680DFE803F05C021D48204603F06AFF8B
:1040E000002800F08C80204603F06CFFD4F8943256
:1040F000A3F5C8739842C0F08280FFF75FFF00EB22
:104100004000454B03EBC0000221FFF737FF76E08C
:10411000FFF754FF834698F8003083420AD000EB43
:1041200040003D4B03EBC0000221FFF727FF88F85A
:1041300000B064E0204603F03DFF00285FD1D9F8CD
:1041400000300093009AD4F8A032D31A042B56D929
:104150002046294603F0A4FCD9F800300193019BC6
:10416000C4F8A0324BE0204603F024FF002846D1DB
:10417000D9F800300293029AD4F8A032D31A042B53
:104180003DD9FFF731FF04238AF8003037E020469D
:1041900003F010FFC8B9D9F800300393039AD4F89C
:1041A000A032D31A042B10D994F89D3253B1204673
:1041B000294603F075FCD9F800300493049BC4F839
:1041C000A03202E0002384F89C32304603F0F2FE75
:1041D000A8B196F89C3293B196F8A8327BB1D9F881
:1041E00000300593059AD6F8A432934207D03046A2
:1041F00003F02AFC002386F89C3286F8A83204F5E6
:104200002C7405F52C75BC427FF458AF07B0BDE89F
:10421000F08F00BF3CB2FF1FB4A4FF1F50DBFF1F95
:10422000DCA2FF1F5CC9FF1FF8B50D461746142816
:1042300024D80138C4B204EB4406114B03EBC60684
:104240003046FEF759FE9DB1002817DA47B13046D7
:104250000C4901EB840100221346FEF7FDFDF8BD79
:104260003046084901EB84010022FEF7FFFDF8BD4E
:10427000002803DBC0B20121FEF702FEF8BD00BF3B
:104280005098FF1FD4BEFF1F08B503481421034AEE
:10429000034BFFF79FFB08BDB0BDFF1F9CCAFF1F6C
:1042A000549DFF1F08B503481421034A034BFFF731
:1042B00091FB08BD5CBFFF1FDCAFFF1FD09AFF1F43
:1042C000F8B510B1012804D02AE01A4B1E8898785E
:1042D00002E0194B1E88987810F0800F22D1174BFE
:1042E0001A780AB3164B03F52C74013AD2B24FF484
:1042F0002C7101FB024147B293F89C425CB1B3F8C8
:10430000AA52B54207D193F9AC22BA4203D1002197
:10431000FEF7B6FD0BE003F52C738B42ECD105E004
:10432000002404E0002402E0002400E000242046F1
:10433000F8BD00BFD09CFF1F4C9AFF1FDCA2FF1FDF
:104340003CB2FF1F10B50446FFF7BAFF40BB14B1E3
:10435000012C13D010BD134B1B780BB3124B1B68F1
:1043600003EB4303114800EBC3001149114B1A78CA
:10437000FEF77CFD0122104B1A7010BD0F4B1B780D
:1043800073B10F4B1B6803EB43030E4800EBC300F4
:104390000D490E4B1A78FEF769FD01220C4B1A707D
:1043A00010BD00BFA0CAFF1F1CC0FF1F549DFF1FF0
:1043B000D09CFF1FCA9CFF1F1ACBFF1F24BFFF1FEB
:1043C000ECCAFF1FD09AFF1F4C9AFF1FD69CFF1FFD
:1043D00048C9FF1FF8B5054610B1012811D0F8BD36
:1043E0004E4B1B78002B00F098804D4B1F684D4BB7
:1043F0001B78002B40F0888001224A4B1A704A4EED
:104400007DE04A4B1B78002B00F08780484B1F68EB
:10441000484B1B78002B79D10122464B1A70464E2F
:104420006DE0122F77DC7C1CE4B2132C2BD804EB4C
:10443000440306EBC3035B7B0BB315B1012D0FD017
:104440001DE004EB4400384B03EBC0003B490C2259
:10445000FEF70CFD324B1C600C22394B1A70F8BD74
:1044600004EB4400344B03EBC00036490F22FEF747
:10447000FDFC2F4B1C600F22334B1A70F8BD01342A
:10448000E4B2132CD3D9002F2EDD0024234603EBF6
:10449000430206EBC202527B0AB315B1012D0FD0C5
:1044A0001DE004EB4400204B03EBC00023490C2229
:1044B000FEF7DCFC1A4B1C600C22214B1A70F8BD75
:1044C00004EB44001C4B03EBC0001E490F22FEF717
:1044D000CDFC174B1C600F221B4B1A70F8BD01332B
:1044E000DBB21C46BB42D2DB184C23685B6820461B
:1044F000174925229847204607F08CFDF8BD28462D
:10450000FFF7DEFE3FB18CE7074E00E00A4E28467B
:10451000FFF7D6FE85E7002489E7F8BDA0CAFF1F94
:104520001CC0FF1F1ACBFF1F549DFF1F24BFFF1F7E
:10453000ECCAFF1F48C9FF1FD09AFF1FD09CFF1F66
:10454000CA9CFF1F4C9AFF1FD69CFF1F14DDFF1F44
:104550008804010070B5054610B101280BD070BD6C
:10456000244B1B78002B44D0234B1C680122234B87
:104570001A70234E09E0234B1B78002B39D0224BB5
:104580001C680122214B1A70214E2846FFF798FE25
:10459000002CC6BF04F1FF34E4B2132404EB44033F
:1045A00006EBC3035B7B0BB315B1012D0FD01DE0F0
:1045B00004EB4400124B03EBC00016490D22FEF73A
:1045C00055FC0D4B1C600D22134B1A7070BD04EB93
:1045D00044000F4B03EBC00010491022FEF746FCCD
:1045E000094B1C6010220E4B1A7070BD013CE4B2E6
:1045F000D4E770BDA0CAFF1F1CC0FF1F1ACBFF1F4E
:10460000549DFF1F24BFFF1FECCAFF1F48C9FF1F97
:10461000D09AFF1FD09CFF1FCA9CFF1F4C9AFF1F00
:10462000D69CFF1F10B50446FFF74AFE14B1012CBB
:1046300014D010BDFFF728FE124B186000EB4000AD
:10464000114B03EBC00011490E22FEF70FFC0E22A6
:104650000F4B1A7001220F4B1A7010BDFFF722FE8C
:104660000D4B186000EB40000C4B03EBC0000C49F5
:104670001122FEF7FBFB11220A4B1A7001220A4B92
:104680001A7010BD1CC0FF1F549DFF1FD09CFF1F40
:10469000CA9CFF1F1ACBFF1FECCAFF1FD09AFF1F37
:1046A0004C9AFF1FD69CFF1F48C9FF1F2DE9F043FE
:1046B00089B0C54B1B78002B00F023820024C34D2A
:1046C000C34F26464FF42C7303FB045393F89C32DC
:1046D000002B00F00F824FF42C7808FB0458404662
:1046E00003F068FC002840F00582BA4B1B68009379
:1046F000009AD8F8A032D31A042B40F2FB8198F824
:10470000AE32013B102B00F29E81DFE813F0110066
:1047100055009300BC00C600EF00F90022017E00A6
:1047200085008C002C013C014C016F017E018D0144
:10473000A94B1B789BB997F86D3083B14FF42C7E51
:104740000EFB045E0EF5217E07F1600CBCE80F0045
:10475000AEE80F009CE803008EE803000FE04FF482
:104760002C7E0EFB065E0EF5217E07F1180CBCE8D0
:104770000F00AEE80F009CE803008EE803004FF442
:104780002C7303FB06F6A919404601F5217103F0CD
:1047900087F9904B1B680193019B2E44C6F8A03209
:1047A000012386F89D32002386F89E3286F8AE32C9
:1047B0002046FCF7A1F89DE14FF42C7303FB04F6AF
:1047C00005EB060909F5217E07F1A80CBCE80F00EE
:1047D000AEE80F009CE803008EE80300404609F5B0
:1047E000217103F05DF97B4B1B680293029BC9F8B2
:1047F000A032012389F89D32002389F89E3289F87E
:10480000AE322046FCF778F874E10021734B197042
:104810002046FEF735FB6DE10021704B59702046B4
:10482000FEF72EFB66E100216C4B99702046FEF7E7
:1048300027FB5FE14FF42C7303FB04F605EB06093D
:1048400009F5217E07F1F00CBCE80F00AEE80F007F
:104850009CE803008EE80300404609F5217103F04F
:104860001FF95C4B1B680393039BC9F8A03201231B
:1048700089F89D32002389F89E3289F8AE322046AD
:10488000FCF73AF836E10023554A1370554A137085
:1048900020460121FEF7F4FA2CE14FF42C7303FBC0
:1048A00004F605EB060909F5217E07F59C7CBCE8BA
:1048B0000F00AEE80F009CE803008EE803004046BE
:1048C00009F5217103F0ECF8424B1B680493049B3B
:1048D000C9F8A032012389F89D32002389F89E325D
:1048E00089F8AE322046FCF707F803E100233C4A82
:1048F00053703C4A537020460121FEF7C1FAF9E09B
:104900004FF42C7303FB04F605EB060909F5217E31
:1049100007F5C07CBCE80F00AEE80F009CE8030080
:104920008EE80300404609F5217103F0B9F8294BE0
:104930001B680593059BC9F8A032012389F89D32B5
:10494000002389F89E3289F8AE322046FBF7D4FF67
:10495000D0E00023224A9370224A9370204601211E
:10496000FEF78EFAC6E04FF42C7303FB04560023C7
:1049700086F89C321C4B1B78002B00F0BB8000207B
:10498000FFF728FDB6E04FF42C7303FB0456002319
:1049900086F89C32144B1B78002B00F0AB80002073
:1049A000FFF7D8FDA6E04FF42C7303FB0456002359
:1049B00086F89C320C4B1B78002B00F09B8000206B
:1049C000FFF730FE96E000BFDCA2FF1F3CB2FF1FE6
:1049D000349FFF1F50DBFF1FA9BDFF1F14C0FF1F27
:1049E0009CC6FF1FD0BEFF1F70B0FF1F4FF42C737B
:1049F00003FB0456002386F89C32434B1B78002BA4
:104A000078D00120FFF7E6FC74E04FF42C7303FB31
:104A10000456002386F89C323B4B1B78002B69D050
:104A20000120FFF797FD65E04FF42C7303FB04565C
:104A3000002386F89C32344B1B78002B5AD001207F
:104A4000FFF7F0FD56E04FF42C7303FB045393F88B
:104A50009D32002B47D04FF42C7303FB045393F883
:104A60009E328BB94FF42C7303FB04F6A919404610
:104A700001F5217103F014F8244B1B680693069B83
:104A80002E44C6F8A03235E04FF42C7303FB0453D8
:104A900093F89F220132D2B283F89F2203F5267346
:104AA0009B79934211D94FF42C7303FB04F6A91997
:104AB000404601F5217102F0F3FF144B1B68079388
:104AC000079B2E44C6F8A03214E04FF42C7303FB6E
:104AD0000453002283F89C2283F89D2283F89E22AF
:104AE00083F89F2206E04FF42C7303FB045300224B
:104AF00083F89C220134E4B2054B1B78A3423FF6B5
:104B0000E0AD09B0BDE8F08330C0FF1F50DBFF1FF0
:104B1000DCA2FF1F10B1012802D00EE0084900E01E
:104B20000849487B50B90023CA1892F8250028B9D3
:104B30001833B3F5E47FF7D170470020704700BF0A
:104B4000549DFF1FD09AFF1F10B52B4803685B6868
:104B50002A490E2298470020FFF7DCFFA0B1264C1F
:104B600023685B682046264914229847254B18780D
:104B7000FCF7F6F823685B68204623490122984732
:104B8000204607F047FA09E01B4C23685B68204683
:104B90001E490E229847204607F03CFA1648036843
:104BA0005B681B490E2298470120FFF7B3FFA0B1B5
:104BB000114C23685B682046114914229847154B15
:104BC0001878FCF7CDF823685B6820460E4901226F
:104BD0009847204607F01EFA09E0074C23685B68F7
:104BE00020460A490E229847204607F013FA024849
:104BF00007F010FA10BD00BF14DDFF1FB004010064
:104C0000C004010070B0FF1F44FC000008FC00005D
:104C1000D804010030C0FF1F10B5114C23685B6839
:104C20002046104900229847204607F0F3F9FBF789
:104C3000B1FF23685B6820460B4912229847204643
:104C400007F0E8F9FBF7A6FF23685B6820460749F1
:104C50001B229847204607F0DDF9FBF79BFF10BDAC
:104C600014DDFF1F38050100E8040100FC04010009
:104C700038B5114C2368114D5B6820462946002247
:104C80009847204607F0C6F9FBF784FF23685B6866
:104C900020460B4910229847204607F0BBF9FBF746
:104CA00079FF23685B682046294600229847204602
:104CB00007F0B0F938BD00BF14DDFF1F3805010053
:104CC0001805010070B506460024174D2B681B68B7
:104CD0002846315D984701340D2CF7D10620FBF7AB
:104CE000D3FF737B63B13069FBF7F8FE0620FBF757
:104CF000CBFF0D4803685B680C490C22984770BDD8
:104D0000094C23685B6820460949012298470D2019
:104D1000FBF7BAFF23685B682046064909229847DB
:104D2000204607F077F970BD14DDFF1F2C05010048
:104D300084FC00003C05010010B584B0404803F03D
:104D400039F9002844D13F4B1B78002B40D03E4B13
:104D50001B680093009A3D4B1B68D31A642B37D90C
:104D60003B4B1B781BB90122394B1A7011E0394BB0
:104D7000B3F90020384B53F822305B7B4BB1374CF2
:104D800023685B682046364904229847204607F08E
:104D900041F900222B4B1A702B4B1B680193019A8F
:104DA000304B1A602B4B1B8801339BB21AB28B2AF3
:104DB00002DC284A13800BE00022264B1A80274C85
:104DC000204607F027F9FBF7E5FE204607F022F919
:104DD0001B4803F0EFF8002830D11A4B1B78002B4A
:104DE0002CD1194B1B680293029A1E4B1B68D31AD5
:104DF000B3F5487F22D9174BB3F90020164B53F86F
:104E0000220003F085FF70B1124BB3F900200C486B
:104E1000114B53F8221002F043FE0B4B1B68039317
:104E2000039A0A4B1A600122064B1A70094BB3F918
:104E30000020094B53F82200FFF744FF04B010BDD7
:104E40003CB2FF1F509DFF1F50DBFF1FFCBCFF1F2C
:104E500099CAFF1FD49CFF1FD8C6FF1F14DDFF1F78
:104E60004805010004CAFF1F38B505460D4B1B78E5
:104E70000D4A12789A420BD00B4A13700B4C2368E0
:104E80005B6820460A491D229847204607F0C2F871
:104E9000284609F0FFF8074909F008FA064B1860A0
:104EA00038BD00BF00A4FF1F0BBEFF1F14DDFF1F96
:104EB000500501000000C8421CB0FF1F10B502469B
:104EC00043780F3B432B00F23D81DFE813F04400B1
:104ED0003B013B013B013B013B013B013B013B01F2
:104EE0003B013B013B013B013B013B013B013B01E2
:104EF0003B013B013B013B013B013B013B013B01D2
:104F00003B013B013B013B0148004B004E0052007E
:104F10005A005E00620066006C006F007900A1001C
:104F2000A400A800AC00B000B400BC00C200C800DF
:104F3000CE00D100D400D900DE00E300E700EE008F
:104F4000EB00880092005600F200000169000701A2
:104F5000B8000E0129018078FCF714FF10BDFDF7A1
:104F600029FE10BDFDF736FE10BD8078FDF73EFE30
:104F700010BD0020FDF73AFE10BD8078FFF70EF857
:104F800010BD0120FEF78EFB10BD0020FEF78AFB4E
:104F900010BD0120FDF7C8FF10BDFDF7E1FF10BDFA
:104FA000FDF7E6FF10BDFDF7F3FF10BD664B1B7864
:104FB000002B40F0C78001200146FEF7F1F910BD3B
:104FC000614B1B78002B00F0BD80604B1B78002BE1
:104FD00040F0B88001200021FEF7E2F910BD5A4BE5
:104FE0005B78002B40F0AE8002200121FEF7D8F95B
:104FF00010BD554B5B78002B00F0A480534B5B78C1
:10500000002B40F09F8002200021FEF7C9F910BD5F
:10501000FDF7B6FF10BD0120FEF7D6F910BD002048
:10502000FEF7D2F910BD0120FEF7B2FA10BD002044
:10503000FEF7AEFA10BD0120FDF7B2FF10BD022051
:10504000FDF7AEFF10BDC07801210022FFF7ECF89C
:1050500010BDC07801210A46FFF7E6F810BDC07800
:1050600000210A46FFF7E0F810BDFEF775FB10BD02
:10507000FEF78AFB10BD8078D178FEF735FB10BDB6
:105080008078D178FEF742FB10BD8078D178FEF7AA
:105090004FFB10BD0120FDF79DFF10BD8078FDF78F
:1050A00099FF10BDFDF7A4FF10BD8078FFF7DCFE6F
:1050B00010BDC47880786428A8BF642008F0EAFF97
:1050C000234909F0F3F8234B43F8240010BD8078FE
:1050D000003018BF0120FDF793FF10BD8278003229
:1050E00018BF01221C4B1A7010BD8078003018BF09
:1050F0000120D378013B082B24D8DFE803F00523F7
:1051000023232323080B0E00FFF71CF910BDFFF724
:1051100061F910BDFFF71EFA10BDFFF783FA10BD4D
:10512000837813B1012B07D010BDC278003218BFAD
:1051300001220A4B1A7010BDC278003218BF01223A
:10514000074B1A7010BD00BF9CC6FF1FD0BEFF1FCB
:105150000000C8424098FF1F31C0FF1F70B0FF1F02
:1051600030C0FF1F70B582B0244C254D254E13E092
:1051700005F000FEC0B2DA2805D101232370DA223F
:1051800032702B7008E0237833B12A78531CDBB2DD
:105190002B70B054042B03D805F0DCFD0028E7D1B8
:1051A000174B1B78042B25D91748164B1A78027019
:1051B0005A7842709A788270DA78C2701B790371DB
:1051C000FCF7D0FD68B1114B1B680193019A104B9D
:1051D0001A60104801F05CFE0B48FFF76FFE0120DB
:1051E00000E000200023074A1370044A1370044AA9
:1051F000137000E0002002B070BD00BF58BFFF1F59
:10520000F0CAFF1FE8C9FF1FFCCAFF1F50DBFF1FCA
:10521000BCC6FF1F2CBFFF1F38B505460D4B1B78C2
:105220000D4A12789A420BD00B4A13700B4C23682C
:105230005B6820460A4919229847204606F0EAFE94
:10524000284608F027FF074909F030F8064B186098
:1052500038BD00BFA5A5FF1F0BBEFF1F14DDFF1F3C
:10526000700501000000C8421CB0FF1F2DE9F0438B
:1052700083B00446064600EB4002AB4B03EBC2038F
:105280005B7D002B00F0FF80FCF79EFCC0B204EBBE
:105290004403A54A02EBC3039B7A834200F0968144
:1052A00004EB440402EBC404A072A04B1B78002B57
:1052B00000F08C8100249E4D06EB460702EBC707E9
:1052C000A04604EB8403EA5C731C9A4240F0D3804E
:1052D00004EB84032B445A78BB7A9A4240F0CB808B
:1052E00004EB84032B4493F803909B78013B072B3A
:1052F00000F2C180DFE803F004070A132B7184A1D8
:10530000FDF758FCB7E0FDF765FCB4E0894B1B786E
:1053100013B1FDF75FFCAEE0FDF74CFCABE009F12B
:10532000FF33854AD25C002A40F0A5800121824AE1
:10533000D1544846FDF7F8FD48460621FCF7A8F988
:10534000B9F1010F40F09780FCF744FD93E004EBC6
:10535000840805EB08031B79022B14D0032B25D0FE
:10536000012B40F08880754B4B4413F8013C002B17
:1053700040F0818048460121FEF712F8484604219A
:10538000FCF786F977E009F1FF336C4AD25C002A1A
:1053900071D06B4AD35C002B6DD148460021FDF7DC
:1053A000FFFF48460221FCF773F964E0634B4B446E
:1053B00013F8013C43B148460021FDF7F1FF484690
:1053C0000221FCF765F956E048460121FDF7E8FFA8
:1053D00048460421FCF75CF94DE004EB84032B44C0
:1053E0001B79013B022B02D84846FDF7D9FD08EB9B
:1053F000880805EB080348461979FCF749F93AE0B3
:1054000004EB840805EB08031B79022B09D0032B5E
:105410000DD0012B2FD1484601210022FEF704FFB9
:1054200029E0484600210A46FEF7FEFE23E04846F2
:1054300001210A46FEF7F8FE1DE019F1FF3018BF02
:10544000012004EB840805EB08031B79013B082BC2
:1054500011D8DFE803F00E101010101005080B0033
:10546000FEF7B8FF07E0FFF775F804E0FFF7DAF89A
:1054700001E0FEF767FF0134E4B22C4B1B78A34236
:105480003FF61EAFA2E000EB4003274A02EBC30346
:105490005888B0F57A7F05DBB0F5FA6FA8BF4FF4F6
:1054A000FA6001E04FF47A7004EB44031E4A02EB09
:1054B000C30358809B7D012B22D0022B40F08680B5
:1054C000642300934FF47A714FF4FA62002306F0DC
:1054D00033FF04EB4403144A02EBC3031A7AC3B24A
:1054E000D31A002BB8BF5B42052B6FDDC0B204EBB3
:1054F00044040D4B03EBC4031872FFF78DFE65E007
:10550000104B1B7803B3A0F2DC500028B8BF404218
:10551000FF23009300B200214FF4FA720B4606F00D
:105520000BFFC0B22CE000BF68C9FF1F64C9FF1F9A
:1055300038BEFF1FA9BDFF1F14C0FF1F9CC6FF1F61
:10554000D0BEFF1FC89CFF1F04EB4403214A02EB9F
:10555000C303DB7953B1FF2300934FF47A714FF407
:10556000FA62002306F0E8FEC0B209E000230093CF
:105570004FF47A714FF4FA62FF2306F0DDFEC0B2F9
:1055800004EB4403134A02EBC3031B7A1B1A002BE0
:10559000B8BF5B42032B04DC0F4B1B78834215D949
:1055A00005E00D4B1B78834288BF002000E00020FF
:1055B000084D6600331905EBC3031872FDF716FB9F
:1055C000344405EBC405287AFEF7E8FC03B0BDE8D7
:1055D000F08300BF68C9FF1F01A4FF1F2DE9F0473A
:1055E000464CA61D0C340025A4F10C0808F16107F7
:1055F000DFF81C91E8B2A24614F8063C002B72D0EA
:1056000034F8083CA3F5487292B2B2F5AF6F1FD8D8
:1056100024F80A3CD6F80630636014F80B3C012BE2
:1056200003D05BB1022B03D02CE0FFF71FFE29E073
:10563000002304F80B3C0123237223E0237A013377
:10564000DBB22372042B1DD9012304F80B3C19E0B3
:10565000D6F806206368D31A29498B4212D9294B00
:105660001B7823B118B9002304F80B3C07E0264B44
:105670001B78012B14BF002302230AF80B3C0023E4
:105680008AF8083000210AF8061C08F101034FF0DF
:10569000010C1A78187E904204BF0CF1010C5FFADD
:1056A0008CFC012A08BF01211833BB42F1D198F8C4
:1056B0007930012B1ED0BCF1050F04D198F80130D0
:1056C00089F8003007E019B1012389F8003002E0C1
:1056D000022389F8003099F800200C4B1B789A427D
:1056E00001D0FCF7EFF9013518361834052D81D1BA
:1056F000BDE8F087BCF1050FE6D1DFE768C9FF1F01
:10570000A0860100B8C6FF1FA0C6FF1F19C0FF1F5B
:10571000E0C9FF1F70B5172004F0A0FD0446164B2A
:105720001B78164A12789A4208D0154A1268821AD3
:10573000002AB8BF52424B2A0CDC70BD204608F04C
:10574000ADFC4FF06A5108F0FDFC0E4B18600C4B9D
:105750001C6070BD094E33700B4D2B685B6828468A
:105760000A491B229847284606F054FC3278024B1F
:105770001B789A42E2D070BDA8BDFF1F0BBEFF1F71
:10578000A0AFFF1F1CB0FF1F14DDFF1F8C05010021
:1057900008B5084B1B78012B02D0022B05D008BDA1
:1057A0000520002104F0D6FE08BD0E20012104F0E2
:1057B000D1FE08BDCB9CFF1F08B5084B1B78012B01
:1057C00002D0022B05D008BD0520012104F0C2FE45
:1057D00008BD0E20002104F0BDFE08BDCB9CFF1FBC
:1057E0002DE9F04F85B000238DF80C308DF80D3089
:1057F0008DF80E308DF80F30FFF78CFF8B4B93F840
:105800009C321BB9894B93F84C354BB101278DF86D
:105810000C70874B1868002108F08CFB064601E0ED
:1058200000270026834B93F89C32019323B9814BC8
:1058300093F84C353BB943E07E4B93F84C352BB98C
:105840004FF07E5904E04FF07E5901E04FF07C5953
:10585000794B93F80080794D0024DFF804A24FF0D3
:105860008F4BB8F1000F17D0032C1AD84846514679
:1058700008F024FE30B94846714908F001FE18B915
:10588000484602E0504600E06D48594608F05AFC90
:1058900008F01EFEA86104E0032C9CBF4FF4803387
:1058A000AB6101340435042CDBD101238DF80D30BC
:1058B00030465F4B596808F03DFB06460137FFB2A2
:1058C000604B1B7873B1604A12785AB13046584B1E
:1058D000996808F02FFB064601238DF80E301F440F
:1058E000FFB25BE0534A92F8FC2722B9514A92F882
:1058F000AC2A002A52D073B9019BABB14D4B93F83F
:105900004C358BB130464A4B596808F013FB0646BC
:105910004FF07C5910E03046454B996808F00AFB7F
:1059200006464FF07E5907E03046414B596808F073
:1059300001FB06464FF07E593F4B93F80080434DE4
:105940000024DFF81CA14FF08F4BB8F1000F17D0E7
:10595000032C1AD84846514608F0B0FD30B94846E5
:10596000374908F08DFD18B9484602E0504600E07E
:105970003348594608F0E6FB08F0AAFDA86104E0A8
:10598000032C9CBF4FF48033AB6101340435042CED
:10599000DBD101238DF80E301F44FFB22C4B93F85E
:1059A000303013F0FF0F0AD03046214BD96808F091
:1059B000C1FA064601238DF80F301F44FFB2254B74
:1059C0001868254B196808F065FD10B1FFF7E0FE77
:1059D00005E017B9FFF7DCFE03E0FFF7EDFE012F4E
:1059E00040D81C4B1E681D4D00241D4F4FF08F48A2
:1059F000DFF84C90032C14D83046394608F05EFD91
:105A000030B93046494608F03BFD18B9304602E04F
:105A1000384600E04846414608F094FB08F058FD3F
:105A2000A86101340435042CE4D184E084C0FF1F54
:105A30004098FF1F3CB2FF1FA8B0FF1F5CCAFF1FAA
:105A400000FEFFC65ABFFF1FA9BDFF1FA4AFFF1F67
:105A5000A4CAFF1F1CB0FF1FF4CAFF1FE4AFFF1F43
:105A600000FEFF463046002108F028FD00285CD0EB
:105A700030464FF07E5108F003FD08B14FF07E56DE
:105A80002E4B93F800B02E4BD3F800902D4D0024F0
:105A9000DFF8BC804FF08F4A03ABE35C002B3BD0B8
:105AA000BBF1000F20D04846274B53F8241008F0D4
:105AB00049FB314608F0FAFB0746032C30D8414633
:105AC00008F0FCFC28B93846204908F0D9FC10B988
:105AD00002E0474600E01D4F3846514608F032FBD1
:105AE00008F0F6FCA8611BE0032C19D84846414693
:105AF00008F0E4FC30B94846144908F0C1FC18B974
:105B0000484602E0404600E01048514608F01AFBC3
:105B100008F0DEFCA86103E0032C9CBF0023AB610E
:105B200001340435042CB7D105E0064B00229A61FC
:105B3000DA611A625A6205B0BDE8F08FA8B0FF1FA3
:105B40001CB0FF1FE4AFFF1F4098FF1F00FEFFC601
:105B500000FEFF4610B582B0594B1B78012B5FD079
:105B600013B1022B45D05FE0FFF7FCFAFFF736FDDB
:105B7000544B1B78012B17D10122514B1A70524BF9
:105B80001B78002B2ED0514C23685B68204650496F
:105B900015229847204606F03DFA204606F03AFACC
:105BA000204606F037FA1AE04A4B1B68BBB10222C6
:105BB000434B1A70FBF710FF434B1B787BB1434CF0
:105BC00023685B682046444919229847204606F01E
:105BD00021FA204606F01EFA204606F01BFA384B42
:105BE0001B780BB33D4801F04BF93D4801F050F9EB
:105BF0001AE03C4B1B780BB9FFF7B4FA384801F0B8
:105C00000DF988B9384B1B680193019A314B1B6819
:105C1000D31AB3F57A7F07D9314801F095F903E03B
:105C2000FFF7DCFCFBF776FF304801F0C9FB2B489F
:105C300001F098F92A4801F095F92D4C204601F021
:105C400091F904F12C0001F08DF904F1580001F0F4
:105C500089F9FFF7C5FD234B1B7893B1254B1B78C2
:105C600063B90122234B1A701C4801F009F91C4842
:105C700001F006F9FDF7A8FEFEF7CEFFFFF75CF88E
:105C80001CE01C4B1B786BB100221A4B1A701A488F
:105C900001F0DAFEFEF7ECFF094B1B7813B90F4851
:105CA00001F052F9FDF7E8FFFDF7D4FEFEF7ACF97D
:105CB000FEF7F4F9FEF7FAFCFDF712FE02B010BD94
:105CC000A0C6FF1FE0C9FF1F339AFF1F14DDFF1F8F
:105CD000A8050100BCC6FF1FC005010074B0FF1F6E
:105CE0002CBFFF1FB8C6FF1F50DBFF1F0CB1FF1FEB
:105CF000E8C5FF1F18C0FF1F3CB2FF1F08B50022F8
:105D0000024B1A60FFF76CFD08BD00BF1CB0FF1FFF
:105D100070B5FFF7F3FFFFF73BFD5048FDF7FEFDC1
:105D20004F48FDF7FBFD4F4C04F178052046FDF789
:105D3000F5FD1834AC42F9D14B48FDF7EFFD4B4C63
:105D400004F178052046FDF7E9FD1834AC42F9D19D
:105D5000474C04F1F006474D2046FDF7DFFD10B13A
:105D60002B7801332B701834B442F5D1424C04F136
:105D700078052046FDF7D2FD1834AC42F9D13F48F2
:105D8000FDF7CCFD3E48FDF7C9FD3E4C04F1F006A1
:105D90003D4D2046FDF7C2FD10B12B7801332B702D
:105DA0001834B442F5D13948FDF7B8FD384C04F544
:105DB0006A752046FDF7B2FD1834AC42F9D1354C76
:105DC00004F5F0752046FDF7A9FD1834AC42F9D171
:105DD000314C04F5F0752046FDF7A0FD1834AC42B7
:105DE000F9D12E4C04F5F0752046FDF797FD1834D7
:105DF000AC42F9D12A4B00210A4683F89C2283F851
:105E00009D2283F89E2283F89F22A3F8AA2283F87A
:105E1000AC1283F8AE2283F8A822013103F52C736B
:105E20000429EAD11F4B002283F89C2283F89D228B
:105E3000A3F8AA2283F8AC2283F8AE2283F8A82222
:105E400083F84C2583F84D25A3F85A25012183F8C2
:105E50005C1583F85E2583F8582570BD1CA4FF1FD0
:105E6000349AFF1F34A4FF1F04A4FF1F589AFF1F7A
:105E700010A3FF1FACBFFF1FD89CFF1FB09CFF1FCC
:105E8000F8A2FF1FB4A4FF1F9DAFFF1FE0A2FF1FDA
:105E9000349FFF1F5098FF1F549DFF1FD09AFF1F74
:105EA0003CB2FF1F84C0FF1F70B590B041F2883034
:105EB00004F0D6FC0620022104F07EFB092002211A
:105EC00004F07AFB0A2004F059FC062004F066FB7B
:105ED00060B10122B54B1A70B54AB64B1A600E225A
:105EE000B54B1A700F22B54B1A7013E0092004F05D
:105EF00055FB18B10222AD4B1A7002E00322AB4BE6
:105F00001A70AF4AAB4B1A600F22AB4B1A700A22C1
:105F1000AA4B1A70A54B1B78012B12D1A94800215E
:105F200001F01CFD322004F029FC0520012104F0C1
:105F300043FB0520012104F00DFB0A2004F01EFCA8
:105F400010E0012B0ED90E20012104F035FB0E20AC
:105F5000012104F0FFFA0A2004F010FC9948022104
:105F600001F0FCFC98480C2105F058FEFFF738FCC6
:105F7000964B13221A7012221A76112283F83020BF
:105F8000102283F848208D4A127883F86020FBF7AE
:105F9000C9FCFBF7F5FC8E481521002200F020FF1C
:105FA0008C481421002200F01BFF8B4C2046052159
:105FB000002200F015FF04F12C000421002200F063
:105FC0000FFF04F158000321002200F009FF082010
:105FD000012104F0F1FA8148082101F0ABF8172003
:105FE000022104F0E9FA7E4B1B7803F0FE017D4AA2
:105FF000126812F4805F02D08B4240F07A81784AB6
:10600000117003F0FC027748006810F4805F02D042
:10601000914240F0788172490A7003F0F8037149A7
:10602000096811F4805F02D09A4240F076816C4A90
:106030001370614C2078012104F0BEFA2078012110
:1060400004F088FA207803F001F810BB604828219A
:106050000A4600F05FFF644B1B680093009D624C92
:106060005B4E304600F07EFF23680193019B5B1B73
:10607000B3F57A7FF5D95D4D2B685B6828465C499E
:1060800036229847284605F0C5FF23680293029DF3
:10609000E7E74FF4FA7004F071FBFFF739FE554B58
:1060A0001B7833B1FAF790FD524B1B780BB1FAF71E
:1060B00023FEFAF759FBFAF78DFB0020FEF72AFDC5
:1060C0004D4B18700120FEF725FD4C4B18704C4BC2
:1060D00000221A705A709A70FBF73CFF494B93F8F4
:1060E0004130032B02D8484802F0A8FF454C03A8D2
:1060F0002146A27E02F030FD9DF8103084F8203059
:10610000059B63629DF8183084F82830079BE36292
:10611000089B2363099B63630A9BA3630B9BE36355
:106120009DF8303084F840309DF8313084F84130AB
:1061300010AB53F80E5D58689968C4F84250C4F823
:106140004600C4F84A101B7B84F84E3003A802F0C6
:1061500061FE94F84130032B09D820460023E376F2
:106160002A49502200F08CFB002874D156E001220D
:10617000244BDA761D4C23685B68204624490A22AA
:106180009847244B1D68284609F0C8F90246236841
:106190005B6820462946984723685B6820461E496D
:1061A00010229847204605F035FF86E0CB9CFF1F64
:1061B0000AD7A33CF4CAFF1FCC9CFF1FADA4FF1F4E
:1061C000A69BC43B80C6FF1F0082FF1F68C9FF1F3C
:1061D00074B0FF1F2CBFFF1FE8C5FF1FD0C6FF1FF5
:1061E00010DDFF1F3C80044050DBFF1F14DDFF1F4C
:1061F000DC050100339AFF1FA0CAFF1F24BFFF1F49
:106200009CC6FF1F08CAFF1F24CAFF1F34C0FF1F00
:1062100014060100509AFF1F20060100454C236818
:106220005B68204644490A229847444D284609F0B5
:1062300075F9024623685B6820462946984723681B
:106240005B6820463E490D2298472846E97E012298
:1062500000F07AFC31E001223A4B1A70FBF74AFF5A
:10626000FAF798FC334C23685B68204636492222B3
:106270009847204605F0CEFE23685B6820463349E8
:1062800016229847204605F0C5FEFAF783FCFAF778
:106290009FFDFAF7FBFDFAF763FEFEF755FCFAF7F0
:1062A000ABFEFAF745FFFBF717F9FAF7C7FC2046F4
:1062B00005F0B0FE204605F0ADFE254A4FF48033D0
:1062C0009361D36113625362224A9361D361136273
:1062D0005362214A9361D361136253620E2003F02B
:1062E000BDFF05F0DDFF1D4800F02EFEFAF73CF97A
:1062F0001DE04FF4A2701A4A10604FF41070A2F51E
:106300007F6210607BE64FF4A270164908604FF47C
:106310000070A1F57F6108607DE64FF4A271124A1A
:1063200011604FF41071A2F57F6211607FE610B02A
:1063300070BD00BF14DDFF1F1406010008CAFF1F57
:1063400034060100A0B0FF1F4406010068060100EA
:1063500038CBFF1F5CCAFF1FA4AFFF1F74B0FF1F25
:1063600008C004400CC0044004C004402DE9F04FB4
:1063700089B0BB4800F07CFFBA4C2046BA4B196884
:106380000022134600F0F6F92046B849B84A08F052
:10639000E5F8B84C04F52C652046FAF7BDF904F58C
:1063A0002C74AC42F8D1B24C0020B349224608F01C
:1063B000D5F8B24F3846FAF7AFF907F52C7B5846B7
:1063C000FAF7AAF90020AE49224608F0C7F8AD480E
:1063D00000210A46FAF74CF9AB4BAA4A1360002495
:1063E0009461104601F01CFFA84E3046012106F1D1
:1063F0002402FAF73DF9DFF81493C6F800904FF045
:10640000FF38C6F8188006F1280A5046012106F127
:106410004C02FAF72DF9C6F82890C6F840809C4D3A
:106420002846012105F12402FAF722F9C5F8009067
:10643000C5F8188005F12800012105F14C02FAF792
:1064400017F9C5F82890C5F840809248FAF734F952
:10645000DFF8BC924846FAF72FF98F48FAF72CF983
:10646000DFF8B0824046FAF727F98C48012100F1A5
:106470001802FAF7FDF88A4B884A1360104601F0BB
:10648000B1F988480760466004724472C46005F040
:10649000B7FC854807604660012707724472C460F4
:1064A00005F0AEFC8148C0F800B0C0F804A004724A
:1064B0004472C46005F0A4FC7D48C0F800B0C0F888
:1064C00004A007724472C46005F09AFC7948066023
:1064D000704B436004724472C46005F091FC7648CE
:1064E000C0F800A06B4A426004724772C46005F0B5
:1064F00087FC72485F4E0660C0F8049004724472D4
:10650000C46005F07DFC6E480660C0F80490077218
:106510004772C46005F074FC6A4806F52C7AC0F82E
:1065200000A0C0F8049004724FF002034372C460EC
:1065300005F066FC6448C0F800A0C0F8049007723B
:106540004FF0030B80F809B0C46005F059FC5F48B8
:1065500006F5AC6AC0F800A0456004724472C460DD
:1065600005F04EFC5A48C0F800A04560077244721E
:10657000C46005F045FC574806F50166066005F164
:106580002802426004724472C46005F039FC52482B
:10659000066005F12803436007724472C46005F089
:1065A0002FFC4E4805603C4A426004724472C4604D
:1065B00005F026FC4A4805F128030360364A42608C
:1065C00004724772C46005F01BFC4648314B0360FF
:1065D000C0F8048004724472C46005F011FC4248A3
:1065E000C0F80090C0F8048004724772C46005F0DF
:1065F00007FC3E48284A0260C0F8048004724FF04D
:1066000002034372C46005F0FBFB39481D4A026077
:10661000C0F80480047280F809B0C46005F0F0FB93
:106620003448C0F800801D4B436004724472C4605B
:1066300005F0E6FB304B1A78304B1A70304B1A6875
:10664000079207992F4A11601968069106995160BF
:106650001A68059205992C4A11601B685CE000BF1E
:106660000CB1FF1F08CAFF1F509AFF1FA967000047
:106670003C98FF1F3CB2FF1F8D04000084C0FF1F29
:1066800065040000A4CAFF1FB009010020B0FF1F6D
:10669000C4BFFF1F38CBFF1FA4AFFF1F80C6FF1F63
:1066A00090090100D8CAFF1F10BDFF1FB4BFFF1F14
:1066B00024BDFF1F34BDFF1FC0C6FF1F44BDFF1F09
:1066C00038C9FF1F54BDFF1F08C9FF1F18C9FF1F8E
:1066D00064BDFF1F4CC9FF1F74BDFF1F84BDFF1F9A
:1066E00020C0FF1F28C9FF1FF4C9FF1F98BDFF1F4F
:1066F000A4C6FF1F08CBFF1FA8BDFF1F0BBEFF1FB7
:1067000050DBFF1F74B0FF1F2CBFFF1F700901007B
:106710005CCAFF1FE4AFFF1F0493049B5360114D3D
:1067200005F12C032E46B0350F4AA3F12804116859
:106730000391039943F82C1C116802910298991B4C
:10674000214441F82C0C2C33AB42F0D1074800F027
:106750006FFC054B1B680193019A054B1A6009B049
:10676000BDE8F08FE8C5FF1F50DBFF1FD0C6FF1F3D
:1067700094CAFF1FF8B504460D4617461E461C3046
:1067800002F038FB284608F0C9FE1A2804D8204633
:10679000294608F065FE01E000232370A77684F8FF
:1067A00050602046F8BD00BF10B504461C3002F012
:1067B00031FB204610BD00BF2DE9F04104460F46D5
:1067C00015461E4690F82500032848D8022A49D9C4
:1067D0002046196802F006FC002846D020463946BB
:1067E0002A4602F023FB804638B1013D27D03B7892
:1067F0000A2B41D00D2B1BD13AE000233B70072020
:10680000BDE8F081104612F8011B0A2936D00D2987
:1068100010D12FE0002202705A1CB85C884218BFC9
:106820001A46336801331A4432600020BDE8F08113
:106830007A1C00230133984501D0AB42E2D1236892
:106840009B682046984728B9002307F8083007209E
:10685000BDE8F08100237B550320BDE8F0810220D4
:10686000BDE8F0810320BDE8F0810420BDE8F0819F
:10687000384600230A21CDE7384600230D21C9E719
:106880002DE9F04182B080460F46164602AC002347
:1068900044F8043D00F11C0528463946324623469B
:1068A000FFF78AFF0028F7D0072804D1002388F8D3
:1068B0001B30012002E088F81B00002002B0BDE878
:1068C000F08100BF3B2804D0232814BF0020012002
:1068D00070470120704700BF38B504462546013493
:1068E000287807F07BFE0028F8D1284638BD00BF85
:1068F00070B5054608F012FE01382C180AD20026A1
:1069000002E06670A54205D814F8010907F066FE9A
:106910000028F6D170BD00BF2DE9F04105461446B0
:106920000F4619B90523C376012445E01C301146F2
:106930001A46069BFFF740FF064690B3072830D063
:10694000E876012438E05B2C22D108F10100FFF742
:10695000C3FF80465D2108F0FBFB0346C0B1002267
:1069600002704046FFF7C4FF95F850403CB14046E6
:10697000394608F067FC58B90023EB761CE0404626
:10698000394608F0C3FB18B90023EB76012413E065
:10699000072E03BF0523EB76012400240CE000241E
:1069A0000AE02046FFF798FF804604782046FFF76C
:1069B00089FF0028F3D1C6E72046BDE8F08100BF7B
:1069C0002DE9F84305460F461C4616460AB11278D3
:1069D0001AB90623EB7601245DE01C301946089AAB
:1069E0000A9BFFF7E9FE804600283ED0072847D0E3
:1069F000E87601244FE00623EB7601244BE02FB12B
:106A00005B2C03D10623EB76012444E048463D216C
:106A100008F09EFB0746F0B1002303704846FFF7DD
:106A200067FF95F8504054B14846314608F00AFCDB
:106A300088B90137099B1F600023EB762BE048469D
:106A4000314608F063FB30B90137099B1F60002312
:106A5000EB7601241FE0B8F1070F03BF0623EB76A6
:106A60000124002417E0002415E02046FFF734FF3E
:106A7000814604782046FFF725FF0028F3D1BEE7C2
:106A80002046FFF729FF814604782046FFF71AFFCA
:106A90000028B0D1B3E72046BDE8F88370B586B0D2
:106AA00004461E460B9D90F84100032803D902239B
:106AB000E376012045E0287901280BD010B10228A7
:106AC00015D035E0002914BF012302232B710020CB
:106AD000286036E0009520461A460A9BFFF71CFF07
:106AE00050B3E37E63BB02232B71002029E00A9B95
:106AF000009305AB0193029520463346FFF760FFF4
:106B0000E0B1E37EE3B90598FFF7E6FE0590FFF7F5
:106B1000EFFE059A137843B1531C0593127806F8DB
:106B2000012B1A461B78002BF6D10023337007E0A7
:106B30000823E376012004E0002002E0002000E0CA
:106B4000012006B070BD00BF10B51446082945D815
:106B5000DFE801F0050C131A21282F363D002548E7
:106B600003685B682449082298473DE02148036890
:106B70005B6822490E22984736E01E4803685B682E
:106B80001F490D2298472FE01A4803685B681D498A
:106B90001022984728E0174803685B681A490A22C0
:106BA000984721E0134803685B6818491122984709
:106BB0001AE0104803685B6815490D22984713E0F6
:106BC0000C4803685B6813490B2298470CE009489E
:106BD00003685B6810490D22984705E00548036883
:106BE0005B680E491322984714B1024805F012FA67
:106BF00010BD00BF14DDFF1FA4060100B006010098
:106C0000C0060100D0060100E4060100F006010004
:106C100004070100140701002007010030070100EC
:106C200000220260027170472DE9F04385B00446EE
:106C3000894690461F460C9E02A8FFF7F1FF02AD61
:106C4000009601952046494642463B46FFF726FFFF
:106C50000028F5D0E07ED0F1010038BF002005B05B
:106C6000BDE8F08330B583B01C46069D0095FFF764
:106C7000DBFF054630B32046144908F047FA48B117
:106C80002046134908F042FA20B12046114908F085
:106C90003DFA18B90123079A137013E020460E49F4
:106CA00008F034FA48B120460C4908F02FFA20B118
:106CB00020460B4908F02AFA18B90023079A1370E6
:106CC00000E00025284603B030BD00BF44070100A6
:106CD0004C07010050070100540701005C07010048
:106CE0006007010030B583B01D46069C0094FFF795
:106CF0009BFF044620B1284607F036FC079B18701E
:106D0000204603B030BD00BF30B583B01D46069CA1
:106D10000094FFF789FF044620B1284607F028FCBD
:106D2000079B1860204603B030BD00BF10B584B08B
:106D3000069C009403AC0194FFF7E6FF034610B1F4
:106D40000399079A1180184604B010BD30B585B07C
:106D50001D46089C0094FFF767FF044678B128465B
:106D600003A90A2208F062FD039BAB4204D01B7802
:106D700023B9099B186002E0002400E000242046AB
:106D800005B030BD08B5C37A3BB1807A03F006FC8C
:106D9000D0F1010038BF002008BD807A03F0FEFB6F
:106DA000003018BF012008BD08B5C37A23B1807A2E
:106DB000002103F0CFFB08BD807A012103F0CAFB5C
:106DC00008BD00BF08B5C37A23B1807A012103F062
:106DD000C1FB08BD807A002103F0BCFB08BD00BFE9
:106DE00010B504468172C2720846012103F0E4FB2B
:106DF0002046FFF7E7FF00232373637310BD00BF36
:106E000010B5847A204603F0C9FBD0F1010138BFE8
:106E10000021204603F09EFB10BD00BF007B7047A1
:106E200082B000230373437383730382034A12689F
:106E30000192019A0260038102B0704750DBFF1F8C
:106E4000F0B583B004460E461746FFF7E9FF01256B
:106E5000A5742782AE40013EA6732046FFF7A4FF2B
:106E6000034B1B680193019B2360257303B0F0BDA6
:106E700050DBFF1F08B50A460121FFF7E1FF08BDFF
:106E800010B50446FFF79EFF2046FFF7C9FF10BD6F
:106E900010B50446037B0BB1FFF7F2FF2046FFF766
:106EA00083FF10BD10B50446037B0BB1FFF7E8FF6D
:106EB0002046FFF787FF10BD84B070B582B005464D
:106EC00007AE86E80E00FFF7ABFF0023AB7405F1B9
:106ED00014040FCE0FC496E8030044F8040B21807D
:106EE000AB8A2B829DF834300A2B28BF0A23AB7360
:106EF0002846FFF759FF064B1B680193019B2B6047
:106F000001232B7302B0BDE8704004B0704700BF8E
:106F100050DBFF1F30B58BB00446ADF81010ADF854
:106F2000122001238DF82430022303936B460AAD0F
:106F300015E9070003C31A8004AB0ECB2046FFF708
:106F4000BBFF0BB030BD00BF08B540F2EE210A46D2
:106F5000FFF7E0FF08BD00BF08B528210A46FFF78C
:106F6000D9FF08BD10B586B0044603896BB12F4A1E
:106F700012680192019942688A1A934205D2FFF77A
:106F800021FF2046FFF74CFF4DE0238A002B4AD01B
:106F9000264A12680292029922688A1A934242D2C1
:106FA000637B0133DBB26373A27B9A4225D913F072
:106FB000010F03D02046FFF705FF02E02046FFF750
:106FC000F3FEA37C9BB9637B0A2B06D92046FFF70F
:106FD000F9FE2046FFF724FF25E004EB43039B8ADC
:106FE0002382124B1B680393039B23601BE00F4B10
:106FF0001B680493049B236015E094F8283063B168
:10700000A38A2382002363732046FFF7CDFE074B3C
:107010001B680593059B236005E02046FFF7D2FE21
:107020002046FFF7FDFE06B010BD00BF50DBFF1F7E
:1070300000230371114B198811F0010F18D102E0E0
:107040000B420AD100E0012319430C4A11800C4A7B
:10705000118821EA0303138070470279013202711B
:107060005B009BB2B3F5805FEAD3FF2303717047E7
:1070700001230371014B19880223E1E77ACBFF1F3B
:1070800070CBFF1F2DE9F041044617461E460579D7
:107090000B2D3BD85FFA81F84046012103F08CFAB2
:1070A00025791C4B03F8058042F6E0621A4B23F861
:1070B00015201A4B012202FA05F51A8815431D8086
:1070C000FF002780F6006680154B1B6813F0010F48
:1070D00018D1134B1A6842F001021A60114B1A784A
:1070E00042F080021A70A3F5143300221A600321C3
:1070F0000D4A116001210432116045221A602022DC
:107100000A4B1A704FF40012094B1A602079BDE83F
:10711000F08100BF94CBFF1F7CCBFF1F70CBFF1F04
:1071200038800440005006400400044055E400E06C
:1071300008E100E008B54FF408724FF41663FFF75A
:10714000A1FF08BDC9000388994203DB4388994227
:10715000B8BF0B4602790B2A9CBF024921F81230B6
:10716000704700BF7CCBFF1F08B5384B93F9003048
:10717000374A12881A4112F0010F07D0354AD05C05
:10718000002103F0E7F90C22304B1A70324B1B78C8
:107190005AB20B2A35DC2E4A10885AB240FA02F154
:1071A00011F0010F26D009E05AB240FA02F111F0B5
:1071B000010F01D1DBB21DE027490B70254B985C14
:1071C000012103F0C7F9244B1A7820490A7052B202
:1071D000224931F81210224A106808441060214AEE
:1071E000106801441160C521083A11601A78013213
:1071F0001A7008BD0133DBB25AB20C2AD4D1164A38
:107200001370174B1968C1F51C3303F58073B3F580
:10721000487F05DB4EF660229342A8BF134601E08B
:107220004FF448730E4A194411600E49086803442C
:107230000B60C5210C4B196012680C4B9A4204D9A3
:107240000023074A1360044A137008BDA6A5FF1F58
:1072500070CBFF1F94CBFF1F78CBFF1F7CCBFF1F92
:1072600074CBFF1F0800044000000440FF700200C0
:1072700030B482B00E4B1B680193019D0123C0F80E
:107280002431034600210A46441884F8C8209A6233
:107290001D60C3F8A020C3F8FC20013104330A2983
:1072A000F2D10023C0F8283102B030BC704700BFD3
:1072B00050DBFF1FD0F82831092B09DC836A53B15A
:1072C0000123C26A4AB1013304300A2BF9D106E026
:1072D0004FF0FF30704700207047184670474FF05E
:1072E000FF3070472DE9F04182B0044688461646CB
:1072F0001F46FFF7DFFF002820DB16B304EB8005F5
:10730000C5F85080AE62AF672318012283F8C82009
:107310000E4B1B680193019B44F82030D4F82401E4
:10732000C5F8FC00D4F828311344C4F82831831878
:10733000002BD8BF0123C4F8243104E04FF0FF3004
:1073400001E04FF0FF3002B0BDE8F08150DBFF1FDD
:1073500008B50123FFF7C6FF08BD00BFD0F8FC3019
:107360008B420AD003460120D3F800218A4208D07C
:10737000013004330A28F7D101E0002070474FF0B4
:10738000FF30704738B50446D0F82851BDB1FFF73B
:10739000E5FFB0F1FF3F12D004EB80039A6A72B1AF
:1073A00000229A62204480F8C820C3F8D4201A65CD
:1073B000C3F8A020C3F8FC20013DC4F8285138BD13
:1073C0002DE9F04383B00546264B1B680193DDF899
:1073D00004C000F12403002217464FF001084FF0CB
:1073E0000209C3F8B07004331968E9B153F8281CD6
:1073F0009C6AC1EB0C06A64216D3214443F8281C14
:10740000A91891F8C81079B1196D11B9C3F8AC80F9
:107410000AE09C6FA14207DDC3F8AC8001349C6791
:10742000A142D8BFC3F8AC9001320A2AD9D12C4668
:1074300005F12807D4F8D430012B02D0022B03D059
:1074400009E0A36A984706E0A36A98472846D4F85B
:10745000FC10FFF797FF0434BC42EBD103B0BDE84A
:10746000F08300BF50DBFF1F10B582B00446FFF76A
:1074700075FFB0F1FF3F05D0034B1B680193019BE3
:1074800044F8203002B010BD50DBFF1F10B5044699
:10749000FFF764FFB0F1FF3F1ABF001990F8C80072
:1074A000002010BD2DE9F04F83B0019084693CB9F4
:1074B000002104F075FC00285AD004F03BFC57E092
:1074C000B4F1FF3F0FD10198002104F069FC04469C
:1074D00000284DD001982146002204F04BFC2046A4
:1074E00004F028FC44E00198002104F065FC80468B
:1074F00000283DD0019BD3F81CC093F820900023B6
:107500001D4F9B464FF0FF3A4E46200EC4F30F210D
:1075100008EB0302B2F90450C1F5803E37F9109030
:10752000013037F9100001FB00F109FB0E110914BD
:1075300001FB05F1C913918026B1E243944506D2BF
:10754000644407E0A44504D2CCEB040402E05446B2
:1075500000E05C460233B3F5807FD6D1019B9C618D
:1075600018464146002204F005FC404604F0E2FBC8
:1075700003B0BDE8F08F00BF6407010072B68369F5
:1075800013B90123836105E0B3F1FF3F04BF6FF03E
:1075900001038361C16180F8202062B6704700BF9B
:1075A00010B5044604F0F6FC204610BD08B50348AB
:1075B0000349044A06F0D2FF08BD00BFA0CBFF1F5D
:1075C000A17500003C98FF1F38B5064D064C0748D2
:1075D0002946224606F0C2FF05482946224606F003
:1075E000BDFF38BDA17500003C98FF1FA8CBFF1F51
:1075F000B0CBFF1F08B503480349044A06F0AEFFAD
:1076000008BD00BFB8CBFF1FA17500003C98FF1F4D
:1076100008B503480349044A06F0A0FF08BD00BFAF
:10762000C0CBFF1FA17500003C98FF1F2DE9F84358
:107630008146804600263746F7B94846314604F071
:10764000BBFB0746002853D0D8F81810B1F5803F8F
:107650004ED0031D00F582741A6831FB02F031FB35
:1076600012F200F30F0002F30F02C0EA024243F8E5
:10767000042B9C42F0D83BE04846314604F090FB96
:107680008446A8B33B1D051DD8F8184007F5827E37
:10769000B4F5803F16D107F10C040C3054F8082CD7
:1076A00050F8081C92FA11F244F8082C5A6850F865
:1076B000041C92FA11F25A600833083408309E45CF
:1076C000ECD812E055F8042B34FB02F034FB12F234
:1076D00000F30F0002F30F02C0EA0242196892FAA7
:1076E00011F143F8041B9E45ECD8604604F022FBE0
:1076F000013608F10408042E9ED13FB148463946B0
:10770000002204F037FB384604F014FBBDE8F88390
:1077100008B5002104F044FB0246A0B172B60A4B42
:10772000186810B91A6062B608BD084B1B681BB90F
:10773000064B1A6062B608BD03490B60034B1A6022
:1077400062B604F0F7FA08BDD8CBFF1FC8CBFF1F05
:1077500038B51C4B1A68126819791B4B19701B4BF2
:107760009A4206D2A3F5807404F5807304F5007480
:1077700002E0174B03F58074164A106898B1021D99
:1077800047F6FF7532F9021B2944091123F8021B41
:107790009C42F7D804F0CEFA0F4B1A680D490A60E4
:1077A00000221A6005E040F2FF7223F8022B9C428F
:1077B000FBD80A4B1B781BB14FF08042084B1A6074
:1077C00038BD00BFCCCBFF1F1F800040308FFF1F94
:1077D000308EFF1FD8CBFF1FC8CBFF1FD4CBFF1F9E
:1077E00008E200E070B54F48012104F075FB4E4BF4
:1077F0001A6842F480521A60802203F5032303F6CC
:10780000F5731A700024494E01253480284602F091
:10781000B5FF0834A4B223B2B3F5006FF5D1444BE1
:107820001B6813F4800F16D0424B1A6848F6A273F7
:107830001A409A420FD1404B1A6840F23F439A4295
:1078400009D13E4B1B68012B05D13D4B1A6840F214
:1078500001139A4217D0364B1A6842F480021A601C
:107860000122A3F59033303B1A6040F23F42083BBF
:107870001A60043B48F6A3721A60324A1A6040F25A
:10788000011210331A60274C23681A6800222E490F
:1078900019602368022119715A7101209871D871F9
:1078A00019725A729A72DA721A736FF0010159736F
:1078B0004FF0FF319973D97319691C4919611A7511
:1078C0005A75D98A4FF48071D9821A765A769A7687
:1078D000DA76D88BD983998B06219983237903F1A2
:1078E000804303F504331A70B0221A7004F0A0FA32
:1078F000164B18702279164B1A70227902F110017A
:107900001448154B43F8210053119B0003F16043C9
:1079100003F5614302F01F02012101FA02F21A602D
:1079200070BD00BFCCCBFF1F2C80044000C00C40BA
:107930003C80044000600340046003400C6003404E
:1079400010600340A28F0100308EFF1FD4CBFF1FB9
:107950001B800040517700000092FF1F0229044B5A
:107960001A780CBF02F0BF0242F040021A70704752
:1079700021C00C4008B503480349044A06F0EEFD57
:1079800008BD00BFCCCBFF1FA17500003C98FF1FB6
:1079900008B503480349044A06F0E0FD08BD00BFEE
:1079A000DCCBFF1FA17500003C98FF1F08B5034802
:1079B0000349044A06F0D2FD08BD00BFE4CBFF1F17
:1079C000A17500003C98FF1F08B503480349044A0D
:1079D00006F0C4FD08BD00BFECCBFF1FA175000081
:1079E0003C98FF1F08B503480349044A06F0B6FD5A
:1079F00008BD00BFF4CBFF1FA17500003C98FF1F1E
:107A000008B503480349044A06F0A8FD08BD00BFB5
:107A1000FCCBFF1FA17500003C98FF1F10B504466A
:107A20000C2380F87F3280F8803200234366006F99
:107A300018B104F07FF900232367606F18B104F0D8
:107A400079F90023636710BD38B5044672B690F823
:107A50007F320C2B1FD0006F00232367656F636795
:107A60000C2384F87F3262B608B104F063F915B1D3
:107A7000284604F05FF904F1180001F0DFFA074B23
:107A80001B8823B1013B9BB2044A138023B95E20BB
:107A900000F030FC38BD62B638BD00BF04CCFF1F1B
:107AA00030B58FB004460D46FFF7CEFF5E2000F0E4
:107AB00007FC2E4B1A8801321A8072B601A829469B
:107AC000002201F049F89DF808302377039B2362D8
:107AD0009DF8103084F82430059BA362069BE36276
:107AE000079B2363089B6363099BA3639DF828306E
:107AF00084F83C309DF8293084F83D300EAB53F8C3
:107B00000E5D58689968C4F83E50C4F84200C4F845
:107B100046101B7B84F84A3001A801F07BF962B65D
:107B200094F83D30032B0DD9104B1B882BB1013B32
:107B30009BB20E4A13800020ABB95E2000F0DAFB46
:107B4000002010E00023A4F87C32A4F87A320C2242
:107B500084F880221422626684F87E32082384F836
:107B60007F320120FFE70FB030BD00BF04CCFF1F04
:107B7000C36C9AB2012A2AD1026D4AF644418A4264
:107B80000AD045F222618A4209D042F611318A4276
:107B90001FD11349042204E01249002201E01249D6
:107BA00004221B0C012B04D0022B14D1490842F0F3
:107BB0000102B0F85A30082B04D0102B0DD149081F
:107BC00042F00202C16680F8802201207047002046
:107BD000704700207047002070470020704700BFAA
:107BE00034EE35178D7BCD051AF79A0B2DE9F84F3A
:107BF0000446B0F87A6206447A360D46002900F051
:107C0000B4814FF008090027DFF898B3DFF898A394
:107C100002E0002D00F0AC8194F87F320C2B00F2D2
:107C20009C81DFE813F0A801A801D8002601A80173
:107C3000A801A801A8010D004F007F00BC00A80109
:107C4000636E9D4234BFA846984604F14C0094F8F8
:107C50007E3218443146424602F058F994F87E329A
:107C6000434484F87E32B4F87A324344A4F87A323A
:107C7000636EC8EB03036366002B40F07F81E36C07
:107C8000534540F06A81636DC54A934240F0658177
:107C9000A36D02F15B4202F5F11202F60F4293422C
:107CA00040F05B81E36DA3F11002082A00F25581D8
:107CB0004644C8EB0505636684F87E72092384F8A0
:107CC0007F32A6E7636E9D4234BFA846984604F112
:107CD0004C0094F87E3218443146424602F016F9C0
:107CE00094F87E32434484F87E32B4F87A324344C6
:107CF000A4F87A32636EC8EB03036366002B40F08E
:107D000040812046FFF734FF002800F026814644DA
:107D1000C8EB0505C4F8649084F87E720A2384F8E1
:107D20007F3276E7636E9D4234BFA846984604F1E1
:107D30004C0094F87E3218443146424602F0E6F890
:107D400094F87E32434484F87E32B4F87A32434465
:107D5000A4F87A32636EC8EB03036366002B40F02D
:107D600013814644C8EB0505236D6366E36C5B45F0
:107D700011D184F8817294F8803284F87F3213F044
:107D8000010F05D003F07AFF6067002800F0FF8044
:107D9000636EA3663DE70B2384F87F3239E7636E99
:107DA000AB4209D95B1B6366B4F87A321D44A4F870
:107DB0007A520020BDE8F88F1E44ED1AB4F87A22FA
:107DC0001344A4F87A32C4F8649084F87E720A23CB
:107DD00084F87F321DE7636E9D4228BF1D465B1B02
:107DE0006366023616F8021C16F8010C023D226F7B
:107DF000B4F8783003F1010CA4F878C002EB430327
:107E000041EA00229A80B4F878307F2B24D92046AA
:107E1000216F002203F0AEFF2046216F012203F004
:107E2000A9FF206F03F086FF00232367636E1D44C4
:107E3000656604F17A03F71AA4F87A72606F08B1E4
:107E400003F078FF636E002B40F0A4800C2384F8CD
:107E50007F320120BDE8F88F0236002DC2D1636E5B
:107E6000002B40F09A800C2384F87F320020BDE87C
:107E7000F88F636E9D4228BF1D465B1B636694F8B6
:107E800081325BB1236FB4F8782003EB4202E36CDC
:107E90009380002384F8813219E03E46337872786B
:107EA000023D0BD1616E002951D043EA0223E36405
:107EB000022384F881320020BDE8F88F0236216F5A
:107EC000B4F8780001EB400143EA02238B80374687
:107ED00017F8021B7078023D626FB4F878305E1CB0
:107EE000A4F8786002EB430341EA00229A80B4F8D8
:107EF00078307F2B22D92046216F002203F03AFFF1
:107F0000206F03F017FF002626672046616F0122CD
:107F100003F030FF606F03F00DFF6667636E1D4472
:107F2000656604F17A03FF1AA4F87A72002D3DD138
:107F30000C2384F87F320120BDE8F88F002DACD1EE
:107F4000636E23B1002084F88102BDE8F88F0C2312
:107F500084F87F320020BDE8F88F0C2384F880324B
:107F600084F87F320020BDE8F88F0020BDE8F88F4C
:107F70000020BDE8F88F0020BDE8F88F0020BDE8A4
:107F8000F88F0020BDE8F88F0020BDE8F88F0020B2
:107F9000BDE8F88F0120BDE8F88F0020BDE8F88F1C
:107FA0005741564564617461524946460120BDE817
:107FB000F88F00BF90F87F0207288CBF00200120B7
:107FC000704700BF90F87F32072B07D8826E436E50
:107FD000D21AC16EA2FB01231846704700207047D9
:107FE00090F87F32072B05D8C36E826EA2FB032365
:107FF00018467047002070472DE9D847044690F88E
:108000007F320C2B00F0AD8003F038FE2067002893
:1080100000F0A78094F87F32072B0BD813F0010FE4
:1080200008D003F02BFE606730B9206F03F082FEAA
:10803000BDE8D887002363670023A4F87830B4F83C
:108040007C12B4F87A32C91A002905DD2046FFF700
:10805000CDFD002840F0858094F87F320C2B2CD089
:1080600004F11806304600F0B5FE30B304F17A088A
:108070004FF400774FF00009304641463A4600F091
:10808000D5FE83B2A4F87C32BBB1A4F87A9294F8FE
:108090007FA220461946FFF7A9FD20B194F87F3250
:1080A0000C2B5ED109E094F87F320C2B05D0BAF18D
:1080B000070F16D9072BDFD913E004F1180000F0E1
:1080C000BDFF294B1B8823B1013B9BB2264A13807D
:1080D00013B95E2000F00EF90C2384F8803284F886
:1080E0007F32236F1BB3B4F87820DAB113467F2AAE
:1080F00007D80021226F02EB430291800133802BCD
:10810000F8D12046216F002203F034FE94F87F322C
:10811000072B07D813F0010F04D12046216F01224D
:1081200003F028FE206F03F005FE00232367636F32
:10813000BBB1B4F878207AB113467F2A07D8002162
:10814000626F02EB430291800133802BF8D120460D
:10815000616F012203F00EFE606F03F0EBFD002360
:108160006367BDE8D88700BF04CCFF1F70B5054624
:1081700090F8303013F0FF0F4FD003F07FFD06462C
:1081800000284AD0296AEB6999421FD201F5807212
:10819000934232D25C1AA8690844311D224601F08C
:1081A000D7FA2B6A23442B62EB6A2344EB62630801
:1081B0007F2B1DD904E022F8024F01337F2BFAD91F
:1081C00028463146002203F0D5FD0DE0134B1B88F5
:1081D00023B1013B9BB2114A138013B95E2000F01A
:1081E00089F8002385F83030304603F0A3FD70BDD8
:1081F00006EB430202320024DDE7A8690844311D82
:108200004FF4807201F0A4FA2B6A03F580732B629D
:10821000EB6A03F58073EB62D2E770BD04CCFF1FFD
:10822000002380F83030C36283627047184B1A68AD
:1082300042F480521A60174B174A1A60174ADA60E4
:1082400002F180421A61164A1A60164B1B7813F02D
:10825000010F07BF4FF41072134B4FF40072134B12
:108260001A60104B1B7813F0020F4FF400720CBF12
:108270000F4B104B1A600B4B1B7813F0040F07BF0A
:108280004FF410720C4B4FF400720C4B1A60704795
:108290003C80044000C0024001401F000110003833
:1082A00000001F8010DDFF1F18B0044008C004400C
:1082B0001CB004400CC0044014B0044004C004408E
:1082C00030B45E2810D84309084A012101FA03F5A9
:1082D00014782C431470064A00F01F00814052F8B5
:1082E00023400C4342F8234030BC704720CCFF1F92
:1082F00008CCFF1F5E2815D8430900F01F0001229B
:1083000002FA00F0084A52F8231021EA000042F86D
:10831000230038B9054A012101FA03F3117821EA53
:1083200003031370704700BF08CCFF1F20CCFF1F52
:1083300072B60D4B4FF0FF30002203F65461C3F8C4
:10834000000283F8082283F8092203F5037343F837
:10835000083C8B42F3D3002243F8082C024A034B1B
:108360001A6062B6704700BF28CCFF1F24CCFF1FE5
:1083700003684BB172B6036893F80822013A83F898
:10838000082262B600230360704700BF2DE9F8435E
:1083900080460F4691462C4B1B680BB9FFF7C8FF70
:1083A000D8F8000030B1D0F80032BB424AD0404685
:1083B000FFF7DEFF72B6244B1868034600252E46F1
:1083C0002A46D3F80012B94214D119463AB1D3F86B
:1083D0000442C2F80442C3F804021B4A136091F835
:1083E0000822013281F8082262B6C8F80010184647
:1083F000BDE8F88393F80842002C08BF1546002C0E
:1084000008BF1E46D3F8044214B11A462346D8E7E3
:10841000B9F1000F13D096B13DB1D6F80432C5F8CA
:108420000432C6F80402084B1E60012386F80832A5
:10843000C6F80072002386F80932C8F8006062B6F8
:10844000D8F80000BDE8F88324CCFF1FF8B50D462E
:1084500017463D4B1B78002B28D072B63A4B1B7841
:1084600013F0010F07D0394B1968394A12680A40D6
:1084700038490A601A60344B1B7813F0020F07D09A
:10848000354B1968324A52680A4032494A601A60CC
:108490002D4B1B7813F0040F07D0304B19682C4A72
:1084A00092680A402B498A601A6062B62C4BDB68DE
:1084B000B3F1384F0AD02A4B2A4A1A604FF038429B
:1084C000DA604FF078421A61274A1A602946012281
:1084D000FFF75CFF0446A8B190F8093213F0010FD2
:1084E00001D0064611E006462846214600F0BCF9B8
:1084F00050B11FB9012384F8093206E0052384F83E
:10850000093202E0002600E000260F4B1B78C3B1C1
:1085100013F0010F03D00F4B1A68144B1A600A4B6B
:108520001B7813F0020F03D00A4B5A68104B1A60E5
:10853000054B1B7813F0040F03D0064B9A680D4BC4
:108540001A603046F8BD00BF20CCFF1F80E100E07C
:1085500008CCFF1F14CCFF1F84E100E088E100E09D
:1085600000C0024001401F0000001F8000E100E049
:1085700004E100E008E100E0F8B505460E461746C4
:10858000414B1B78002B28D072B63F4B1B7813F061
:10859000010F07D03D4B19683D4A12680A403D491A
:1085A0000A601A60384B1B7813F0020F07D03A4B61
:1085B0001968374A52680A4036494A601A60324B95
:1085C0001B7813F0040F07D0344B1968304A9268B7
:1085D0000A4030498A601A6062B6314BDB68B3F1F9
:1085E000384F0AD02E4B2F4A1A604FF03842DA60CB
:1085F0004FF078421A612C4A1A6028463146002210
:10860000FFF7C4FE044620B190F8093213F0010FC1
:1086100005D13046394600F027F9064600E001262C
:10862000194B1B78C3B113F0010F03D0194B1A6813
:108630001E4B1A60144B1B7813F0020F03D0154B1E
:108640005A681B4B1A60104B1B7813F0040F03D0B1
:10865000104B9A68174B1A60A4B194F8093213F0C2
:10866000010F0AD0384621464FF4007201F04EFC4B
:108670002846FFF77DFE0120F8BD2846FFF778FE6B
:108680003046F8BD3046F8BD20CCFF1F80E100E049
:1086900008CCFF1F14CCFF1F84E100E088E100E05C
:1086A00000C0024001401F0000001F8000E100E008
:1086B00004E100E008E100E01B4B1B68012283F8A5
:1086C00000211A4B4FF00042DA62020A5A631A463E
:1086D000D36A002BFCDA154B9A6B4FF00042DA623A
:1086E0000A0C42F080525A631A46D36A002BFCDA15
:1086F0000E4B9A6B4FF00042DA6289B241F0805122
:1087000059631A46D36A002BFCDA084B9A6B4FF078
:108710000042DA62C0B258631A46D36A002BFCDA10
:10872000024B9B6B704700BF7CDAFF1F00C002400A
:1087300030B40921094A4FF00045FF24D562546343
:10874000D36A002BFCDA906B10F0800F03D04B1E25
:1087500013F0FF01F2D1C0B230BC704700C002403C
:108760000D4B4FF00042DA620C4A5A631A46D36A44
:10877000002BFCDA084B986B00044FF00042DA62E1
:10878000064A5A631A46D36A002BFCDA024B9B6BEB
:108790009BB21843704700BF00C00240FFFF0010AB
:1087A000084B1B68012283F88020074B4FF00042E2
:1087B000DA62FF225A631A46D36A002BFCDA024BB4
:1087C0009B6B70477CDAFF1F00C0024010B544F27B
:1087D00095000021FFF770FFFFF7AAFF0446FFF79F
:1087E000DFFF204610BD00BF10B544F687004FF4F0
:1087F000D571FFF761FFFFF79BFF012818BF4FF00E
:10880000004403D1FFF7ACFF0446FFE7FFF7C8FFC2
:10881000204610BD10B5044647F2FF700021FFF757
:108820004BFFFFF785FFFFF7BBFF46F6FF10214622
:10883000FFF742FFFFF77CFF0446FFF7B1FF20463A
:1088400010BD00BF10B547F6FF200021FFF734FF31
:10885000FFF76EFF18B9FFF783FF044600E000241E
:10886000FFF79EFF204610BD70B503460D46324A05
:108870001278012A98BF430245F2FF101946FFF70C
:108880001BFFFFF755FF18B1FFF78AFF002070BDEF
:108890002A4A4FF00044FF20D4625063D36A002B71
:1088A000FCDA936BDBB2FE2B05D0FF2BF4D0FFF785
:1088B00077FF002070BD05F5FF76204B204A5A63F4
:1088C0005A63B54213D2A81C05F500751A461C4C14
:1088D000D36A13F0F00FFBD05463936B190A00F8BE
:1088E000021C00F8013C0230A842F1D100E02E4603
:1088F000124AD36A13F0F00FFBD0104B9B6B1A0A8D
:10890000327073700D4AD36A13F0F00FFBD00B4B2B
:108910009A6B0C4A1268012182F880104FF00042D5
:10892000DA62FF225A631A46D36A002BFCDA034B41
:108930009B6B012070BD00BF80DAFF1F00C00240AA
:10894000FFFF00107CDAFF1F10B400230361CB6926
:1089500043618A8A4B8B43EA02438361C361CB7ACA
:1089600003F01003DBB2002B0CBF0023022380F8BE
:1089700025300A78202A08BF00F1260308D020E01D
:1089800014F8012F202A03D003F8012B8342F7D1DA
:108990000A7A202A12D02E221A700A7A5A704A7A3B
:1089A000202A02D1981C093102E0D81C0A319A70A1
:1089B0000A78202A1ABF431C0270034600221A704C
:1089C00006E000F1270380F826200C462E30D7E77A
:1089D0005DF8044B704700BF2DE9F04F87B00646A5
:1089E00091460B78002B00F0A3802F2B0DD1A5E032
:1089F00011F8013F002B00F0A2802F2B0CD19EE03C
:108A000002F8011B9A42FBD321E003AA05A8202407
:108A10000DF1150C0DF117052E2B0BD1824214D23E
:108A2000134603F8014B8342FBD1531CC3EB0C03E9
:108A30001A440AE07E2B08D8A3F16107FFB2192F70
:108A40009CBF203BDBB213700132AA42D0D396F810
:108A50002530032B05D1D6F818B073695B0A019352
:108A60000EE0022B66D1B269F261394B1B78023AF3
:108A700002FA03FB374A1268934401229A4001929A
:108A80000021009101278A4639E006A840F810AD80
:108A900059465246FFF7DAFC044648B355464FF0B4
:108AA0000B08204603A9424606F04EF828B948466E
:108AB0002146FFF749FF01241DE023783FB10BB1A8
:108AC000E52B05D1C9F820B089F8245057468BB161
:108AD00033692033336120340135102DE1D10BF19E
:108AE000010B02A8FFF744FC009A0132009206E055
:108AF000002400E0002402A8FFF73AFC23E0009BDA
:108B000001998B42C1D396F82530032B14D03046FF
:108B100000F012F90446B0B1F369023B0C490A783F
:108B200003FA02FB0B4A13689B44CDF800A0E6E76A
:108B3000002408E0002406E0002404E003AA202129
:108B40000DF117035CE7204607B0BDE8F08F00BFCA
:108B50008CDAFF1F88DAFF1F30B59BB005460C4644
:108B600000F048F9684B1A798DF804209A6802924F
:108B70001A7B8DF80C20654A00921A6904925A6992
:108B800005929A690692DA6907921A6A089293F82E
:108B900024208DF8242093F825208DF8252053F8E3
:108BA000260F59689A68CDF82600CDF82A10CDF81E
:108BB0002E201B7B8DF8323000E0013423782F2BE0
:108BC000FBD043BB9DF804302B71029BAB609DF83A
:108BD0000C302B73049B2B61059B6B61069BAB6177
:108BE000079BEB61089B2B629DF8243085F82430AD
:108BF0009DF8253085F825301AAB53F8424D58685A
:108C00009968C5F82640C5F82A00C5F82E101B7BC8
:108C100085F8323071E00DA800F0ECF86846214686
:108C20000DAAFFF7D9FE631C1C4613F8012B2F2A4F
:108C30005DD0002AF8D15DE09DF838302B710F9B94
:108C4000AB609DF840302B73119B2B61129B6B61C5
:108C5000139BAB61149BEB61159B2B629DF8583005
:108C600085F824309DF8593085F825301AAB53F833
:108C70000E4D58689968C5F82640C5F82A00C5F811
:108C80002E101B7B85F832302DE09DF838308DF8A2
:108C900004300F9B02939DF840308DF80C30119BEF
:108CA0000493129B0593139B0693149B0793159BA8
:108CB00008939DF858308DF824309DF859308DF880
:108CC00025301AAB53F80E0D59689A68CDF8260076
:108CD000CDF82A10CDF82E201B7B8DF832300DA850
:108CE00000F098F86AE70DA800F094F805E0002875
:108CF000CBD1F8E700289FD1F5E7684600F08AF865
:108D000028461BB030BD00BF90DAFF1FC00901002C
:108D100010B58EB0014601A80022FFF71DFF9DF897
:108D20002940032C8CBF0024012401A800F072F814
:108D300020460EB010BD00BF30B583B004460023FE
:108D40000193174B1968C569164B1B78102B0AD174
:108D500001A801EB15210122FFF778FBB0B1EDB2BC
:108D600030F815300AE001A801EBD5110122FFF718
:108D70006DFB68B105F07F0550F82530E3610A4AC4
:108D80001468A3428CBF0024012402E0002400E008
:108D9000002401A8FFF7ECFA204603B030BD00BF65
:108DA000C4DAFF1FC8DAFF1FCCDAFF1F10B582B08C
:108DB00002AB03F8011D0268546819460122A0475E
:108DC00002B010BD90F82530012B1CBF01230371A8
:108DD0000020704790F82530012B07D803694069BF
:108DE000C01A0028B8BF6FF00040704700207047DD
:108DF000704700BF002202714FF47A7181600273E4
:108E000003490160042180F8251080F8262070476E
:108E1000C0090100044A0260042280F825200022D3
:108E200080F82620704700BFC00901002DE9F04FEF
:108E300083B00646884690F82530012B00F2A380C7
:108E400003694169C91A8A4234BF91468946B9F11A
:108E5000000F00F09A804F4A127802F109010120B8
:108E600000FA01F101390B40F1698C1E94404A4A25
:108E70001068044404EB5324C3F30805002D3CD0D0
:108E8000002202A840F8042D2146FFF7DFFA014630
:108E900010B3C5F5007BCB4509D9404629444A4665
:108EA00001F034F833694B4433614D4615E04046D8
:108EB00029445A4601F02AF833695B44336101A81A
:108EC000FFF756FA0134334B1B78012202FA03F301
:108ED000013B1C420BD104E0002501A8FFF748FA32
:108EE00054E03046FFF728FF08B95D464EE0CB4519
:108EF00001D2D84403E05D4648E04FF0000BCBEBD5
:108F000009075D46CBEB080BDFF888A00BEB0508E3
:108F100000230193B7F5007F0FD201A821461A461E
:108F2000FFF794FA014608B340463A4600F0EEFFD8
:108F300033693B4433614D4618E001A8214642465F
:108F4000FFF71AFB90B1336903F50073336105F540
:108F5000007501A8FFF70CFA01349AF800300122DD
:108F600002FA03F3013B1C4208D103E001A8FFF71A
:108F7000FFF90BE03046FFF7DFFE38B1A7F50077C9
:108F8000A945C3D802E0002500E00025284603B02B
:108F9000BDE8F08F8CDAFF1F88DAFF1F00B583B0C1
:108FA0000DF107010122FFF741FF01280CBF9DF8D9
:108FB00007004FF0FF3003B05DF804FB70B582B0DE
:108FC00004460669C5690DF107010122FFF72EFF6E
:108FD000012803BF2661E5619DF807004FF0FF30CF
:108FE00002B070BDF8B505460E4690F82530012B4D
:108FF0001DD843698B421CD3C7690F4B1B780933BB
:1090000021FA03F4026922FA03F3E31A52BF1C4661
:109010008369C36144B12846FFF78EFE034608B951
:10902000EF6107E0013CF6D12E61012302E000234D
:1090300000E000231846F8BD8CDAFF1F042380F8F7
:109040002530002380F82630704700BF2DE9F04F0F
:1090500087B07D4D7D4B53F830302B6001247C4B25
:109060001C70214601F0A8FA2B6883F88040FFF7B6
:10907000DDF8784B1B78002B28D072B6754B1B7827
:1090800013F0010F07D0744B1968744A12680A4034
:1090900073490A601A606F4B1B7813F0020F07D0F8
:1090A000704B19686D4A52680A406D494A601A60EF
:1090B000684B1B7813F0040F07D06B4B1968674A95
:1090C00092680A4066498A601A6062B6674BDB683C
:1090D000B3F1384F0AD0654B654A1A604FF03842F9
:1090E000DA604FF078421A61624A1A6005215F4ADD
:1090F0004FF000446048D4625063D36A002BFCDA1E
:10910000936B4B1E13F0FF01F5D15C4B1B68029370
:10911000029D504CDFF87491DFF86CA1DFF84881B4
:10912000504F4D4EFFF752FB012858D02378B3B172
:1091300013F0010F03D04A4B1A68514B1A60237881
:1091400013F0020F03D0464B5B68CAF80030237857
:1091500013F0040F03D0424B9B68C9F80030474B13
:109160001B680393039B5B1BFA2B00F2C1812378DE
:1091700023B372B6237813F0010F06D03268374B51
:109180001B681340364A13603360237813F0020FD4
:1091900006D03A68314B5B681340314A53603B60FC
:1091A000237813F0040F08D0D8F800202B4B9B68CD
:1091B00013402B4A9360C8F8003062B62B4BDB6833
:1091C000B3F1384FAED0294B294A1A604FF03842DC
:1091D000DA604FF078421A61264A1A60A2E7FFF778
:1091E00003FBB0F1004F04D10122264B1A70002579
:1091F0004EE0B0F5D57F05D10222224B1A704FF018
:10920000804545E0134B1B78002B00F0738113F071
:10921000010F03D0124B1A68194B1A600D4B1B78C3
:1092200013F0020F03D00E4B5A68174B1A60094B0C
:109230001B7813F0040F00F05F81094B9A68134B01
:109240001A6000245DE100BF7CDAFF1F240A0100E0
:1092500081DAFF1F20CCFF1F80E100E008CCFF1F58
:1092600014CCFF1F84E100E088E100E000C0024070
:1092700001401F0000001F80FFFF001050DBFF1F98
:1092800000E100E080DAFF1F04E100E008E100E017
:109290009E4B1B680493049E9D4CDFF89CA2DFF854
:1092A00094B2DFF8B492DFF8B4829A4F2846FFF701
:1092B000B1FA024600285FD02378B3B113F0010F52
:1092C00003D0954B1968954B1960237813F0020F62
:1092D00003D0914B5B68CBF80030237813F0040F78
:1092E00003D08D4B9B68CAF80030012A00F206813A
:1092F000864B1B680593059A921B40F2DC539A42F9
:1093000000F2FE80237833B372B6237813F0010F96
:1093100006D03A68824B1B6813407F4A13603B605B
:10932000237813F0020F08D0D8F800207C4B5B683C
:109330001340794A5360C8F80030237813F0040FC3
:1093400008D0D9F80020764B9B681340724A93608E
:10935000C9F8003062B6734BDB68B3F1384FA5D063
:10936000704B714A1A604FF03842DA604FF0784221
:109370001A616E4A1A6099E76D4B1B78022B07D170
:10938000FFF760FA800F032802D10322684B1A709E
:109390005F4B1B78C3B113F0010F03D05E4B1A680B
:1093A0005E4B1A605A4B1B7813F0020F03D05A4BD6
:1093B0005A68604B1A60564B1B7813F0040F03D0A9
:1093C000554B9A685C4B1A60002206A840F8142D91
:1093D0001146FFF73BF8B0F8FE214AF655239A42B2
:1093E00077D190F8C231062B03D00B3BDBB2012BB7
:1093F00002D8D0F8C64100E0002401A8FEF7B8FF6B
:1094000001A821460022FFF721F8B0F8FE214AF614
:1094100055239A425FD1B0F80B30B3F5007F5CD191
:10942000037C022B5BD1C589002D5AD0427BB2FA56
:1094300082F2C2F11F02414B1A70C38A03B9436A18
:10944000B0F8117007F10F0E4FEA1E1EB0F813604E
:1094500006B9066A61193A4C21601944394C2160F9
:1094600003EB0E0C8C44384CC4F800C0741BCEEBDC
:109470000404A4EB430424FA02F2551C334C256087
:1094800040F6F474A2422ED94FF6F474A2420BD8DF
:1094900010202F4A10702F4A7F0157610B449361AF
:1094A000032382F825300AE02022294B1A70294B29
:1094B00000225A61C26A9A61022283F82520254B54
:1094C0009A69DA6100221A6101A8FEF751FF0124AE
:1094D0000AE0002408E0002406E0002404E0002460
:1094E00002E0002400E0002401A8FEF741FF08E0AC
:1094F000002406E0002404E0002402E0002400E050
:109500000024204607B0BDE8F08F00BF50DBFF1FEE
:1095100020CCFF1F80E100E014CCFF1F00E100E041
:1095200008CCFF1F00C0024001401F0000001F8048
:1095300080DAFF1F04E100E008E100E08CDAFF1FA1
:10954000C4DAFF1F84DAFF1F88DAFF1FCCDAFF1F9F
:10955000C8DAFF1F90DAFF1F88E100E084E100E035
:1095600010B5054C2046FFF745FC20460349044A48
:1095700004F0F4FF10BD00BF90DAFF1F158E00004D
:109580003C98FF1F014A024B1A60704701100138D6
:10959000D0DAFF1F2DE9F0075E495F4E5F48604D4E
:1095A000604C614BDFF8A0A1DFF8A0C10A782AB3B4
:1095B00072B60A7812F0010F07D0226807683A40A5
:1095C000DFF87881C8F8002022600A7812F0020FD4
:1095D00007D02A6847683A40DFF86081C8F804205D
:1095E0002A600A7812F0040F07D0326887683A4080
:1095F000DFF84881C8F80820326062B6DA68B2F154
:10960000384F09D0494A1A604FF03842DA604FF0BB
:1096100078421A61464A1A60464AD2F8008001220E
:1096200088F80021444A127812F0020F35D04FF02A
:109630000042DA6270225A63DA6A002AFCDA9A6B14
:109640004FF00042DA6200225A63DA6A002AFCDA3A
:109650009A6B5FFA82F9012288F880200A78C2B1F9
:1096600012F0010F05D0354AD2F80080344AC2F812
:1096700000800A7812F0020F03D0304A5268CCF80A
:1096800000200A7812F0040F03D02C4A9268CAF81E
:10969000002019F0800F89D035E04FF00042DA62E7
:1096A00005225A63DA6A002AFCDA9A6B4FF000420C
:1096B000DA6200225A63DA6A002AFCDA9A6B5FFAED
:1096C00082F9012288F880200A78C2B112F0010FD5
:1096D00005D01A4AD2F80080194AC2F800800A78E8
:1096E00012F0020F03D0154A5268CCF800200A7815
:1096F00012F0040F03D0114A9268CAF8002019F042
:10970000010F7FF453AF00220E4B1A70BDE8F00733
:10971000704700BF20CCFF1F88E100E008CCFF1F8E
:1097200084E100E080E100E000C0024001401F0051
:1097300000001F80D8DAFF1FD4DAFF1F14CCFF1FF0
:1097400000E100E0D5DAFF1F08E100E004E100E0FD
:109750002DE9F04F85B080468A46914608460021A3
:1097600005F086FA7D4B1B7803937D4B1B78002B0D
:1097700028D072B67A4B1B7813F0010F07D0794BC3
:109780001968794A12680A4078490A601A60744B6D
:109790001B7813F0020F07D0754B1968724A526894
:1097A0000A4072494A601A606D4B1B7813F0040F2F
:1097B00007D0704B19686C4A92680A406B498A60FE
:1097C0001A6062B66C4BDB68B3F1384F0AD06A4B53
:1097D0006A4A1A604FF03842DA604FF078421A61F4
:1097E000674A1A60674B1B780293002B00F02B81AD
:1097F000654B1B68012283F80021584B1B7813F03E
:10980000020F1BD05C4B4FF00042DA6270225A63A9
:109810001A46D36A002BFCDA574B9A6B4FF0004282
:10982000DA6200225A631A46D36A002BFCDA524BE2
:109830009B6B13F0800F00F0D681F9E14E4B4FF097
:109840000042DA6205225A631A46D36A002BFCDA18
:10985000494B9A6B4FF00042DA6200225A631A4673
:10986000D36A002BFCDA444B9B6B13F0010F00F022
:10987000DF81B8E1012381F800313F4B4FF0004216
:10988000DA6206225A631A46D36A002BFCDA3A4B94
:109890009B6B012381F880302023013B7FF4FDAFD7
:1098A000039A12F0040F05D0029B012B0CBF8522F6
:1098B000752200E07522012381F800312E4B4FF014
:1098C0000040D8625A631A46D36A002BFCDA2A4B4E
:1098D0009B6B012381F88030039A12F0020F1DD098
:1098E00081F80031244B4FF00042DA6270225A6353
:1098F000DA6A002AFCDA204B9B6B1F4A4FF00044C7
:109900000020D4625063D36A002BFCDA936B13F00F
:10991000800FF6D0012381F8803094E0012381F894
:109920000031154B4FF00042DA6205225A63DA6AC1
:10993000002AFCDA104B9B6B0F4A4FF000440020CA
:10994000D4625063D36A002BFCDA936B13F0010FDF
:10995000F6D1012381F8803075E000BFD4DAFF1F13
:1099600020CCFF1F80E100E008CCFF1F14CCFF1FBC
:1099700084E100E088E100E000C0024001401F00F7
:1099800000001F80D5DAFF1FD8DAFF1F9B4B1B7822
:10999000C3B113F0010F03D0994B1A68994B1A60A9
:1099A000964B1B7813F0020F03D0954B5A68964BD9
:1099B0001A60924B1B7813F0040F03D0904B9A68F7
:1099C000924B1A60FFF7E6FD8C4B1B78002B28D0DA
:1099D00072B68A4B1B7813F0010F07D08C4B1968B5
:1099E0008C4A12680A4086490A601A60834B1B78C9
:1099F00013F0020F07D0884B1968864A52680A4054
:109A00007F494A601A607D4B1B7813F0040F07D022
:109A1000824B19687F4A92680A4079498A601A60C5
:109A200062B67F4BDB68B3F1384F0AD07C4B7D4A7E
:109A30001A604FF03842DA604FF078421A617A4A81
:109A40001A6000230293039901F00803DBB200932C
:109A5000DFF8D8C1012001EA00020192704B4FF0FB
:109A60000042009961B108EB0901013981EA08015E
:109A700011F07E4F06D028F07E4BCBF1007B02E048
:109A8000CB4600E0CB46DCF8001081F800010199DC
:109A9000D9B1DA6203215963D96A0029FCDA996BDA
:109AA000DA624FEA184141F080515963D96A0029BE
:109AB000FCDA996BDA621FFA88F141F08051596340
:109AC000D96A0029FCDA996B15E0DA62C8F307411C
:109AD00041F0805141F440715963D96A0029FCDAA0
:109AE000996BDA621FFA88F141F080515963D96AA3
:109AF0000029FCDA996BBBF1000F18D09AF800101E
:109B00001C6844F480641C60DA625963BBF101078D
:109B100007D0574451464D78DC6A002CC0F2928041
:109B2000FAE75746D96A0029C0F29980FAE7DCF8CB
:109B3000004084F88000DA44D844B9EB0B0990D196
:109B4000029A002A31D0012384F80031344B4FF0BF
:109B50000042DA6206225A631A46D36A002BFCDA04
:109B60002F4B9B6B012384F880302023013B7FF433
:109B7000FDAF039B13F0040F05D0029901290CBF20
:109B80008A227A2200E07A22012384F80031244BD1
:109B90004FF00041D9625A631A46D36A002BFCDAAF
:109BA0001F4B9B6B012384F88030144B1B78002BD8
:109BB00058D013F0010F03D0114B1A68114B1A60E3
:109BC0000E4B1B7813F0020F03D00D4B5A680E4B4F
:109BD0001A600A4B1B7813F0040F43D0084B9A68A5
:109BE0000A4B1A603EE0114B1968012381F880305E
:109BF000029A022A7FF63EAEC8E600BF20CCFF1FC5
:109C000014CCFF1F00E100E004E100E008E100E007
:109C100080E100E008CCFF1F84E100E088E100E083
:109C200000C0024001401F0000001F80D8DAFF1F63
:109C30000E4B1B68012283F8802000230C4A13700E
:109C4000029300E79C6B1E6846F480661E60DA6231
:109C50005D6301F8014BB9427FF45DAF62E7996B38
:109C6000397064E705B0BDE8F08F00BFD8DAFF1F98
:109C7000D5DAFF1F0B4B1B7813B90B4B1B7873B155
:109C80000A4B1B78202B03D9012303710020704756
:109C9000581C064A1070064AD15401207047002013
:109CA000704700BF46DBFF1F08DBFF1F47DBFF1FBE
:109CB000E4DAFF1F704700BF024B1878024B1B7895
:109CC000C01A704745DBFF1F44DBFF1F074B1B78A3
:109CD000074A12789A4205D9591C044A1170054A5C
:109CE000D05C70474FF0FF30704700BF44DBFF1F70
:109CF00045DBFF1F0CDBFF1F054B1B78054A127865
:109D00009A4286BF044AD05C4FF0FF30704700BFD4
:109D100044DBFF1F45DBFF1F0CDBFF1F08B5104BAB
:109D2000DB7813F0200F0CD1122000F0B9FB0D4BA3
:109D30001B689BB100210C4A11700C4A107898479F
:109D400008BD0B4A13780133DBB21370012B02D824
:109D5000084B1B7813B9122000F0A2FB08BD00BF0E
:109D600000600640E0DAFF1F44DBFF1F45DBFF1FFA
:109D700030DBFF1F08DBFF1F38B514460D4B1B7887
:109D800013B90D4B1B7893B10C4B1D78C5F1210312
:109D9000A34202D2012202711C46094828442246ED
:109DA00000F0B4F82544054B1D70204638BD002056
:109DB00038BD00BF46DBFF1F08DBFF1F47DBFF1F6F
:109DC000E4DAFF1F002202714FF47A71816002739E
:109DD000014A0260704700BFE009010008B53D4B31
:109DE000DB78DBB213F0100F06D01021394AD170A6
:109DF00013F0400F03D108BD13F0400F2CD013F027
:109E0000040F1BD00023344A1370344A1370344BB0
:109E10001B681BB19847314B1B782BB901222F4B84
:109E20001A7000222F4B1A702A4BD0229A702D4A9A
:109E300012781A7101222C4B1A7009E00122264B6C
:109E40001A700022294B1A70224BC0229A701B797B
:109E50000222204BDA7008BD1E4A927812F0100FD1
:109E60001CD013F0010F14D11F4B1B781B4A127822
:109E70009A4207D9591C1C4A11701A4AD25C154BD8
:109E80001A7102E00022134B1A71D022114B9A7002
:109E90001BE0104BC0229A701B7916E00022144B75
:109EA0001A7012201349032200F0C6FB094B1B79DC
:109EB000DAB20E4B1B781F2B07D80749097821B15E
:109EC000581C0A4908700C49CA540222014BDA7026
:109ED00008BD00BF00600640DCDAFF1F47DBFF1F44
:109EE0002CDBFF1FE4DAFF1F48DBFF1F45DBFF1FF2
:109EF00030DBFF1F1D9D00000CDBFF1F08B5024873
:109F0000FFF760FF08BD00BF34DBFF1F844641EA56
:109F1000000313F003036DD1403A41D351F8043BE1
:109F200040F8043B51F8043B40F8043B51F8043B33
:109F300040F8043B51F8043B40F8043B51F8043B23
:109F400040F8043B51F8043B40F8043B51F8043B13
:109F500040F8043B51F8043B40F8043B51F8043B03
:109F600040F8043B51F8043B40F8043B51F8043BF3
:109F700040F8043B51F8043B40F8043B51F8043BE3
:109F800040F8043B51F8043B40F8043B51F8043BD3
:109F900040F8043B51F8043B40F8043B403ABDD242
:109FA000303211D351F8043B40F8043B51F8043BE4
:109FB00040F8043B51F8043B40F8043B51F8043BA3
:109FC00040F8043B103AEDD20C3205D351F8043B73
:109FD00040F8043B043AF9D2043208D0D2071CBF3F
:109FE00011F8013B00F8013B01D30B880380604668
:109FF000704700BF082A13D38B078DD010F00303DE
:10A000008AD0C3F10403D21ADB071CBF11F8013B4D
:10A0100000F8013B80D331F8023B20F8023B7BE79C
:10A02000043AD9D3013A11F8013B00F8013BF9D2C7
:10A030000B7803704B7843708B7883706046704761
:10A0400030B4394A3949136813F0800FFBD10B68DB
:10A0500013F0800FF7D172B6354B1B78002B5FD011
:10A06000344B1C6804331D680433186804331968C2
:10A0700004331A6804331B682C44204401440A4406
:10A080001A44C2F34E0242F400422B4B1A602C33A6
:10A090001C6804331D6804331868043319680433DA
:10A0A0001A6804331B682C44204401440A441A44AF
:10A0B000C2F34E0242F40042204B1A6003F108132F
:10A0C0001C6804331D6804331868043319680433AA
:10A0D0001A6804331B682C44204401440A441A447F
:10A0E000C2F34E0242F40042154B1A602C331C6836
:10A0F00004331D68043318680433196804331A687C
:10A1000004331B682C44204401440A441A44C2F31B
:10A110004E0242F400420B4B1A600022044B1A70AC
:10A1200062B630BC704700BF24B0034024B00B407F
:10A130004ADBFF1F38B003402CB0034030B003406F
:10A140002CB00B4030B00B4060223A4B1A70E12229
:10A1500001331A70384B1B78082B10D1012203F100
:10A16000804303F56C331A60132334490B6001F507
:10A17000FF2101F2FC710A60314A13601FE00A2BD3
:10A180000DD139222F4B1A6013232C490B6001F596
:10A19000FF2101F2FC710A60294A13600FE00C2BC9
:10A1A0000CBF35223D22274B1A60122323490B6036
:10A1B00001F5FF2101F2FC710A60214A1360224B74
:10A1C0001B7833B10123214A136002F5002213608A
:10A1D00005E000231D4A136002F5002213601C4BAA
:10A1E0001B78012B06D880231A4A136002F500223F
:10A1F00013601AE0042B06D88423164A136002F574
:10A200000022136011E0082B06D88523114A136041
:10A2100002F50022136008E0102B94BF86238723E9
:10A220000C4A136002F50022136001220A4B1A70D7
:10A23000704700BF00400740A7A5FF1F0CB00340B8
:10A240000CB00B4008B003404DDBFF1F20B00340B3
:10A25000A8A5FF1F24B003404ADBFF1F2DE9F843E8
:10A26000282873D83C4B1E5CFF2E72D03B4B1B78CA
:10A270000BB1FFF7E5FE16F0800F29D172B6384C0E
:10A28000384D4FF0010726602F7062B672B6236812
:10A2900013F0800F04D12B7813F0FF0F0FD1F2E7EA
:10A2A000314B186800222F4B1A7062B62F4B1B7867
:10A2B0001841BDE8F8832B7813F0FF0FE3D062B6A6
:10A2C00002F0F8F872B6236813F0800FF3D0E7E7D6
:10A2D00072B606F040095FFA89F9254F254C06F061
:10A2E0003F06254D4FF00108B9F1000F04D03B683F
:10A2F00023F010033B6003E03B6843F010033B6036
:10A30000266085F8008062B672B6236813F0800F6D
:10A3100004D12B7813F0FF0F0FD1E5E7174B186826
:10A320000022154B1A7062B6104B1B781841BDE81D
:10A33000F8832B7813F0FF0FD6D062B602F0BAF88C
:10A3400072B6236813F0800FF3D0E7E70020BDE872
:10A35000F8830020BDE8F883F80901004ADBFF1FFD
:10A3600000B003404CDBFF1F10B0034049DBFF1F70
:10A370000CB00B4000B00B404BDBFF1F10B00B408C
:10A38000024B1A6801321A60704700BF50DBFF1F92
:10A3900008B50D4C236813F4802F01D000F0D8FECF
:10A3A000236813F4806F01D000F05EFD236813F47E
:10A3B000006F01D002F0C2FB236813F4805FE9D084
:10A3C00002F07AFEE6E700BF3480044008B5FFF7EC
:10A3D000DFFF00BF1022014B1A80704700200540AC
:10A3E000704700BF024A136818441060184670474F
:10A3F000ACA5FF1FFEE700BFEFF31383ABB9EFF38C
:10A400001083ABB9EFF3058323B10F2B05D9094AAC
:10A41000985C03E04FF4807000E00020EFF31183BC
:10A420003BB1834238BF184670474FF0FF3070474A
:10A4300000207047F0E300E030B40023B0FBF2F4FA
:10A4400002FB14041D46092C94BF30343734E4B2A7
:10A45000CC54B0FBF2F008B10133EFE70D44002219
:10A460006A70934207DD885CCC5C8C54C85401321E
:10A47000013B9A42F7DB084630BC704710B50C46EA
:10A48000002802DBFFF7D8FF10BD2D2301F8013BA8
:10A490004042FFF7D1FF204610BD00BF704700BF0C
:10A4A0001D4B03EBC000436803F14042A2F592222A
:10A4B0007C2A18D903F14042A2F594227C2A14D9AF
:10A4C00003F14042A2F596227C2A10D903F14042C2
:10A4D000A2F598227C2A0CD903F14042A2F59A22D7
:10A4E0007C2A08D970470D4906E00D4904E00D4962
:10A4F00002E00D4900E00D4972B61A6822F0877239
:10A5000022F4803242F080721A60C3F38403084A56
:10A5100041F8232062B67047240A0100B0A5FF1F4E
:10A52000E8A5FF1F38A6FF1F68A6FF1F88A6FF1F0C
:10A530009DA40000044B00221A6004490A60044AEA
:10A54000106010221A60704714D0034004D00340FA
:10A5500000D0034021281ED80F4B53F8303093F819
:10A56000802212F0FF0F08D019B1012283F8802059
:10A570007047012283F800217047074B03EBC000AE
:10A58000436821B11A6842F003021A6070471A68E2
:10A5900022F002021A607047240A0100212806D81E
:10A5A000044B53F8303093F80002C0B270470020DB
:10A5B000704700BF240A010021283AD81D4B03EB45
:10A5C000C0035B68012919D0042925D0194A52F823
:10A5D0003020002082F8800219B94FF480721A608E
:10A5E0007047022903D140F203121A607047032911
:10A5F0000CBF4FF4817200221A6070470D4A52F866
:10A600003020012182F880124FF4A2721A601A6879
:10A6100022F020021A607047064A52F830200121C9
:10A6200082F880124FF4A2721A601A6842F0200277
:10A630001A607047240A010070B50D46212861D8C0
:10A64000042A5FD8DFE802F00709050B03000B239B
:10A6500006E00A2304E0082302E00C2300E00923BB
:10A660001E04294B03EBC0035C68236813F4E06FFE
:10A6700002D10021FFF7A0FF244B254AC3F89C21FB
:10A68000244AC3F8A021244AC3F8A421234AC3F8CA
:10A69000A821234AC3F8AC2104F14043A3F5922337
:10A6A0007C2B18D904F14042A2F594227C2A14D9BB
:10A6B00004F14043A3F596237C2B10D904F14043C9
:10A6C000A3F598237C2B0CD904F14043A3F59A23DE
:10A6D0007C2B08D970BD134906E0134904E01349E7
:10A6E00002E0134900E0134972B6236823F4702393
:10A6F0002360C4F3840241F8225043F080731E4368
:10A70000266062B670BD00BF240A01000092FF1FE0
:10A710001198FF1FE597FF1FB997FF1F8D97FF1F28
:10A720006197FF1FB0A5FF1FE8A5FF1F38A6FF1FF9
:10A7300068A6FF1F88A6FF1F72B60C4B1B680C4A49
:10A7400012680C49096862B611F0806F02D0322B92
:10A7500088BF0132C3F5BB33FF330749A1FB0303B5
:10A760009B094FF47A7000FB0230704718E000E05C
:10A7700050DBFF1F04ED00E0ABAAAAAA38B50546DE
:10A78000FFF7DAFF044625B938BD013D0AD004F5CC
:10A790007A74FFF7D1FF001BB0F57A7FF5D201F094
:10A7A00089FEF6E738BD00BF10B5264B4FF4000216
:10A7B0001A604FF080721A604FF000721A604FF00A
:10A7C00080621A604FF000621A6000201E4B186011
:10A7D0004BF6FF710433196028231C4A13600832BA
:10A7E00013600832136008321360083213600832B5
:10A7F000136008321360083213600922144C22607F
:10A8000004F580540434206004342160043423604F
:10A8100008342360143C226004F5FE2404342060D4
:10A820000C4801600C490B6008310B600B4B1A603F
:10A83000FFF78AFC4FF4C870FFF7A0FF01F008F89B
:10A8400010BD00BF08E100E0048003400C8003401D
:10A850000080034008800B400C800B4000800B40C0
:10A86000254B1A6842F480621A600023234A137051
:10A87000234A1370234A1370234A1370234A137018
:10A88000234B1B7813B1152B05D008E040F213328F
:10A89000204B1A6003E040F213321F4B1A601F4B2B
:10A8A0001B78012B02D0052B05D008E04FF4517224
:10A8B0001B4B1A6003E04FF451721A4B1A60C0F33D
:10A8C0004432194B1A70C0F347125A7000F01F003F
:10A8D000987204229A700221D9745A7588221A74C7
:10A8E0003C22DA704022114B1A704FF40052A3F24E
:10A8F00029331A60704700BF34800440E0DBFF1F3B
:10A9000059DBFF1FE8DBFF1FE1DBFF1F58DBFF1FE9
:10A910009CDBFF1F40A0044018C0044090A6FF1F0E
:10A9200044A004401CC0044000A006402DE400E008
:10A93000164B9B7803F0EC0300F00302134310F076
:10A94000040F18BF43F01003104A937000F00F0378
:10A95000042B04D11346927942F040029A710B4BBA
:10A960005A7902F0EF0210F0100F18BF42F01002F7
:10A97000064B5A719B7903F0EF0310F0200F18BFBC
:10A9800043F01003014A9371704700BF00A00640D6
:10A9900010B5144B1B6813F4806F21D0124B1B7839
:10A9A00013F0FF0F06D0104C01F084FD237813F054
:10A9B000FF0FF9D14FF400520C4B1A6000230C4AE0
:10A9C000D37040F203120B490A6004310A600A4A4C
:10A9D00013700A4A13700A4B1B680BB101221A70DC
:10A9E00010BD00BF3480044058DBFF1F84E100E04D
:10A9F00000A0064040A00440E0DBFF1F59DBFF1F22
:10AA000054DBFF1F10B50446094A137813F0FF0FFB
:10AA1000FBD120460121FFF7CFFD20460021FFF7A3
:10AA200099FD044B53F83420034B1A6010BD00BF4E
:10AA300058DBFF1F240A0100E4DBFF1F10B40C46A3
:10AA400009B140F08000184B1B78984228D0174A73
:10AA5000126812F4806F21D003F07F03012B02D023
:10AA6000052B04D006E00022114B1A6002E0002200
:10AA7000104B1A60002C0CBF4422602200F07F03B0
:10AA8000012B02D0052B05D008E042F44072084BA0
:10AA90001A6003E042F44072064B1A60024B1870D1
:10AAA0005DF8044B704700BF90A6FF1F3480044040
:10AAB00044A004401CC00440114B1B7898421ED097
:10AAC000104A126812F4806F17D013B1152B04D0FE
:10AAD00006E000220C4B1A6002E000220B4B1A60C9
:10AAE00010B1152805D008E040F21332064B1A6069
:10AAF00003E040F21332054B1A60014B18707047A7
:10AB00009CDBFF1F3480044040A0044018C0044078
:10AB100010B50D4B1B6813F4806F12D021280CD890
:10AB20000A4C0B4B53F8303023600121FFF744FDF2
:10AB3000236800221A70012010BD0020034B18600A
:10AB400010BD002010BD00BF3480044054DBFF1F47
:10AB5000240A0100114B1B6813F4806F1BD01228CC
:10AB600004D140F202320E4B1A600DE0142804D1D9
:10AB700040F202320B4B1A6006E00B4B5A7B02F09C
:10AB8000FE025A7300207047074B5A7B42F00102C5
:10AB90005A73012070470020704700BF3480044082
:10ABA0000CA0044014C0044000A006402DE9F04170
:10ABB00007461F4B1B6813F4806F37D01D4B1B6873
:10ABC0000BB101221A701C4B1C780134402C28BF99
:10ABD00000241A4D1A4EDFF86C8017E0FFF70CFCCA
:10ABE00040280FDC337913F0800F0FD02B7801331E
:10ABF000402B28BF002318F80320D2B2F271DBB239
:10AC00002B7003E0FF2801DD01F054FC2B78DBB250
:10AC10009C42E3D0FFB20B4B1F5501220A4B1A7026
:10AC2000E4B2054B1C70BC22054BDA70BDE8F08124
:10AC300034800440E4DBFF1FE8DBFF1FE1DBFF1F84
:10AC400000A006405CDBFF1F58DBFF1F2DE9F84F1B
:10AC50000746284B1B6813F4806F49D0264B1B68AE
:10AC60000BB101221A7007EB010B5F453DD2DFF8F3
:10AC70009890224EDFF88C80DFF890A099F8004081
:10AC80000134402C28BF00243578EDB2A54220D1F4
:10AC9000BC2388F80330FFF7AFFB402811DC98F89D
:10ACA000043013F0800F10D033780133402B28BFCD
:10ACB00000231AF80320D2B288F80720DBB23370E1
:10ACC00003E0FF2801DD01F0F5FB3378DBB29D42A4
:10ACD000E1D017F8013B0AF804300122084B1A7042
:10ACE000E4B289F800405F45C8D1BC22054BDA7058
:10ACF000BDE8F88F34800440E4DBFF1FE1DBFF1F79
:10AD000058DBFF1F00A00640E8DBFF1F5CDBFF1FD6
:10AD100010B5064B1B7813F0FF0F06D0034C01F063
:10AD2000C9FB237813F0FF0FF9D110BD58DBFF1FCB
:10AD3000064B1B78DBB2064A1278D2B293422CBF84
:10AD40003F3202F1FF32D01A704700BFE8DBFF1F2D
:10AD5000E1DBFF1F054B1878C0B2054B1B78DBB257
:10AD6000984238BF4030C01A704700BFE0DBFF1F79
:10AD700059DBFF1F10B4184B1A78D2B2174B1B784F
:10AD8000DBB29A4218D001333F2B18D81449C85C63
:10AD9000C0B2DCB211490C7012490968C9B19A42BB
:10ADA00003D300E00023D31A01E04032D31A1A2B58
:10ADB0000FDC00230B700CE04FF0FF3009E0084B74
:10ADC0001878C0B20021054B1970064B196800298C
:10ADD000E8D15DF8044B7047E0DBFF1F59DBFF1F34
:10ADE000A0DBFF1F54DBFF1F094B1A78D2B2094BBF
:10ADF0001B78DBB29A4207D00133402B28BF0023D7
:10AE0000054AD05CC0B270474FF0FF30704700BFBA
:10AE1000E0DBFF1F59DBFF1FA0DBFF1F0D4B1B6893
:10AE200013F4806F14D00C4BDA7802F0CB02DA7096
:10AE300040225A74DA7842F03402DA70074B1A78FA
:10AE4000D2B2074B1A70074B1B680BB100221A7065
:10AE5000704700BF3480044000A0064059DBFF1F4C
:10AE6000E0DBFF1F54DBFF1F70B43D4B1B7913F079
:10AE7000300F33D072B63A4B9B7D03F0FF022BB9F3
:10AE8000374BDA7940225A7462B627E062B6354B06
:10AE90001978C9B2344B1C78E4B2314D334EEB799A
:10AEA000D8B24B1C402B28BF0023A3421CBFF05438
:10AEB0001946531E13F0FF02F1D1CAB2294B1A7082
:10AEC0002B4B1B6853B1A1422EBFC4EB0101C4F14F
:10AED000400409192729C4BF01221A70204BDA78CF
:10AEE000D2B212F0800F27D01B7913F0800F23D03D
:10AEF000204B1C78E4B2204B1B78DBB29C4210D074
:10AF000017491E4D01E0A3420BD00133402B28BF4F
:10AF100000230879E85CC0B2C871087DC0B2072878
:10AF2000F1D9DBB214490B700D4B1B7913F0800F74
:10AF300002D07C210A4BD97012F0400F0ED0084B82
:10AF40001B7913F0400F09D000220D4B1A700D4BE6
:10AF50001B6803B11A703C22014BDA7070BC704759
:10AF600000A00640E0DBFF1F59DBFF1FA0DBFF1F37
:10AF700054DBFF1FE8DBFF1FE1DBFF1F5CDBFF1F74
:10AF800058DBFF1FE4DBFF1F30B40E4B1B7843F090
:10AF900002020D4C04EBC20460600C4800780028EB
:10AFA0000CBF8824C82444EA0141074D45F83210FB
:10AFB00080F00100054A107083F00103014A13700C
:10AFC00030BC704754DCFF1F0080FF1FCDDCFF1F2B
:10AFD00010B4431E032B11D872B60A4A52F823004C
:10AFE00050B14268074941F82320074A32F813401C
:10AFF0000188611A22F8131062B600E000205DF8A3
:10B00000044B704744DCFF1F84DEFF1F0138032818
:10B010000DD872B6074B53F820302BB10020013009
:10B020005B68002BFBD100E0002062B67047002077
:10B03000704700BF98DCFF1F38B572B601231B496B
:10B040001B4C5A1812F8012C12F0080F24D09A0049
:10B0500054F832506DB9164B03EBC201083048600A
:10B06000144943F83210144B1A78013A1A7062B638
:10B0700038BD42F0010254F832506DB90C4B03EB6D
:10B08000C201083048600D4943F832100A4B1A7863
:10B09000013A1A7062B638BD0133052BD1D162B6C0
:10B0A0000022054B1A7000F037FC38BD700B010010
:10B0B0000080FF1F88004000C2DCFF1FC800400066
:10B0C00010B4431E032B37D8400140F010001C4A37
:10B0D000104472B61B4AD25C032A09D8DFE802F09A
:10B0E00019021B050830022216E00830042213E082
:10B0F000154A52F823201AB9134A42F8231003E0E4
:10B10000124A52F823205160104A42F8231062B6C6
:10B1100012E0032200E005220A4CE25401F1080388
:10B12000436000F00803002B0CBF8823C8230A8863
:10B1300043EA0243036062B65DF8044B704700BF08
:10B140000080FF1F00DCFF1F98DCFF1FA8DCFF1F33
:10B150002DE9F84FA34CDFF8E092DFF8E0A2DFF82A
:10B16000E0B22578EDB215F0040F1DD09E4B1B7890
:10B1700013F0FF0F16D09D4B1B7803F0FF022BB18D
:10B18000531EDBB2994A137003B900BE984B1B786B
:10B1900003F0FF0233B1531EDBB2954A13700BB9B3
:10B1A00000F018FD0423237015F0080F00F0E4826E
:10B1B00099F80030DBB21D0940F021828D4D9E08C8
:10B1C00005EBC6035A6855F83630C3F38303013BD9
:10B1D0000C2B00F21082DFE813F0CB01CB010E0242
:10B1E0000E020E020E020E020E02E8010E020E0206
:10B1F0000E020D00804913680B6052684A607F4A56
:10B2000045F8362000227E490A607A490A618A613F
:10B2100001217C4A11709BB240F28162934218D89E
:10B22000B3F5D06F2ED2B3F5817F00F01E8106D822
:10B23000802B00F0C980822B00F0CC8066E140F2C8
:10B240000232934200F02681B3F5A06F00F06281D4
:10B250005CE142F22102934200F0868107D8B3F507
:10B26000086F00F0AB80B3F5106F11D04EE142F2E1
:10B270002122934200F0418142F22132934200F0B8
:10B28000498143E1604B5D68002D40F0188130E159
:10B29000594B9A78544B1A70564D05F180062B6A1B
:10B2A00013F0800F03D0686A083800F035FB0835CA
:10B2B000B542F4D1DFF88C8100263746534AB058A6
:10B2C00028B1456800F028FB0DB12846F9E70023B6
:10B2D0004E4973504E4AB3504E4BF05828B1456812
:10B2E00000F01AFB0DB12846F9E7002349497350D5
:10B2F000494AB35028F8023F484BFB5C023B032B02
:10B300000AD8DFE803F0020602060022434BDA55B2
:10B3100002E00122414BDA5501370436102ECDD11F
:10B3200000223F4B1A7001253E4EDFF81C81314F41
:10B3300005EB080313F8013C06F8043B13F0080F73
:10B340002DD000F0C9FA48B1A90007EB451200F171
:10B3500008035360344A47F8312007E0AB0000226D
:10B3600047F833202E4B1A7801321A7000F0B4FAE5
:10B3700058B1AB0043F0010307EBC30100F1080231
:10B380004A601E4A47F8332009E0AB0043F001034E
:10B39000002247F83320224B1A7801321A70AA0093
:10B3A00042F00201002347F8313042F0030247F82F
:10B3B000323001351D4B9E42BAD11EE20A4B1B783A
:10B3C0001B4D2B700127AAE0194D00232B706B70C9
:10B3D0000227A4E0084B9B88042B37D90F22154B7A
:10B3E0001A70C1E080200740CCDCFF1F55DCFF1F36
:10B3F000CEDCFF1F0080FF1FB8DCFF1FC80040002D
:10B40000ECDBFF1FCDDCFF1F740B010044DCFF1FD2
:10B41000F0DBFF1F98DCFF1FA8DCFF1F00DCFF1F15
:10B42000C2DCFF1FC420074088004000D420074032
:10B43000C4DCFF1FC0200740902007409420074035
:10B440009820074082DEFF1F700B0100A04A0021F8
:10B45000117051709F4A12F8233013F0020F5CD024
:10B460009B4D01232B70022759E09B4B9B8803F0D7
:10B470007F03042B02DC984A52881AB10F22954BA5
:10B480001A7071E0934A12F8231021F0020102F8B9
:10B490002310B2E1904B9B8803F07F03042B02DC66
:10B4A0008D4A52881AB10F228A4B1A705CE0894A81
:10B4B00012F8231041F0020102F823109DE1864B9F
:10B4C0005E889F88854BA3F10C02114633F80C0C63
:10B4D000B04209D133F80A0CB84205D1360A032E1E
:10B4E0000CBF2F7817891AE00D690C330C32002D30
:10B4F000EBD10F22774B1A7036E0794B1A68794BF3
:10B500001A60754B9A78784B1A7076E10F22714B5E
:10B510001A7029E000273D4601E002276C4D6E4B72
:10B52000DB889F4228BF1F46402F34BF3E4640263F
:10B5300028463146FFF728FD3544BF1B03D13F2E77
:10B5400000F2608110E0402F34BF3E46402628467E
:10B550003146FFF719FD3544BF1B01D13F2E03D9FA
:10B56000624B1D60624B1F8001238AF8003042E06D
:10B57000594B198842F22103994212D15D4BD81DD3
:10B5800012F8011B03F8011F8342F9D15A4B1B68C3
:10B59000862B02D10F22594B1A7000200146FFF76B
:10B5A000F3FC574B45F8363025E0504B1E68BEB1D2
:10B5B0004F4FB7F80080B8F1400F34BF45464025E3
:10B5C00030462946FFF7E0FCC5EB08039BB23B8001
:10B5D0000BB9402D01D1354400E00025434B1D60DF
:10B5E0003D4B1B88B3F5A06F05D13B4B00225A7031
:10B5F0009B788BF8003001238AF80030B9E0414E87
:10B600009F0806EBC708D8F80420A2F10800013D06
:10B61000EDB213F0080F47D000F07EF93A4B53F823
:10B6200025304BB35A68384941F8252003F1080208
:10B63000C8F80420354A525D032A12D8DFE802F028
:10B6400002060A0E0321314A51550AE002212F4A0F
:10B65000515506E005212D4A515502E004212B4A9F
:10B66000515518F0080F0CBF8822C8221B8842EAE7
:10B67000034346F837307CE0244B5B5D032B0BD84B
:10B68000DFE803F0777702060022204B5A5570E07E
:10B6900001221E4B5A556CE018F0080F0CBF022215
:10B6A00003221A4B5A5564E056F837301B0C22F827
:10B6B000083C002B55D0002322F8063C42F8043CFD
:10B6C000134B53F825302BBB114B43F8250025E0D5
:10B6D000C4DCFF1FC0200740B8DCFF1F800B010047
:10B6E00050DBFF1F94DEFF1FDCDCFF1FECDBFF1FC6
:10B6F000C0DCFF1F8BDEFF1F8CDEFF1F55DCFF1F32
:10B70000C80040000080FF1F98DCFF1F00DCFF1F07
:10B7100044DCFF1F3F4B53F8253058603D4B43F846
:10B7200025003D4B33F8151032F8082C0A4423F855
:10B73000152000F0D1F860B100F10803C8F804301A
:10B7400018F0080F354B364A08BF134646F8373015
:10B750000FE0002346F83730324B1A7801321A7066
:10B7600007E018F0080F2D4B2D4A08BF134646F886
:10B77000373008232370F4E415F0010F22D02A4952
:10B7800002230B700022294B1A70294B24481860A1
:10B79000284C5C6098602848D8601A619A610D2036
:10B7A000264B1870FF2326480370083803701830A2
:10B7B0000270244A13709F22234B1A7001230B70CE
:10B7C000BDE8F88F15F0800F05D00D221B4B1A70C5
:10B7D0008022403B1A7015F0020F06D0184B1A78E1
:10B7E000D2B21A700222083B1A7015F0100F0ED058
:10B7F0001022164B1A70BDE8F88F00200146FFF7A3
:10B80000C3FBB1E628460021FFF7BEFBACE6BDE86E
:10B81000F88F00BFF0DBFF1F84DEFF1FC800400071
:10B8200088004000C2DCFF1F9420074054DCFF1F4B
:10B830000080FF1F04DCFF1F58DCFF1FC0200740F3
:10B84000882007408C200740842007408020074044
:10B8500008B501F0A5FC00231B491A465A50C81828
:10B8600042600833882BF9D1184B1A6842F48022C1
:10B870001A60154BC3F30721154A1170C3F3074132
:10B88000143211701B0E04321370FF23343A1370FC
:10B8900008321370783A1370012384321370002138
:10B8A0006C3211707C3A137070220A4B1A704FF48C
:10B8B0000072A3F241331A60102203F1C04303F572
:10B8C000C8231A7008BD00BF0080FF1F34800440E9
:10B8D0009C20074049E400E072B60D4B1A68B2FAAA
:10B8E00082F30B2B02D962B6002070474FF0004163
:10B8F000D94022EA010206490A6062B6054903EB13
:10B90000C303DB00C8180022CA504260704700BF62
:10B9100094A6FF1F0094FF1F08B50F4BC31A0F4AD0
:10B92000A2FB03131B090B2B14D80D4A12783AB152
:10B930000C4A127812F0FF0F02D0FFF77DFB08BD12
:10B9400072B6094A4FF0004121FA03F31168194316
:10B95000116062B608BD00BF0094FF1F398EE33846
:10B96000C2DCFF1FCCDCFF1F94A6FF1F10B5134BDA
:10B970001B6853B9124B1B7813F0FF0F18D003202C
:10B98000FFF726FB0D4B1860A8B10C4B18684388D5
:10B990005A1C03441C7A03889A4206D3FFF7BCFF63
:10B9A0000022064B1A60204610BD4280204610BD82
:10B9B0004FF0FF3010BD4FF0FF3010BDD8DCFF1F3F
:10B9C000CCDCFF1F08B50D4B1B6883B90C4B1B78F3
:10B9D00013F0FF0F08D00320FFF7FAFA074B1860A7
:10B9E00028B94FF0FF3008BD4FF0FF3008BD034BC2
:10B9F0001B685A881344187A08BD00BFD8DCFF1FA3
:10BA0000CCDCFF1F044B9888044B1B681BB11A88C1
:10BA10005B88D31A1844704784DEFF1FD8DCFF1FF1
:10BA200010B50B4B1B7813F0FF0F0FD0094B1868A4
:10BA300020B1FFF771FF0022064B1A600324204655
:10BA4000FFF7C6FA10B1FFF767FFF8E710BD00BFB8
:10BA5000CCDCFF1FD8DCFF1F2DE9F84F0446012284
:10BA6000384B1A708B46002965D00E46DFF8E0800F
:10BA7000DFF8E0909A46344FD8F8003083BB99F84D
:10BA8000003013F0FF0F06D100222E4B1A704FF03A
:10BA9000FF30BDE8F88F4AF2F9250420FFF7B6FA27
:10BAA00007280AD801238AF80030FFF715FFC8F8E5
:10BAB0000000A8B900238AF80030013D01D03B788E
:10BAC00033B10122204B1A704FF0FF30BDE8F88FE0
:10BAD00000F0F0FC99F8003013F0FF0FDDD1D3E750
:10BAE00000233B70D8F800104A88C2F14005AE42EE
:10BAF00038BF354602F108030B442A444A80761BBE
:10BB00003DB1254414F8012B03F8012BAC42F9D1C7
:10BB100000E025464B883F2B07D940230B800420AB
:10BB2000FFF7CEFA0023C8F800300522074B1A7041
:10BB30000EB12C46A0E70022024B1A705846BDE811
:10BB4000F88F00BFCFDCFF1FD4DCFF1FCEDCFF1F50
:10BB5000D0DCFF1FCCDCFF1F00B583B002AB03F8C5
:10BB6000010D18460121FFF777FF03B05DF804FBD4
:10BB700010B5144B1B7813F0FF0F21D00122124B8C
:10BB80001A70124B196851B10024114B1C704B886C
:10BB90000B800420FFF794FA0C4B1C600DE0FFF7BC
:10BBA0009BFE014630B10022094B1A700420FFF7BA
:10BBB00087FA02E00122064B1A700022024B1A702B
:10BBC00010BD00BFCCDCFF1FCFDCFF1FD0DCFF1F90
:10BBD000CEDCFF1F08B50E4B1B7813F0FF0F16D1FC
:10BBE0000C4B196841B14B880B800420FFF768FAB1
:10BBF0000022084B1A6008BDFFF76EFE014618B11F
:10BC00000420FFF75DFA08BD0122034B1A7008BD3E
:10BC1000CFDCFF1FD0DCFF1FCEDCFF1FF0B4C0293C
:10BC200028BFC02172B6134B1860134B00221A6054
:10BC30005A609A60DA601A615A61C1B113460E4CBB
:10BC400001275A0903F01F0607FA06F654F8225096
:10BC5000354344F8225001338B42F2D1002213467F
:10BC600084186370013302F582728B42F8D162B698
:10BC7000F0BC7047E8DCFF1FF0DCFF1F10B472B6A9
:10BC8000234B1B688BB9224B5B6883B9204B9B68A5
:10BC90007BB91F4BDB6873B91D4B1B696BB91C4B20
:10BCA0005B6963B962B600202EE0194A08E0194AC0
:10BCB00006E0194A04E0194A02E0194A00E0194A6C
:10BCC000B3FA83F14FF00040C84023EA0003136049
:10BCD000154803780133DBB2037062B60C48121AC0
:10BCE0009210C1EB421202EB821241F67C7101EB21
:10BCF00082020E490968881801248C540C4A127873
:10BD00009A423CBF0A4A13705DF8044B704700BF6B
:10BD1000F0DCFF1FF4DCFF1FF8DCFF1FFCDCFF1F63
:10BD200000DDFF1F04DDFF1FEDDCFF1FE8DCFF1F50
:10BD3000E4DCFF1F427872B60378012B02D9013B85
:10BD4000037011E05111094BD24302F01F024FF072
:10BD5000004020FA02F253F82100104343F821007A
:10BD6000034B1A78013A1A7062B67047F0DCFF1F75
:10BD7000EDDCFF1F30B4C36883B1187A90420AD15A
:10BD800058685C7A006950F8245025B940F82410AE
:10BD9000087801300870DB68002BEED130BC7047AA
:10BDA000437A8B4206D9036953F82100002243F8F5
:10BDB000212070470020704738B5437A8B4218D94C
:10BDC000036953F82140002243F821209CB12378D5
:10BDD000012B12D9FFF752FF054628B10430211D6F
:10BDE0004FF48072FEF792F82378013B23702846C7
:10BDF00038BD002038BD204638BD204638BD00BFC4
:10BE00004368427A5B7A9A4210D872B60368DA685D
:10BE10000AB9D86004E0D3680BB11A46FBE7D060DA
:10BE20000268012313724268137262B6704700BF42
:10BE3000084B1B785BB9D022074B1A704FF0804239
:10BE4000A3F256331A600120024B1870704700208D
:10BE5000704700BFECDCFF1F5EE400E0F8B5184B54
:10BE60001A6842F080721A60164B1A6842F001029A
:10BE70001A6004331F68144B1C689CB1134D237A5D
:10BE80006BB12E6823681B68204698472B689B1B64
:10BE90001B099AB2A280E1888B4288BFE280646964
:10BEA000002CECD1094B1B68DF1B3F09BBB2084AD1
:10BEB0001380084A1288974284BF064A1380F8BD4F
:10BEC000FCED00E0001000E0E0DCFF1F041000E0EB
:10BED00008DDFF1FEEDCFF1F30B472B699B90268AF
:10BEE0008AB103790F2B0ED827490988194111F01F
:10BEF000010F08D003F1007303F59063B2EB431F09
:10BF000001D162B63EE0204B1D882946002341FA4C
:10BF100003F212F0010F2DD1012202FA03F425439E
:10BF2000194A158062B6DAB2027118490C6844F0F9
:10BF300002040C6004390C6844F002040C60822492
:10BF400013490C601A310A7004310A7006390A70FC
:10BF500007310A7003F1007303F590635B0103601E
:10BF600000221A605A609A60DA601A615A619A6116
:10BF7000DA6107E00133102BC9D162B600230360F8
:10BF80001023037130BC70470ADDFF1F408004405E
:10BF90000080004003790F2B10D8094A137072B645
:10BFA000084B0279012101FA02F2198821EA020202
:10BFB0001A8062B61023037100230360704700BF2C
:10BFC0001A8000400ADDFF1F2DE9F0438BB00746C1
:10BFD00088468C68C4B100252E464FF021094046A2
:10BFE00001A94A462B4600F015FA202C34BF224600
:10BFF00020221544A41A3B685B68384601A998477B
:10C000000644002CEBD100E0002630460BB0BDE822
:10C01000F08300BF00B583B0054B1B88ADF804303A
:10C0200003685B6801A90222984703B05DF804FB2E
:10C03000340B0100F0B58BB0164622B903681B68BB
:10C04000C9B298472FE0012A08BF0A2621B9302239
:10C050008DF82520212417E021243746B1FBF6F581
:10C0600006FB1515EDB22246092D94BF3035373544
:10C07000EDB20DF1280E724402F8245CB1FBF7F129
:10C0800011B1013CE4B2E9E733B1013CE4B20AABDF
:10C0900023442D2203F8242C03685B6801A9214462
:10C0A000C4F1220298470BB0F0BD00BF08B50029CB
:10C0B000BABF49422D2300230A22FFF7BBFF08BD68
:10C0C0002DE9F04F85B0804614461D469DF8389006
:10C0D0001046194601F08EFA40B9D8F800305B6876
:10C0E00040466749032298470746BEE02046294656
:10C0F00001F080FA012808D1D8F800305B6840468A
:10C100006049032298470746AFE0204629464FF092
:10C1100060425D4B01F0DEFE40B1D8F800305B6854
:10C1200040465A490322984707469EE02046294642
:10C130004FF06042564B01F0AFFE40B1D8F80030EE
:10C140005B68404651490322984707468DE02046E8
:10C1500029460022002301F09FFE28B105F100438B
:10C160001D464FF0010A01E04FF0000AB9F1000F3F
:10C170006CD04FF0000B0022464B3FA7D7E9006779
:10C180001046194632463B4601F014FC02460B4667
:10C190000BF1010B5FFA8BF18945F1D82CE04E468B
:10C1A0002046294600223C4B01F004FC04460D4683
:10C1B00001F09AFEC0B206F101095FFA89F904ABF9
:10C1C0001E4400F1300306F8103C01F08DFB0246DE
:10C1D0000B462046294601F039FA04460D46D14562
:10C1E000DDD101E04FF0010AD8F800305B6840462D
:10C1F00069465246984738E02046294601F028FA19
:10C2000004460D4601F070FE064601F05DFB024655
:10C210000B462046294601F019FA04460D464046D1
:10C2200031460A225346FFF705FF07462E238DF8B5
:10C230000030B9F10F0F34BF4B460F23002BD1D084
:10C2400003F1010A5FFA8AFA0126A9E72046294686
:10C250000022104B01F0FCF901F046FE0146404679
:10C260000A225346FFF7E6FE0746384605B0BDE80A
:10C27000F08F00BFAFF30080000000A09999B93F94
:10C28000380B01003C0B0100FFFFEF41400B0100A8
:10C29000FFFFEFC10000E03F00002440AFF300804B
:10C2A00008B1014A106070470CDDFF1F10B4124B3B
:10C2B0001968D9B1114C81FB0423CA18CB17C3EB01
:10C2C00022420F4800FB121284FB01042144C3EBFD
:10C2D00021430C4800FB03F344F2A71000FB02309B
:10C2E000002804DA00F10040013800E00648024B63
:10C2F00018605DF8044B70470CDDFF1F5F0B4E8329
:10C300001DF30100ECF4FFFF42CE0C1F10B50446F4
:10C3100030B1FFF7CBFFB0FBF4F303FB140010BD0B
:10C32000002010BD10B50446884204DA081AFFF751
:10C33000EDFF204410BD10BD10B4401A019CE41A5A
:10C3400004FB00F4521A94FBF2F018445DF8044B1D
:10C35000704700BF10B50446006802F051F920464E
:10C3600010BD00BF38B504460D460068013102F02B
:10C37000CDFC18B120606560012038BD002038BDBB
:10C3800010B5044643688B420AD2FFF7EBFF034621
:10C3900048B1A36833B9236800221A70012302E070
:10C3A000012300E00123184610BD00BF70B504460C
:10C3B0000E4615462AB9036803B11A700023A3601C
:10C3C00012E01146FFF7DCFF48B9206818B102F00F
:10C3D00017F90023236000236360A36004E0A560D5
:10C3E0002068314603F03CF8204670BD38B504465D
:10C3F000002303604360836003730D4639B1084630
:10C4000003F08CF8024620462946FFF7CFFF20466E
:10C4100038BD00BF38B50C469AB191B181689942D8
:10C4200002D80023237038BD551EC91A8D4228BF7B
:10C430000D460168204619442A4603F09FF8002360
:10C44000635538BD08B5F9F72FFDF9F783FB00F008
:10C4500031F8FAE708B5FFF7D5FA08BD08B5FFF7D8
:10C4600085FA08BD08B5FFF7ADFA08BD08B5FFF7B6
:10C470007FFB08BD08B5FFF7D3FA08BD08B508462D
:10C48000FFF76AFB08BD00BF08B508461146FFF775
:10C49000E3FA08BD704700BF044B00221A714FF445
:10C4A0007A7199601A73024A1A60704714DDFF1F8F
:10C4B000500B010008B50F4B1B78CBB901220D4B77
:10C4C0001A70FFF79FFA08B1FFF7E4FFFEF742FC8E
:10C4D00008B100F03BFF00F0A7FA08B100F0D8FF68
:10C4E00000F074FD08B101F075F80022014B1A70DC
:10C4F00008BD00BF24DDFF1F254B1A6842F400620F
:10C500001A600023234A1370234A1370234A1370BE
:10C51000234A1370234A1370234B1B78092B02D034
:10C520001A2B05D008E040F21332204B1A6003E0CA
:10C5300040F213321E4B1A601E4B1B780A2B02D09E
:10C540001F2B05D008E04FF451721B4B1A6003E01B
:10C550004FF45172194B1A60C0F34432184B1A70E1
:10C56000C0F347125A7000F01F00987204229A70AC
:10C570000221D9745A7588221A743C22DA7040223A
:10C58000104B1A704FF40042A3F22B331A6070471D
:10C590003480044098DDFF1F2DDDFF1FA0DDFF1F4D
:10C5A00099DDFF1F2CDDFF1F98A6FF1F0CB0044074
:10C5B00004D0044099A6FF1F10B0044000D00440EE
:10C5C00000B006402FE400E0164B9B7803F0EC032C
:10C5D00000F00302134310F0040F18BF43F01003E0
:10C5E000104A937000F00F03042B04D11346927984
:10C5F00042F040029A710B4B5A7902F0EF0210F0B0
:10C60000100F18BF42F01002064B5A719B7903F0CD
:10C61000EF0310F0200F18BF43F01003014A93718D
:10C62000704700BF00B0064010B5224B1B6813F4E2
:10C63000006F3ED0204B1B7813F0FF0F06D01E4C2E
:10C64000FFF738FF237813F0FF0FF9D14FF40042C2
:10C650001A4B1A6000221A4BDA701A4B1B78092BFE
:10C6600002D01A2B05D008E040F20312164B1A60D4
:10C6700003E040F20312154B1A60154B1B7803F0D0
:10C680007F030A2B02D01F2B05D008E040F20312D3
:10C69000104B1A6003E040F203120F4B1A600023A4
:10C6A0000E4A13700E4A13700E4B1B680BB1012219
:10C6B0001A7010BD348004402CDDFF1F84E100E0BF
:10C6C00000B0064098A6FF1F0CB0044004D0044000
:10C6D00099A6FF1F10B0044000D0044098DDFF1F52
:10C6E0002DDDFF1F28DDFF1F10B50446094A137812
:10C6F00013F0FF0FFBD120460121FDF75DFF20461F
:10C700000021FDF727FF044B53F83420034B1A6038
:10C7100010BD00BF2CDDFF1F240A01009CDDFF1FA0
:10C7200010B40C4609B140F08000184B1B789842B9
:10C7300028D0174A126812F4006F21D003F07F034B
:10C740000A2B02D01F2B04D006E00022114B1A60E6
:10C7500002E00022104B1A60002C0CBF4422602221
:10C7600000F07F030A2B02D01F2B05D008E042F413
:10C770004072084B1A6003E042F44072064B1A60A4
:10C78000024B18705DF8044B704700BF99A6FF1F5D
:10C790003480044010B0044000D00440124B1B7899
:10C7A000984220D0114A126812F4006F19D0092B58
:10C7B00002D01A2B04D006E000220D4B1A6002E0D2
:10C7C00000220C4B1A60092802D01A2805D008E074
:10C7D00040F21332064B1A6003E040F21332054B6D
:10C7E0001A60014B1870704798A6FF1F34800440F0
:10C7F0000CB0044004D0044010B50D4B1B6813F47A
:10C80000006F12D021280CD80A4C0B4B53F8303053
:10C8100023600121FDF7D0FE236800221A70012059
:10C8200010BD0020034B186010BD002010BD00BFDC
:10C830003480044028DDFF1F240A01000D4B1B68D3
:10C8400013F4006F13D017280AD140F202320A4BBA
:10C850001A600A4B5A7B42F001025A73012070475A
:10C86000064B5A7B02F0FE025A73002070470020EC
:10C87000704700BF3480044008B0044000B0064058
:10C880002DE9F04107461F4B1B6813F4006F37D0AA
:10C890001D4B1B680BB101221A701C4B1C78013414
:10C8A000282C28BF00241A4D1A4EDFF86C8017E0A0
:10C8B000FDF7A2FD40280FDC337913F0800F0FD075
:10C8C0002B780133282B28BF002318F80320D2B27D
:10C8D000F271DBB22B7003E0FF2801DDFFF7EAFD08
:10C8E0002B78DBB29C42E3D0FFB20B4B1F550122E9
:10C8F0000A4B1A70E4B2054B1C70BC22054BDA706F
:10C90000BDE8F081348004409CDDFF1FA0DDFF1FE7
:10C9100099DDFF1F00B0064030DDFF1F2CDDFF1F3B
:10C920002DE9F84F0746284B1B6813F4006F49D0D8
:10C93000264B1B680BB101221A7007EB010B5F45F8
:10C940003DD2DFF89890224EDFF88C80DFF890A07F
:10C9500099F800400134282C28BF00243578EDB226
:10C96000A54220D1BC2388F80330FDF745FD4028BF
:10C9700011DC98F8043013F0800F10D033780133B5
:10C98000282B28BF00231AF80320D2B288F80720EA
:10C99000DBB2337003E0FF2801DDFFF78BFD337856
:10C9A000DBB29D42E1D017F8013B0AF804300122C6
:10C9B000084B1A70E4B289F800405F45C8D1BC2228
:10C9C000054BDA70BDE8F88F348004409CDDFF1F12
:10C9D00099DDFF1F2CDDFF1F00B00640A0DDFF1F0B
:10C9E00030DDFF1F10B5064B1B7813F0FF0F06D08C
:10C9F000034CFFF75FFD237813F0FF0FF9D110BD53
:10CA00002CDDFF1F064B1B78DBB2064A1278D2B230
:10CA100093422CBF273202F1FF32D01A704700BF79
:10CA2000A0DDFF1F99DDFF1F054B1878C0B2054B35
:10CA30001B78DBB2984238BF4030C01A704700BF45
:10CA400098DDFF1F2DDDFF1F10B4184B1A78D2B2EE
:10CA5000174B1B78DBB29A4218D001333F2B18D802
:10CA60001449C85CC0B2DCB211490C7012490968A3
:10CA7000C9B19A4203D300E00023D31A01E0403247
:10CA8000D31A1A2B0FDC00230B700CE04FF0FF3091
:10CA900009E0084B1878C0B20021054B1970064B0D
:10CAA00019680029E8D15DF8044B704798DDFF1F35
:10CAB0002DDDFF1F58DDFF1F28DDFF1F094B1A78F2
:10CAC000D2B2094B1B78DBB29A4207D00133402B1C
:10CAD00028BF0023054AD05CC0B270474FF0FF303A
:10CAE000704700BF98DDFF1F2DDDFF1F58DDFF1FC2
:10CAF0000D4B1B6813F4006F14D00C4BDA7802F066
:10CB0000CB02DA7040225A74DA7842F03402DA70DA
:10CB1000074B1A78D2B2074B1A70074B1B680BB140
:10CB200000221A70704700BF3480044000B00640F5
:10CB30002DDDFF1F98DDFF1F28DDFF1F70B43D4B6B
:10CB40001B7913F0300F33D072B63A4B9B7D03F054
:10CB5000FF022BB9374BDA7940225A7462B627E0CC
:10CB600062B6354B1978C9B2344B1C78E4B2314DFA
:10CB7000334EEB79D8B24B1C402B28BF0023A34285
:10CB80001CBFF0541946531E13F0FF02F1D1CAB274
:10CB9000294B1A702B4B1B6853B1A1422EBFC4EB1B
:10CBA0000101C4F1400409192729C4BF01221A70E8
:10CBB000204BDA78D2B212F0800F27D01B7913F015
:10CBC000800F23D0204B1C78E4B2204B1B78DBB2C3
:10CBD0009C4210D017491E4D01E0A3420BD00133F7
:10CBE000282B28BF00230879E85CC0B2C871087DF3
:10CBF000C0B20728F1D9DBB214490B700D4B1B7979
:10CC000013F0800F02D07C210A4BD97012F0400F34
:10CC10000ED0084B1B7913F0400F09D000220D4BAA
:10CC20001A700D4B1B6803B11A703C22014BDA706D
:10CC300070BC704700B0064098DDFF1F2DDDFF1F60
:10CC400058DDFF1F28DDFF1FA0DDFF1F99DDFF1F3F
:10CC500030DDFF1F2CDDFF1F9CDDFF1F174B1A6807
:10CC600042F480521A600023154A1370154A13705B
:10CC7000154A1370154A1370154A137040F2133198
:10CC8000144A11604FF4517104321160C0F3443101
:10CC9000114A1170C0F34711517000F01F009072DB
:10CCA000937013742C23D37040220C4B1A704FF4E2
:10CCB0000032A3F22D331A60704700BF3480044065
:10CCC00014DEFF1FA9DDFF1F1CDEFF1F15DEFF1F87
:10CCD000A8DDFF1F08C0044000C0064031E400E0AA
:10CCE000164B9B7803F0EC0300F00302134310F0A3
:10CCF000040F18BF43F01003104A937000F00F03A5
:10CD0000042B04D11346927942F040029A710B4BE6
:10CD10005A7902F0EF0210F0100F18BF42F0100223
:10CD2000064B5A719B7903F0EF0310F0200F18BFE8
:10CD300043F01003014A9371704700BF00C00640E2
:10CD400010B5144B1B6813F4805F21D0124B1B7875
:10CD500013F0FF0F06D0104CFFF7ACFB237813F055
:10CD6000FF0FF9D14FF400320C4B1A6000230C4A2C
:10CD7000D37040F203120B490A6004310A600A4A78
:10CD800013700A4A13700A4B1B680BB101221A7008
:10CD900010BD00BF34800440A8DDFF1F84E100E027
:10CDA00000C0064008C0044014DEFF1FA9DDFF1FBD
:10CDB000A4DDFF1F10B50446094A137813F0FF0FD6
:10CDC000FBD120460121FDF7F7FB20460021FDF7AE
:10CDD000C1FB044B53F83420034B1A6010BD00BF55
:10CDE000A8DDFF1F240A010018DEFF1F10B40C4647
:10CDF00009B140F08000104B1B78984219D00F4ABF
:10CE0000126812F4805F12D003F07F03082B02D166
:10CE100000220B4B1A60002C0CBF4422602200F051
:10CE20007F03082B03D142F44072054B1A60024B7A
:10CE300018705DF8044B70479AA6FF1F34800440B9
:10CE40000CC00440704700BF10B50D4B1B6813F4B5
:10CE5000805F12D021280CD80A4C0B4B53F830308D
:10CE600023600121FDF7A8FB236800221A7001202E
:10CE700010BD0020034B186010BD002010BD00BF86
:10CE800034800440A4DDFF1F240A01000D4B1B6801
:10CE900013F4805F13D00E280AD140F202320A4BFD
:10CEA0001A600A4B5A7B42F001025A730120704704
:10CEB000064B5A7B02F0FE025A7300207047002096
:10CEC000704700BF3480044004C0044000C00640E6
:10CED0002DE9F04107461F4B1B6813F4805F37D0E4
:10CEE0001D4B1B680BB101221A701C4B1C780134BE
:10CEF000282C28BF00241A4D1A4EDFF86C8017E04A
:10CF0000FDF77AFA40280FDC337913F0800F0FD049
:10CF10002B780133282B28BF002318F80320D2B226
:10CF2000F271DBB22B7003E0FF2801DDFFF7C2FADC
:10CF30002B78DBB29C42E3D0FFB20B4B1F55012292
:10CF40000A4B1A70E4B2054B1C70AC22054BDA7028
:10CF5000BDE8F0813480044018DEFF1F1CDEFF1F97
:10CF600015DEFF1F00C00640ACDDFF1FA8DDFF1F60
:10CF700038B505460C4629B115F8010BFFF7A8FF97
:10CF8000013CF9D138BD00BF10B5064B1B7813F03A
:10CF9000FF0F06D0034CFFF78DFA237813F0FF0F35
:10CFA000F9D110BDA8DDFF1F064B1B78DBB2064A86
:10CFB0001278D2B293422CBF273202F1FF32D01A3C
:10CFC000704700BF1CDEFF1F15DEFF1F054B1878E2
:10CFD000C0B2054B1B78DBB2984238BF4030C01A54
:10CFE000704700BF14DEFF1FA9DDFF1F10B4184BF0
:10CFF0001A78D2B2174B1B78DBB29A4218D00133A1
:10D000003F2B18D81449C85CC0B2DCB211490C706F
:10D0100012490968C9B19A4203D300E00023D31A28
:10D0200001E04032D31A1A2B0FDC00230B700CE006
:10D030004FF0FF3009E0084B1878C0B20021054BD3
:10D040001970064B19680029E8D15DF8044B704748
:10D0500014DEFF1FA9DDFF1FD4DDFF1FA4DDFF1FAE
:10D06000094B1A78D2B2094B1B78DBB29A4207D02F
:10D070000133402B28BF0023054AD05CC0B2704763
:10D080004FF0FF30704700BF14DEFF1FA9DDFF1F08
:10D09000D4DDFF1F054B1A78D2B2054B1A70054B31
:10D0A0001B680BB100221A70704700BFA9DDFF1F7B
:10D0B00014DEFF1FA4DDFF1F2F4B1B7913F0200F81
:10D0C00023D02D4BDB79D9B22C4B1B780133402B6D
:10D0D00028BF00232A4A1278D2B29A4204D0294AA1
:10D0E000D154D9B2254A1170274A116869B1274A2B
:10D0F0001278D2B293422EBFC2EB0303C2F14002B8
:10D100009B18272BC4BF01230B701B4BDB78DBB2B2
:10D1100013F0800F1CD0184A127912F0800F17D02C
:10D120001B4A1178C9B2194A1278D2B2914203D17E
:10D130006C21114AD1700BE00132282A28BF00224D
:10D140001449885CC0B20C49C871D2B20F490A7048
:10D1500013F0400F0ED0084B1B7913F0400F09D08D
:10D1600000220D4B1A700D4B1B6803B11A702C2254
:10D17000014BDA70704700BF00C0064014DEFF1F8D
:10D18000A9DDFF1FD4DDFF1FA4DDFF1F15DEFF1F7C
:10D190001CDEFF1FACDDFF1FA8DDFF1F18DEFF1F19
:10D1A00000B585B072B61B4B70221A7041211A4A25
:10D1B00011700F21013A117080221A701A461378EB
:10D1C00013F0800FFBD0154B186862B6144B9842D1
:10D1D0009CBF00EB8000400001A90A22FDF72CF95A
:10D1E0009DF804307BB908E001A9595C31B1918008
:10D1F000023201330A2BF7D100E0002301335B0038
:10D20000084A137003E0074A53800123ECE705B096
:10D210005DF804FB000002400700024008000240E5
:10D220007F96980028A7FF1F08B503681B68C9B23E
:10D23000984708BD08B503681B68C9B2984708BD80
:10D2400008B503681B68C9B2984708BD08B50368EC
:10D250001B68C9B2984708BD08B54B0803F1376091
:10D2600000F5D830B0FBF1F0FDF7FAFA08BD00BFC9
:10D2700010B514464B0803F1376000F5D830B0FB09
:10D28000F1F0FDF7EDFA2046FDF752FB10BD00BFAF
:10D2900008B5FDF77DFB08BD08B50846FDF7B2FBF4
:10D2A00008BD00BF08B50846FDF706FC08BD00BF75
:10D2B00008B508461146FDF7C1FB08BD08B508468C
:10D2C000FDF726FC003018BF012008BD08B5084650
:10D2D000FDF740FC003018BF012008BD08B5FDF780
:10D2E00039FD08BD08B5FDF77FFD08BD08B5FDF7A0
:10D2F00041FD08BD08B5FDF70BFD08BD08B5FDF7FC
:10D300008DFD08BD08B5FDF713FD08BD08B508463D
:10D31000FDF74CFC012008BD08B50846FDF746FCAA
:10D32000012008BD10B5144608461146FDF78EFCD5
:10D33000204610BD38B50D46084602F0EFF8044609
:10D3400028462146FDF782FC204638BD704700BFC5
:10D35000044B00221A714FF47A7199601A73024AD1
:10D360001A60704720DEFF1FD00B010008B503686C
:10D370001B68C9B2984708BD08B503681B68C9B2E5
:10D38000984708BD08B503681B68C9B2984708BD2F
:10D3900008B503681B68C9B2984708BD08B54B08B3
:10D3A00003F1376000F5D830B0FBF1F0FFF7A4F8D7
:10D3B00008BD00BF10B514464B0803F1376000F5F7
:10D3C000D830B0FBF1F0FFF797F82046FFF7FCF8F4
:10D3D00010BD00BF08B5FFF727F908BD08B508461E
:10D3E000FFF782F908BD00BF08B50846FFF7D6F978
:10D3F00008BD00BF08B508461146FFF791F908BD02
:10D4000008B50846FFF7F8F9003018BF012008BD3D
:10D4100008B50846FFF712FA003018BF012008BD12
:10D4200008B5FFF701FB08BD08B5FFF747FB08BDCE
:10D4300008B5FFF709FB08BD08B5FFF7D3FA08BD2B
:10D4400008B5FFF755FB08BD08B5FFF7DBFA08BDC7
:10D4500008B50846FFF714FA012008BD08B50846CC
:10D46000FFF70EFA012008BD10B514460846114614
:10D47000FFF756FA204610BD38B50D46084602F0B3
:10D480004DF8044628462146FFF74AFA204638BDA3
:10D49000704700BF044B00221A714FF47A719960F3
:10D4A0001A73024A1A60704730DEFF1F300C010009
:10D4B00008B503681B68C9B2984708BD08B503687A
:10D4C0001B68C9B2984708BD08B503681B68C9B294
:10D4D000984708BD08B503681B68C9B2984708BDDE
:10D4E00008B54B0803F1B76000F55840B0FBF1F008
:10D4F000FFF7B4FB08BD00BF10B514464B0803F19D
:10D50000B76000F55840B0FBF1F0FFF7A7FB2046ED
:10D51000FFF7E6FB10BD00BF08B5FFF711FC08BD23
:10D5200008B50846FFF746FC08BD00BF08B5084629
:10D53000FFF788FC08BD00BF08B508461146FFF795
:10D5400055FC08BD08B50846FFF77EFC003018BF43
:10D55000012008BD08B50846FFF798FC003018BF49
:10D56000012008BD08B5FFF731FD08BD08B5FFF77C
:10D5700077FD08BD08B5FFF739FD08BD08B5FFF711
:10D5800003FD08BD08B5FFF785FD08BD08B5FFF729
:10D590000BFD08BD08B50846FFF79AFC012008BD41
:10D5A00008B50846FFF794FC012008BD10B51446E5
:10D5B00008461146FFF7DCFC204610BD38B50D4685
:10D5C000084601F0ABFF044628462146FFF7D0FC91
:10D5D000204638BD704700BF044B00221A714FF43B
:10D5E0007A7199601A73024A1A60704740DEFF1F11
:10D5F000900C010031F0004310B408D00F4AA3F59D
:10D60000801494420AD804205DF8044B7047002827
:10D610000CBF022003205DF8044B7047B3F5801F58
:10D6200001D20320F7E7064A934201D00020F2E737
:10D63000D0F1010038BF0020EDE700BFFFFFDF7F22
:10D640000000F07F81F0004102E000BF83F0004362
:10D6500030B54FEA41044FEA430594EA050F08BF8D
:10D6600090EA020F1FBF54EA000C55EA020C7FEA51
:10D67000645C7FEA655C00F0E2804FEA5454D4EBCE
:10D680005555B8BF6D420CDD2C4480EA020281EA98
:10D69000030382EA000083EA010180EA020281EAD0
:10D6A0000303362D88BF30BD11F0004F4FEA013122
:10D6B0004FF4801C4CEA113102D0404261EB410131
:10D6C00013F0004F4FEA03334CEA133302D05242B7
:10D6D00063EB430394EA050F00F0A780A4F1010473
:10D6E000D5F1200E0DDB02FA0EFC22FA05F28018AD
:10D6F00041F1000103FA0EF2801843FA05F3594193
:10D700000EE0A5F120050EF1200E012A03FA0EFC11
:10D7100028BF4CF0020C43FA05F3C01851EBE3713B
:10D7200001F0004507D54FF0000EDCF1000C7EEB58
:10D7300000006EEB0101B1F5801F1BD3B1F5001F96
:10D740000CD349085FEA30004FEA3C0C04F10104B5
:10D750004FEA445212F5800F80F09A80BCF1004FDE
:10D7600008BF5FEA500C50F1000041EB045141EA60
:10D77000050130BD5FEA4C0C404141EB010111F461
:10D78000801FA4F10104E9D191F0000F04BF01460C
:10D790000020B1FA81F308BF2033A3F10B03B3F1EA
:10D7A00020020CDA0C3208DD02F1140CC2F10C027A
:10D7B00001FA0CF021FA02F10CE002F11402D8BFD8
:10D7C000C2F1200C01FA02F120FA0CFCDCBF41EAA4
:10D7D0000C019040E41AA2BF01EB0451294330BD73
:10D7E0006FEA04041F3C1CDA0C340EDC04F1140450
:10D7F000C4F1200220FA04F001FA02F340EA030027
:10D8000021FA04F345EA030130BDC4F10C04C4F16C
:10D81000200220FA02F001FA04F340EA030029464C
:10D8200030BD21FA04F0294630BD94F0000F83F496
:10D83000801306BF81F480110134013D4EE77FEA79
:10D84000645C18BF7FEA655C29D094EA050F08BFC5
:10D8500090EA020F05D054EA000C04BF19461046A6
:10D8600030BD91EA030F1EBF0021002030BD5FEAEA
:10D87000545C05D14000494128BF41F0004130BD12
:10D8800014F580043CBF01F5801130BD01F0004566
:10D8900045F0FE4141F470014FF0000030BD7FEAD9
:10D8A000645C1ABF194610467FEA655C1CBF0B46D4
:10D8B000024650EA013406BF52EA033591EA030FEB
:10D8C00041F4002130BD00BF90F0000F04BF0021E3
:10D8D000704730B54FF4806404F132044FF0000516
:10D8E0004FF0000150E700BF90F0000F04BF00218F
:10D8F000704730B54FF4806404F1320410F00045F5
:10D9000048BF40424FF000013EE700BF42004FEAEF
:10D91000E2014FEA31014FEA02701FBF12F07F436C
:10D9200093F07F4F81F06051704792F0000F14BF69
:10D9300093F07F4F704730B54FF4607401F00045AD
:10D9400021F0004120E700BF50EA010208BF704704
:10D9500030B54FF000050AE050EA010208BF7047F9
:10D9600030B511F0004502D5404261EB41014FF462
:10D97000806404F132045FEA915C3FF4DCAE4FF066
:10D9800003025FEADC0C18BF03325FEADC0C18BF4D
:10D99000033202EBDC02C2F1200300FA03FC20FA9E
:10D9A00002F001FA03FE40EA0E0021FA02F11444EB
:10D9B000C1E600BF70B54FF0FF0C4CF4E06C1CEA00
:10D9C00011541DBF1CEA135594EA0C0F95EA0C0F75
:10D9D00000F0DEF82C4481EA030621EA4C5123EAE8
:10D9E0004C5350EA013518BF52EA033541F4801117
:10D9F00043F4801338D0A0FB02CE4FF00005E1FBCA
:10DA000002E506F00042E0FB03E54FF00006E1FB13
:10DA100003569CF0000F18BF4EF0010EA4F1FF0456
:10DA2000B6F5007F64F5407404D25FEA4E0E6D4196
:10DA300046EB060642EAC62141EA55514FEAC520A7
:10DA400040EA5E504FEACE2EB4F1FD0C88BFBCF523
:10DA5000E06F1ED8BEF1004F08BF5FEA500E50F1D4
:10DA6000000041EB045170BD06F0004646EA01019A
:10DA700040EA020081EA0301B4EB5C04C2BFD4EBCC
:10DA80000C0541EA045170BD41F480114FF0000EC5
:10DA9000013C00F3AB8014F1360FDEBF002001F033
:10DAA000004170BDC4F10004203C35DA0C341BDCAD
:10DAB00004F11404C4F1200500FA05F320FA04F07F
:10DAC00001FA05F240EA020001F0004221F00041B3
:10DAD00010EBD37021FA04F642EB06015EEA430E26
:10DAE00008BF20EAD37070BDC4F10C04C4F1200556
:10DAF00000FA04F320FA05F001FA04F240EA020009
:10DB000001F0004110EBD37041F100015EEA430ED9
:10DB100008BF20EAD37070BDC4F1200500FA05F2F9
:10DB20004EEA020E20FA04F301FA05F243EA020378
:10DB300021FA04F001F0004121FA04F220EA020087
:10DB400000EBD3705EEA430E08BF20EAD37070BDCD
:10DB500094F0000F0FD101F00046400041EB0101AD
:10DB600011F4801F08BF013CF7D041EA060195F08F
:10DB7000000F18BF704703F00046520043EB030349
:10DB800013F4801F08BF013DF7D043EA0603704736
:10DB900094EA0C0F0CEA135518BF95EA0C0F0CD041
:10DBA00050EA410618BF52EA4306D1D181EA030187
:10DBB00001F000414FF0000070BD50EA410606BF81
:10DBC0001046194652EA430619D094EA0C0F02D1C6
:10DBD00050EA013613D195EA0C0F05D152EA03360B
:10DBE0001CBF104619460AD181EA030101F0004129
:10DBF00041F0FE4141F470014FF0000070BD41F072
:10DC0000FE4141F4780170BD70B54FF0FF0C4CF44B
:10DC1000E06C1CEA11541DBF1CEA135594EA0C0F6A
:10DC200095EA0C0F00F0A7F8A4EB050481EA030EB7
:10DC300052EA03354FEA013100F088804FEA03339E
:10DC40004FF0805545EA131343EA12634FEA02226C
:10DC500045EA111545EA10654FEA00260EF000412D
:10DC60009D4208BF964244F1FD0404F5407402D27F
:10DC70005B084FEA3202B61A65EB03055B084FEA10
:10DC800032024FF480104FF4002CB6EB020E75EB0D
:10DC9000030E22BFB61A754640EA0C005B084FEA35
:10DCA0003202B6EB020E75EB030E22BFB61A7546B2
:10DCB00040EA5C005B084FEA3202B6EB020E75EBFD
:10DCC000030E22BFB61A754640EA9C005B084FEA75
:10DCD0003202B6EB020E75EB030E22BFB61A754682
:10DCE00040EADC0055EA060E18D04FEA051545EA71
:10DCF00016754FEA06164FEAC30343EA52734FEA1A
:10DD0000C2025FEA1C1CC0D111F4801F0BD141EA92
:10DD100000014FF000004FF0004CB6E711F4801FF7
:10DD200004BF01430020B4F1FD0C88BFBCF5E06FD7
:10DD30003FF6AFAEB5EB030C04BFB6EB020C5FEAE7
:10DD4000500C50F1000041EB045170BD0EF0004E3C
:10DD50004EEA113114EB5C04C2BFD4EB0C0541EA6E
:10DD6000045170BD41F480114FF0000E013C90E66B
:10DD700045EA060E8DE60CEA135594EA0C0F08BF2F
:10DD800095EA0C0F3FF43BAF94EA0C0F0AD150EA2E
:10DD900001347FF434AF95EA0C0F7FF425AF1046C1
:10DDA00019462CE795EA0C0F06D152EA03353FF4E9
:10DDB000FDAE1046194622E750EA410618BF52EA66
:10DDC00043067FF4C5AE50EA41047FF40DAF52EA3A
:10DDD00043057FF4EBAE12E74FF0FF3C06E000BFD7
:10DDE0004FF0010C02E000BF4FF0010C4DF804CDE4
:10DDF0004FEA410C7FEA6C5C4FEA430C18BF7FEAA4
:10DE00006C5C1BD001B050EA410C0CBF52EA430CD1
:10DE100091EA030F02BF90EA020F0020704710F151
:10DE2000000F91EA030F58BF994208BF90422CBFE0
:10DE3000D8176FEAE37040F0010070474FEA410CD9
:10DE40007FEA6C5C02D150EA013C07D14FEA430CF7
:10DE50007FEA6C5CD6D152EA033CD3D05DF8040B68
:10DE6000704700BF8446104662468C46194663469A
:10DE700000E000BF01B5FFF7B7FF002848BF10F171
:10DE8000000F01BD4DF808EDFFF7F4FF0CBF0120B6
:10DE900000205DF808FB00BF4DF808EDFFF7EAFF32
:10DEA00034BF012000205DF808FB00BF4DF808EDED
:10DEB000FFF7E0FF94BF012000205DF808FB00BFE2
:10DEC0004DF808EDFFF7CEFF94BF012000205DF86C
:10DED00008FB00BF4DF808EDFFF7C4FF34BF012079
:10DEE00000205DF808FB00BF4A0011D212F50012B5
:10DEF00011D20DD56FF47873B3EB62520ED44FEAA2
:10DF0000C12343F0004343EA505323FA02F0704721
:10DF10004FF00000704750EA013002D14FF0FF305F
:10DF200070474FF00000704780F0004002E000BFF3
:10DF300081F0004142001FBF5FEA410392EA030FF4
:10DF40007FEA226C7FEA236C6AD04FEA1262D2EB3E
:10DF50001363C1BFD218414048404140B8BF5B4243
:10DF6000192B88BF704710F0004F40F4000020F0DC
:10DF70007F4018BF404211F0004F41F4000121F0F2
:10DF80007F4118BF494292EA030F3FD0A2F101023C
:10DF900041FA03FC10EB0C00C3F1200301FA03F17A
:10DFA00000F0004302D5494260EB4000B0F5000F9D
:10DFB00013D3B0F1807F06D340084FEA310102F15C
:10DFC0000102FE2A51D2B1F1004F40EBC25008BF0E
:10DFD00020F0010040EA03007047490040EB0000D8
:10DFE00010F4000FA2F10102EDD1B0FA80FCACF107
:10DFF000080CB2EB0C0200FA0CF0AABF00EBC25006
:10E0000052421843BCBFD0401843704792F0000FF3
:10E0100081F4000106BF80F400000132013BB5E746
:10E020004FEA41037FEA226C18BF7FEA236C21D0BC
:10E0300092EA030F04D092F0000F08BF0846704721
:10E0400090EA010F1CBF0020704712F07F4F04D1EF
:10E05000400028BF40F00040704712F100723CBF02
:10E0600000F50000704700F0004343F0FE4040F42C
:10E07000000070477FEA226216BF08467FEA2363EA
:10E080000146420206BF5FEA412390EA010F40F4D5
:10E09000800070474FF0000304E000BF10F0004321
:10E0A00048BF40425FEA000C08BF704743F0964308
:10E0B00001464FF000001CE050EA010208BF704723
:10E0C0004FF000030AE000BF50EA010208BF7047AA
:10E0D00011F0004302D5404261EB41015FEA010CBF
:10E0E00002BF84460146002043F0B64308BFA3F1B7
:10E0F0008053A3F50003BCFA8CF2083AA3EBC25399
:10E1000010DB01FA02FC634400FA02FCC2F12002B7
:10E11000BCF1004F20FA02F243EB020008BF20F0EE
:10E120000100704702F1200201FA02FCC2F1200254
:10E1300050EA4C0021FA02F243EB020008BF20EA49
:10E14000DC7070474FF0FF0C1CEAD0521EBF1CEA77
:10E15000D15392EA0C0F93EA0C0F6FD01A4480EA65
:10E16000010C400218BF5FEA41211ED04FF000634E
:10E1700043EA501043EA5111A0FB01310CF000407A
:10E18000B1F5000F3EBF490041EAD3715B0040EAA0
:10E19000010062F17F02FD2A1DD8B3F1004F40EB70
:10E1A000C25008BF20F00100704790F0000F0CF043
:10E1B000004C08BF49024CEA502040EA51207F3A07
:10E1C000C2BFD2F1FF0340EAC250704740F40000E2
:10E1D0004FF00003013A5DDC12F1190FDCBF00F0D3
:10E1E00000407047C2F10002410021FA02F1C2F181
:10E1F000200200FA02FC5FEA310040F1000053EA1D
:10E200004C0308BF20EADC70704792F0000F00F06A
:10E21000004C02BF400010F4000F013AF9D040EA70
:10E220000C0093F0000F01F0004C02BF490011F404
:10E23000000F013BF9D041EA0C018FE70CEAD15302
:10E2400092EA0C0F18BF93EA0C0F0AD030F0004C82
:10E2500018BF31F0004CD8D180EA010000F0004036
:10E26000704790F0000F17BF90F0004F084691F0F4
:10E27000000F91F0004F14D092EA0C0F01D142022E
:10E280000FD193EA0C0F03D14B0218BF084608D1F7
:10E2900080EA010000F0004040F0FE4040F4000041
:10E2A000704740F0FE4040F4400070474FF0FF0CD4
:10E2B0001CEAD0521EBF1CEAD15392EA0C0F93EA1B
:10E2C0000C0F69D0A2EB030280EA010C49024FEA6D
:10E2D000402037D04FF0805343EA111143EA101326
:10E2E0000CF000408B4238BF5B0042F17D024FF4DE
:10E2F000000C8B4224BF5B1A40EA0C00B3EB510FB9
:10E3000024BFA3EB510340EA5C00B3EB910F24BFA1
:10E31000A3EB910340EA9C00B3EBD10F24BFA3EB26
:10E32000D10340EADC001B0118BF5FEA1C1CE0D1EE
:10E33000FD2A3FF650AF8B4240EBC25008BF20F0A1
:10E34000010070470CF0004C4CEA50207F32C2BFF5
:10E35000D2F1FF0340EAC250704740F400004FF092
:10E360000003013A37E792F0000F00F0004C02BFC3
:10E37000400010F4000F013AF9D040EA0C0093F08D
:10E38000000F01F0004C02BF490011F4000F013BE7
:10E39000F9D041EA0C0195E70CEAD15392EA0C0F4F
:10E3A00008D142027FF47DAF93EA0C0F7FF470AF87
:10E3B000084676E793EA0C0F04D14B023FF44CAFCA
:10E3C00008466EE730F0004C18BF31F0004CCAD15F
:10E3D00030F000427FF45CAF31F000437FF43CAF9B
:10E3E0005FE700BF4FF0FF3C06E000BF4FF0010CBD
:10E3F00002E000BF4FF0010C4DF804CD4FEA40029F
:10E400004FEA41037FEA226C18BF7FEA236C11D0E8
:10E4100001B052EA530C18BF90EA010F58BFB2EB9B
:10E42000030088BFC81738BF6FEAE17018BF40F01B
:10E43000010070477FEA226C02D15FEA402C05D1CF
:10E440007FEA236CE4D15FEA412CE1D05DF8040B54
:10E45000704700BF844608466146FFE70FB5FFF7E7
:10E46000C9FF002848BF10F1000F0FBD4DF808ED9F
:10E47000FFF7F4FF0CBF012000205DF808FB00BF90
:10E480004DF808EDFFF7EAFF34BF012000205DF8EA
:10E4900008FB00BF4DF808EDFFF7E0FF94BF012037
:10E4A00000205DF808FB00BF4DF808EDFFF7D2FF34
:10E4B00094BF012000205DF808FB00BF4DF808ED77
:10E4C000FFF7C8FF34BF012000205DF808FB00BF44
:10E4D0004FEA4002B2F1FE4F0FD34FF09E03B3EB71
:10E4E00012620DD94FEA002343F0004310F0004FB1
:10E4F00023FA02F018BF404270474FF00000704707
:10E5000012F1610F01D1420205D110F0004008BFA5
:10E510006FF0004070474FF00000704742000ED28D
:10E52000B2F1FE4F0BD34FF09E03B3EB126209D44E
:10E530004FEA002343F0004323FA02F070474FF004
:10E540000000704712F1610F01D1420202D14FF079
:10E55000FF3070474FF00000704700BF0346084689
:10E56000194600F009B800BF00210A2201F0C2B824
:10E5700000210A2201F0BEB810B40C461346014631
:10E58000224602205DF8044B01F05CB970B50F4ED5
:10E590000F4D761BB61007D0043D0024013455F80A
:10E5A000043F9847A642F9D10A4E0B4D761B02F064
:10E5B0001FFCB61008D0043D0024013455F8043F78
:10E5C0009847A642F9D170BD70BD00BFFC0D010097
:10E5D000FC0D01004C0E0100FC0D0100034B1B68FB
:10E5E0001844407800F00800704700BF7CAFFF1F60
:10E5F000024B0146186800F00BB800BF68ABFF1F64
:10E60000024B0146186801F0E7B900BF68ABFF1F75
:10E610002DE9F04F01F10B05162D83B0064627D9E1
:10E6200035F0070527D4A94225D8304600F06AFB0B
:10E63000B5F5FC7F26D2C14F4FEAD50C07EBCC03D2
:10E64000DC689C4200F0D2816368E268A16823F034
:10E650000303234430465D68CA6045F001059160BC
:10E660005D6000F051FB0834204603B0BDE8F08F38
:10E670001025A942D9D900240C232046336003B0C9
:10E68000BDE8F08F5FEA552C00F08A80BCF1040FE2
:10E6900000F260814FEA951C0CF1380C4FEA4C01F6
:10E6A000A64F07EB8101CC68A14205D10CE0002BFD
:10E6B0007ADAE468A14207D0626822F00302531BB1
:10E6C0000F2BF4DD0CF1FF3C0CF1010C9B4B3C6972
:10E6D00003F1080E744500F07E81616821F00301AA
:10E6E0004A1B0F2A00F36481002AC3F814E0C3F820
:10E6F00010E06ADAB1F5007F80F03A81C90803EBD7
:10E70000C1004FEAA1085A688168A1604FF0010971
:10E7100009FA08F848EA0202E0605A608460CC60B6
:10E720004FEAAC030120984090425BD8024206D1E8
:10E730002CF0030C400002420CF1040CFAD007EB61
:10E74000CC084446E146E3689C4207D145E1002AF3
:10E7500080F25681DB689C4200F03F81596821F0CD
:10E7600003014A1B0F2AF2DD1C46D3F80CC054F8F3
:10E77000088F591945F0010942F00105C3F80490CA
:10E780003046C8F80CC0CCF8088079613961C1F80E
:10E790000CE0C1F808E04D608A5000F0B5FA63E77C
:10E7A0007E214FF03F0C7BE72244E3685068A1686C
:10E7B00040F00105CB6030469960556000F0A4FA46
:10E7C0000834204603B0BDE8F08F214430464B6842
:10E7D00043F001034B6000F097FA0834204603B081
:10E7E000BDE8F08FBC68636823F00309A94504D332
:10E7F000C5EB09030F2B00F39180514B514A196867
:10E800001368013305EB010A04EB090B00F0618189
:10E810000AF5805A0AF10F0A2AF47F6A2AF00F0AD1
:10E8200030465146019200F05FFCB0F1FF3F804658
:10E83000019A00F00081834500F2FA80DFF810C1F0
:10E84000DCF80030C3455344CCF8003000F04A8176
:10E8500012683C4901321BBFCBEB080B5B44C1F88B
:10E860000080CCF8003018F0070300F01381C3F1EA
:10E870000802C3F5805390440833C244CAF30B0A1C
:10E88000CAEB030A51463046CDF804C000F02CFC18
:10E89000431CDDF804C000F03581C8EB000252448F
:10E8A00042F00102DCF80030C7F808805344BC4253
:10E8B000C8F80420CCF80030DFF894A015D0B9F1E6
:10E8C0000F0F40F2EA806168A9F10C0222F0070202
:10E8D00001F0010EA118052042EA0E0E0F2AC4F81D
:10E8E00004E04860886000F21181174ABC68116832
:10E8F0008B4288BF1360154A11688B4288BF136032
:10E90000626822F003029542C5EB020301D80F2B87
:10E9100004DC304600F0F8F90024A5E6621943F063
:10E92000010345F0010565603046BA60536000F0B0
:10E93000EBF90834204603B0BDE8F08F6CABFF1F45
:10E9400058DEFF1F78AFFF1F54DEFF1F50DEFF1F92
:10E950005CDEFF1FBCF1140F61D9BCF1540F00F253
:10E960008F804FEA153C0CF16E0C4FEA4C0197E694
:10E970004B0A042B58D9142B00F2AE8003F15B0232
:10E98000500007EB8000DFF8BC818368834200F011
:10E990008A805A6822F00302914202D29B68984210
:10E9A000F7D1D9687A68E160A3608C60DC60B7E673
:10E9B000611942F0010745F0010565603046596173
:10E9C0001961C1F80CE0C1F808E04F608A500834C2
:10E9D00000F09AF948E65A68A2E609F1010919F02F
:10E9E000030F04F108047FF4AEAE2DE004F1080338
:10E9F0006469A34208BF0CF1020C3FF467AE23E642
:10EA000019441C464868DB6854F8082F40F001059B
:10EA10004D603046D3609A6000F076F924E60CF140
:10EA20005B0C4FEA4C013BE68A0938325000A8E7FC
:10EA3000BC423FF403AFBC68626822F0030262E7A5
:10EA4000D8F8008098457BD11CF0030FA8F108038B
:10EA50000CF1FF3CF4D17B6823EA00037B604000AB
:10EA600098423FF6BFAE00283FF4BCAE0342CC460E
:10EA70007FF465AE400003420CF1040CFAD05EE670
:10EA8000BCF5AA7F1AD84FEAD53C0CF1770C4FEAB7
:10EA90004C0105E64FF48053EFE60123C8F804303B
:10EAA000444600222FE791100120D8F8042000FAF4
:10EAB00001F10A43C8F80420194674E740F25453A0
:10EAC0009C451BD84FEA954C0CF17C0C4FEA4C014D
:10EAD000E6E50AF1100AA3E6542B1FD80A0B6E32A2
:10EAE00050004EE7CBF30B0100297FF4B1AE0AEBE7
:10EAF0000901BA6841F001015160F6E6FC214FF0CE
:10EB00007E0CCDE501224FF0000ACBE604F10801AE
:10EB1000304600F061FFDAF80030E6E6B3F5AA7F90
:10EB200003D8CA0B773250002BE740F2545293427D
:10EB300003D88A0C7C32500023E7FC207E2220E799
:10EB40007B688CE76CABFF1F032A70B428D940EABE
:10EB500001039B0713D005780C78A54224D1013A14
:10EB6000002305E010F8015F11F8014FA5421BD109
:10EB7000934203F10103F5D1002070BC70470C46AD
:10EB8000034625681E68AE422146184604F1040477
:10EB900003F1040304D1043A032A18462146F0D8AD
:10EBA000002AD8D11046E8E7281B70BC704700BF88
:10EBB0008842F0B410D98C18A0420DD28518531E8B
:10EBC00042B121462A4611F8014D02F8014D013BA0
:10EBD0005C1CF8D1F0BC70470F2A3FD940EA010312
:10EBE0009B073FD1A2F110073F0900EB0716103633
:10EBF0000C46034625681D6065685D60A5689D60DC
:10EC0000E568DD601033B34204F11004F2D17B1CDF
:10EC100002F00F0C1B01BCF1030F1944034423D96C
:10EC20000E461D466446043C56F8047B45F8047BBA
:10EC3000032CF8D8ACF1040424F00304043402F0EB
:10EC4000030223442144002AC4D01A4411F8014B82
:10EC500003F8014B9342F9D1F0BC70470346002AF8
:10EC6000F3D1B7E70346F0E76246002AEDD1B1E7FA
:10EC7000F0B4840743D0541E002A3ED0CDB20346E0
:10EC800003E0621E002C38D0144603F8015B9A079B
:10EC9000F7D1032C2AD9CDB245EA05250F2C45EA38
:10ECA000054515D9A4F110073F0903F1100606EB3D
:10ECB00007161A46156055609560D5601032B2424D
:10ECC000F8D104F00F040137032C03EB07130DD91F
:10ECD0001E462246043A032A46F8045BFAD8221F4D
:10ECE00022F003020432134404F003042CB1C9B22D
:10ECF0001C4403F8011BA342FBD1F0BC704714462F
:10ED00000346C6E7704700BF704700BF024B0A4684
:10ED10000146186800F002B868ABFF1F2DE9F04FFC
:10ED20000C4683B090468146002900F0E280FFF750
:10ED3000E9FF08F10B0654F8043C162E23F00305F6
:10ED4000A4F108074BD810210E46B0454CD88D428F
:10ED500078DADFF890B3DBF808E07819864500F040
:10ED6000CE80426822F0010C8444DCF804C01CF020
:10ED7000010F7AD000221046DB0700F1928054F890
:10ED8000083CC3EB070ADAF8043023F003032B44F2
:10ED900088B3704500F0ED8002EB030E8E452ADB50
:10EDA000C36882685746D3609A6057F8081FDAF83C
:10EDB0000C30CB602A1F242A996000F22681132A86
:10EDC00040F2B3802368CAF808306368CAF80C3090
:10EDD0001B2A00F2308108340AF11003A6E026F065
:10EDE0000706002E3146B0DA0C230020C9F80030A7
:10EDF00003B0BDE8F08F8B4253DB5746DAF80C10B6
:10EE000057F8080F2A1F242AC160886000F2098180
:10EE1000132A40F204812168CAF808106168CAF810
:10EE20000C101B2A00F21C8108340AF11002216820
:10EE3000116061685160A16891601D46DAF8043084
:10EE40003C465746AA1B0F2A03F0010319D82B434F
:10EE50003D447B606B6843F001036B604846FFF7FD
:10EE600053FF204603B0BDE8F08F22F0030202EB0F
:10EE7000050C8C4580DBC26881686546CA6091607C
:10EE8000E0E7B91942F001001E430A447E60486081
:10EE9000536843F0010308315360484600F09CFD7D
:10EEA000DCE741464846FFF7B3FB8046D0B154F853
:10EEB000043C23F001023A44A0F10801914200F021
:10EEC0009E802A1F242A50D8132A23D8034622467C
:10EED000116819605168596092689A6021464846E5
:10EEE00000F07AFD4846FFF70FFF404603B0BDE84B
:10EEF000F08F114603B0BDE8F04FFFF789BBDEF895
:10EF0000042022F00302501906F1100C604519DAB2
:10EF1000704631E723680360636843601B2A63D847
:10EF200000F1080304F10802D2E73B4622681A60A8
:10EF300062685A60A2689A603C467546DAF8043006
:10EF400057467FE73744831B43F00103CBF8087033
:10EF50007B6054F8043C03F001031E43484644F828
:10EF6000046CFFF7D1FE20467CE72146FFF720FE28
:10EF7000B4E702EB030C06F110029445FFF63BAF39
:10EF80005746DAF80C3057F8081F2A1F242ACB609E
:10EF9000996000F28780132A78D92368CAF808306C
:10EFA0006368CAF80C301B2A00F2858008340AF125
:10EFB000100322681A6062685A60A2689A600AEBBD
:10EFC0000603C6EB0C0242F00102CBF808305A608F
:10EFD000DAF8043003F001031E434846CAF804601F
:10EFE000FFF792FE38463DE7A3688360E368C3609D
:10EFF000242A2CD000F1100304F1100268E750F825
:10F00000042C22F0030215441CE7214638467546BD
:10F010003C46FFF7CDFD5746DAF8043012E73A4692
:10F0200005E7214638461D463C46FFF7C1FD5746D9
:10F03000DAF8043006E7A368CAF81030E368CAF8C3
:10F040001430242A18D010340AF118036EE723690B
:10F0500003616369436104F1180200F1180337E7A3
:10F06000A168CAF81010E168CAF81410242A0FD059
:10F0700010340AF11802DAE62369CAF81830636915
:10F08000CAF81C3018340AF120034FE73B4690E7DA
:10F090002269CAF818206269CAF81C2018340AF1DB
:10F0A0002002C4E621463846CDF804C0FFF780FDB3
:10F0B000DDF804C083E7A368CAF81030E368CAF833
:10F0C0001430242A03D010340AF1180371E723699D
:10F0D000CAF818306369CAF81C3018340AF12003E2
:10F0E00067E700BF6CABFF1F38B5074C0023054630
:10F0F00008462360FBF776F9431C00D038BD23682F
:10F10000002BFBD02B6038BD98DEFF1F0F4B30B4B7
:10F110001C68054602E0D01A16D1ABB115F8013BC8
:10F12000E0181A46407800F00300012808BF03F1F8
:10F13000200211F8013BE018407800F0030001289C
:10F14000E9D12033D01AE9D030BC70477CAFFF1F23
:10F15000C9B2F0B4002947D085070FD00278002A41
:10F160003FD091423ED0431C05E013F8012B002A0A
:10F1700037D0914236D09A071846F6D1036841EA53
:10F18000012747EA074783EA0702A2F10135A3F105
:10F19000013425EA020224EA0303134313F0803FFB
:10F1A00011D1021D104652F8043B83EA0704A4F172
:10F1B0000136A3F1013526EA040425EA03032343BB
:10F1C00013F0803FEED00378002B39D0994209D05C
:10F1D000431C01E0914205D0184613F8012B002A88
:10F1E000F8D11046F0BC704784070BD00378002B91
:10F1F000F8D0431C03E002780133002AF2D09907CB
:10F200001846F8D10368A3F1013222EA030313F090
:10F21000803F0AD1031D184653F8042BA2F1013197
:10F2200021EA020212F0803FF5D00378002BD9D0FA
:10F23000431C184601330278002AFAD1F0BC70470B
:10F240001846CFE740EA010C1CF0070F23D1BDF1AF
:10F25000100DCDE90245CDE900676FF000064FF0D3
:10F26000000700BFF0E80223F1E80245A24282FA5B
:10F2700046FCA7FA86FC08BFBCF1000F40F0D7801F
:10F28000AB4283FA46FCA7FA86FC08BFBCF1000F2C
:10F2900040F0CA80E6E710F0030C21D020F0030014
:10F2A00050F8042B5FEACC7C08D00FD211F801CBC8
:10F2B0005FFA92F3B3EB0C0C10D17BB111F801CBD8
:10F2C0005FFAA2F3B3EB0C0C08D13BB111F801CB00
:10F2D0005FFAB2F3B3EB0C0C00D10BB96046704788
:10F2E000BDF1100DCDE90245CDE900676FF00006D4
:10F2F0004FF0000711F0030C2DD110F0040F0DD0CA
:10F3000050F8042B51F8044BA24282FA46FCA7FAAB
:10F3100086FC08BFBCF1000F40F0898011F0040F9B
:10F320009FD051F8045B00BFF0E80223AA4282FAA2
:10F3300046FCA7FA86FC08BFBCF1000F71D1F1E8CA
:10F340000245A34283FA46FCA7FA86FC08BFBCF13B
:10F35000000F63D1E8E721F00301BCF1020F1ED0DA
:10F360003BDA51F8045B00BF50F8043B4FEA152527
:10F3700083FA46FCA7FA86FCB7EB0C2F03EA1622A9
:10F3800008BFAA424DD151F8045BBCF1000F82EADC
:10F3900003034FEA056208BF93423CD1E4E751F80A
:10F3A000045B00BF50F8043B4FEA154583FA46FC66
:10F3B000A7FA86FCB7EB0C4F03EA164208BFAA4235
:10F3C0002FD151F8045BBCF1000F82EA03034FEA2E
:10F3D000054208BF93421ED1E4E751F8045B00BF29
:10F3E00050F8043B4FEA156583FA46FCA7FA86FC01
:10F3F000B7EB0C6F03EA166208BFAA4211D151F8AD
:10F40000045BBCF1000F82EA03034FEA052208BF48
:10F41000934200D1E4E719BA12BA0AE019BA22BA43
:10F4200007E011BA2ABA04E019BA2ABA01E011BAFF
:10F4300022BA9CFA8CF0DDE90067DDE902451DF196
:10F44000100D38B1B0FA80F0C0F1180021FA00F1C7
:10F4500022FA00F20120914298BF8041704700BF1C
:10F4600080EA0102844612F0030F4FD111F0030F1E
:10F4700032D14DF8044D11F0040F51F8043B0BD07C
:10F48000A3F101329A4312F0803F04BF4CF8043BD1
:10F4900051F8043B16D100BF51F8044BA3F10132DF
:10F4A0009A4312F0803FA4F101320BD14CF8043B97
:10F4B000A24312F0803F04BF51F8043B4CF8044BC8
:10F4C000EAD023460CF8013B13F0FF0F4FEA332339
:10F4D000F8D15DF8044B704711F0010F06D011F818
:10F4E000012B0CF8012B002A08BF704711F0020F06
:10F4F000BFD031F8022B12F0FF0F16BF2CF8022BF1
:10F500008CF8002012F47F4FB3D1704711F8012B13
:10F510000CF8012B002AF9D1704700BF20F003013D
:10F5200010F00300C0F1000051F8043B00F1040C9E
:10F530004FEACC0C6FF000021CBF22FA0CF213430E
:10F540004FF0010C4CEA0C2C4CEA0C4CA3EB0C02D7
:10F5500022EA030212EACC1204BF51F8043B043041
:10F56000F4D013F0FF0F1FBF013013F47F4F0130B1
:10F5700013F47F0F18BF0130704700BF40EA01034A
:10F580009B0770B42AD1032A28D90C46034621468A
:10F5900054F8045BA5F1013626EA050616F0803F13
:10F5A00005D1043A032A43F8045B2146EFD89AB107
:10F5B0000C781C70013A01333CB16AB111F8014F6B
:10F5C00003F8014B013A002CF7D12AB11A4400216B
:10F5D00003F8011B9342FBD170BC70470346E6E77A
:10F5E0002DE9F00F424C82B0D4F800C001900E46D5
:10F5F00000E02646344614F8015B0CEB0500407829
:10F6000000F0080000F0FF0A0028F2D12D2D5BD099
:10F610002B2D04BF7578B41C33F010003CD09946F4
:10F62000BAF1000F0CBF6FF0004B4FF0004BBBFB6B
:10F63000F9F8002709FB18BB38460CE0303DAB4217
:10F6400019DD7E1C05D0404523D820D009FB005091
:10F65000012714F8015B0CEB0506767816F0040F11
:10F66000ECD116F0030606D0012E14BF572637261C
:10F67000AD1BAB42E5DC7B1C15D0BAF1000F21D1EC
:10F680000AB1EFB9116002B0BDE8F00F70475D45F7
:10F69000DCDD4FF0FF37DCE7302D1AD0002BBED178
:10F6A0000A239946BCE70199BAF1000F4FF02203F3
:10F6B0000CBF6FF000404FF000400B60002AE2D01A
:10F6C000611EDFE74042DBE7B41C75784FF0010AAA
:10F6D000A2E7207800F0DF00582803D0002B9ED14D
:10F6E00008239CE7102365789946023498E700BF09
:10F6F0007CAFFF1F30B4044C0D46134601462A462A
:10F70000206830BCFFF76CBF68ABFF1F2DE9F00F1E
:10F71000444C82B0D4F800C001900E4600E026466A
:10F72000344614F8015B0CEB0500407800F008004B
:10F7300000F0FF070028F2D12D2D57D02B2D08BF48
:10F740007578BA4608BFB41C33F0100039D04FF0BA
:10F75000FF38B8FBF3F803FB08FB6FEA0B0B994685
:10F76000002738460CE0303DAB4219DD002F25DB89
:10F77000404523D820D009FB0050012714F8015B35
:10F780000CEB0506767816F0040FECD116F00306A4
:10F7900006D0012E14BF57263726AD1BAB42E5DC41
:10F7A000002F1DDBBAF1000F18D10AB1A7B9116003
:10F7B00002B0BDE8F00F70475D45DCDD4FF0FF376C
:10F7C000DCE7302D17D0002BC1D10A2399464FF02A
:10F7D000050BDFF85480C3E7611EE8E74042E4E729
:10F7E0000198222303604FF0FF30DEE7B41C7578E8
:10F7F0004FF0010AA8E7207800F0DF00582808D071
:10F80000002BA4D1082399464FF0070B6FF06048F6
:10F81000A6E71023657899464FF00F0B02346FF07E
:10F8200070489DE77CAFFF1F9999991930B4044C3B
:10F830000D46134601462A46206830BCFFF766BFD6
:10F8400068ABFF1FF0B5274C2668D6F8484185B055
:10F850000746002C41D065681F2D1EDD224818B9CF
:10F860004FF0FF3005B0F0BD4FF4C8700391029225
:10F870000193FEF7BDFE0399029A019B04460028FE
:10F88000EED0D6F848512560002060600546C6F8E5
:10F890004841C4F88801C4F88C013FB9AB1C002072
:10F8A0000135656044F8231005B0F0BD04EB850018
:10F8B0004FF0010CC0F88820D4F888610CFA05F2EA
:10F8C0001643022FC4F88861C0F80831E6D1D4F895
:10F8D0008C311A43C4F88C21E0E706F5A674C6F80B
:10F8E0004841B8E7E80C0100F1E50000024B13B114
:10F8F000024800F005B87047000000000DF9000054
:10F900000146002002460346FFF79CBF38B5094D6B
:10F91000094C641BA41018BF05EB840505D0013CFD
:10F9200055F8043D9847002CF9D1BDE8384001F066
:10F930008DBA00BF0000000000000000F8B5234DA4
:10F940000F460446FFF7DEF9AB685E6826F0030653
:10F95000F11B01F6EF7121F47F6121F00F01A1F598
:10F960008057B7F5805F07DB20460021FFF7BCFB1F
:10F97000AB683344984204D02046FFF7C5F9002015
:10F98000F8BD20467942FFF7AFFB01300DD0104B98
:10F99000AA681968F61B46F001062046C91B566086
:10F9A0001960FFF7B1F90120F8BD20460021FFF7EB
:10F9B0009BFBAB68C21A0F2ADEDD064D04492D6899
:10F9C00042F00102401B5A600860D5E76CABFF1F94
:10F9D0005CDEFF1F78AFFF1F2DE9F0410D460646A4
:10F9E000002955D0FFF78EF955F8041CDFF874C1D3
:10F9F00021F00103A5F10804E218DCF808005768BB
:10FA0000904227F0030769D011F00101576032D00E
:10FA10000021D0194068C00706D43B4490680029F3
:10FA20004ED0D268C260906043F001026260E35041
:10FA3000E1B9B3F5007F2DD35A0A042A6AD8980990
:10FA4000383041000CEB810C4649DCF80820624557
:10FA500066D0516821F003018B4202D2926894452E
:10FA6000F7D1D368E360A2609C60D4603046BDE803
:10FA7000F041FFF749B955F8085C641B0CF1080820
:10FA8000A06840452B4443D0E568C560A860C0E746
:10FA9000BDE8F081DB080CEBC3020125DCF80400B3
:10FAA0009168A1609B1005FA03F31843E260CCF85B
:10FAB000040094603046CC60BDE8F041FFF724B903
:10FAC000294DA842ADD143F00102CCF81440CCF846
:10FAD0001040E060A0606260E350C7E71F44CB07BE
:10FAE00007D455F8083CE41A1F44A268E368D360C1
:10FAF0009A601E4B1B6847F001029F426260CCF87F
:10FB00000840B3D31A4B30461968FFF717FFADE72B
:10FB100001217EE7142A0CD802F15B00410091E735
:10FB20004B688010012505FA00F003434B60134633
:10FB300098E7542A03D8180B6E30410082E7B2F5DB
:10FB4000AA7F03D8D80B773041007BE740F25451AD
:10FB50008A4203D8980C7C30410073E7FC217E2058
:10FB600070E700BF6CABFF1F74ABFF1F74AFFF1FCC
:10FB700058DEFF1FFFFFFFFF000000000000000035
:10FB8000F5A3000000000000E803D007E803DC054F
:10FB9000D0070000E803B004780540060807D00746
:10FBA000456E67696E6520736F756E647320646956
:10FBB0007361626C6564202D2066696C6573206DCD
:10FBC000697373696E670000547261636B206F76AE
:10FBD00065726C617920736F756E647320707265E5
:10FBE00073656E7400000000547261636B204F7681
:10FBF00065726C617920736F756E647320646973CC
:10FC000061626C6564202D206E6F2066696C65737F
:10FC100020666F756E640000537461727420706C9E
:10FC20006179696E6720000020696E20456E676902
:10FC30006E6520736C6F742000000000202849441A
:10FC40003A2000002900000020696E2046582073E9
:10FC50006C6F74200000000053746F702020706C73
:10FC60006179696E6720000053717565616B2000D2
:10FC700020616761696E20696E200000206D53006D
:10FC80003A0000002D0000004841524457415245BF
:10FC90002056455253494F4E3A2000004649524D96
:10FCA000574152452056455253494F4E3A20000085
:10FCB000302E39332E343100202D2000207C2000BE
:10FCC000534F554E442046494C4520494E464F001F
:10FCD00046696C656E616D65202020202020202003
:10FCE0002020204D4D3A53533A6D532020202020A0
:10FCF0005072696F72697479000000005452554562
:10FD00000000000046414C53450000005965730057
:10FD10004E6F000048494748000000004C4F570014
:10FD200025000000566F6C756D657300456E676940
:10FD30006E6520766F6C756D653A20004566666568
:10FD400063747320766F6C756D653A200000000057
:10FD5000547261636B204F7665726C617920766FA7
:10FD60006C756D653A20000053717565616B2053A9
:10FD7000657474696E677300204D696E3D00000004
:10FD8000204D61783D00000020456E61626C656425
:10FD90003D00000053717565616B206D696E2073C5
:10FDA000706565643D0000004C6967687420000060
:10FDB00020466C6173682054696D653A200000002C
:10FDC00020426C696E6B204F6E2054696D653A203D
:10FDD0000000000020426C696E6B204F6666205464
:10FDE000696D653A200000005468726F74746C6528
:10FDF0002F456E67696E652053657474696E67730D
:10FE0000000000004175746F2053746172742045C6
:10FE10006E67696E652077697468205468726F74C4
:10FE2000746C653A200000004175746F2053746F44
:10FE30007020456E67696E65204166746572205456
:10FE4000696D652061742049646C653A200000008A
:10FE5000206D696E75746573000000004E2F4100BF
:10FE60005468726F74746C6520537469636B2049B5
:10FE7000646C652061743A2000000000537469636B
:10FE80006B2043656E7465720000000053746963F3
:10FE90006B20456E6400000049646C652044656118
:10FEA0006462616E643A2000536572766F20536518
:10FEB0007474696E67730000536572766F205265C3
:10FEC0007665727365643A200000000054696D65C0
:10FED00020746F207265636F696C3A200000000027
:10FEE00054696D6520746F2072657475726E3A2066
:10FEF00000000000456E6420706F696E74733A20D4
:10FF00000000000025207265636F696C656420281D
:10FF100000000000207553292C200000252062617C
:10FF20007474657279202800207553290000000040
:10FF3000456E67696E65205374617274000000003D
:10FF4000456E67696E652053746F7000456E676912
:10FF50006E6520546F67676C6500000043616E6ECC
:10FF60006F6E200020466972650000004D61636875
:10FF7000696E652047756E20000000002053746193
:10FF8000727400002053746F7000000020546F677B
:10FF9000676C6500204F6E00204F66660000000011
:10FFA00020537461727420626C696E6B696E6700B5
:10FFB00020546F67676C6520626C696E6B696E6751
:10FFC0000000000020466C61736800005573657284
:10FFD00020536F756E64200020506C617900000022
:10FFE0002052657065617400536F756E64204261C4
:10FFF0006E6B2000410000004200000020506C6148
:020000021000EC
:10000000792F53746F70000020506C6179204E6519
:100010007874000020506C61792050726576696FA9
:100020007573000020506C61792052616E646F6DB1
:10003000000000004368616E6E656C205479706545
:10004000730000004368616E6E656C200000000064
:1000500053776974636820280000000020706F7374
:100060006974696F6E7329005661726961626C65AB
:1000700020496E707574202D200000004E756C6C48
:1000800000000000456E67696E6520537065656409
:10009000000000004D617374657220566F6C756DC1
:1000A00065000000556E6B6E6F776E002028436808
:1000B000616E6E656C2052657665727365642900A9
:1000C0004368616E6E656C20547269676765727310
:1000D0000000000020506F7320000000206F6E00B1
:1000E000206F66660000000020746F67676C6520F3
:1000F0006F6E000020746F67676C65206F66660026
:1001000020737461727420626C696E6B696E670033
:100110002073746F7020626C696E6B696E6700008B
:1001200020666C61736800006368616E6E656C5F69
:1001300066756E63000000006368315F66756E630C
:10014000000000006368325F66756E6300000000A7
:100150006368335F66756E63000000006368345F38
:1001600066756E63000000006368355F66756E63D8
:10017000000000006368616E6E656C5F7265766595
:1001800072736564000000006368315F72657665B4
:10019000727365006368325F7265766572736500BD
:1001A0006368335F72657665727365006368345F98
:1001B00072657665727365006368355F7265766532
:1001C000727365006368616E6E656C5F706F735FFC
:1001D000636F756E740000006368315F706F730049
:1001E0006368325F706F73006368335F706F7300B2
:1001F0006368345F706F73006368355F706F73009E
:100200006368616E6E656C5F706F735F747269674F
:10021000676572730000000073717565616B5F73D1
:10022000657474696E67730073316D696E000000E8
:1002300073316D61780000007331656E000000005D
:1002400073326D696E00000073326D6178000000DA
:100250007332656E0000000073336D696E0000003C
:1002600073336D61780000007333656E0000000029
:1002700073346D696E00000073346D6178000000A6
:100280007334656E0000000073356D696E00000008
:1002900073356D61780000007335656E00000000F5
:1002A00073366D696E00000073366D617800000072
:1002B0007336656E000000006D696E73706565646D
:1002C00000000000766F6C756D657300656E676980
:1002D0006E65000065666665637473006F766572AF
:1002E0006C6179006C696768747300006C315F66DB
:1002F0006C617368000000006C315F626C696E6B4A
:100300006F6E00006C315F626C696E6B6F666600C9
:100310006C325F666C617368000000006C325F6273
:100320006C696E6B6F6E00006C325F626C696E6B35
:100330006F6666006C335F666C6173680000000076
:100340006C335F626C696E6B6F6E00006C335F6262
:100350006C696E6B6F666600736F756E6462616E5A
:100360006B0000005342415F6C6F6F700000000033
:100370005342425F6C6F6F700000000073657276CD
:100380006F000000736572766F5F726576657273D9
:100390006500000074696D655F7265636F696C006C
:1003A00074696D655F72657475726E0065705F72F9
:1003B00065636F696C00000065705F6261747465ED
:1003C000727900006175746F73746172740000005B
:1003D0006175746F73746F70000000007468726FE1
:1003E00074746C650000000063656E7465727468F7
:1003F000726F74746C65000069646C656465616437
:1004000062616E6400000000537461727420456E76
:1004100067696E650000000053687574646F776EDD
:1004200020456E67696E650053746F702053717557
:1004300065616B7300000000537461727420537126
:100440007565616B730000004552524F523A205956
:100450006F75206E65656420746F207570646174BB
:10046000652074686520434F554E545F544F544186
:100470004C5F534F554E4446494C4553206E756D65
:1004800062657221000000004572726F723A204E60
:1004900065787420736F756E642062616E6B206680
:1004A000696C65206E6F7420666F756E6400000065
:1004B000536F756E642042616E6B20413A200000DC
:1004C00050726573656E7420284175746F2D6C6F62
:1004D0006F703A2000000000536F756E6420426117
:1004E0006E6B20423A200000535441525420544530
:1004F000535420524F5554494E45000046696C658F
:100500006E616D6520202020202020202020204D9D
:100510004D3A53533A6D5300454E4420544553547D
:1005200020524F5554494E4500000000506C6179EF
:10053000696E672E2E2E2020000000004E6F742062
:10054000666F756E64000000446F6E650000000009
:10055000566F6C756D6520436F6E74726F6C2053AF
:100560006F757263653A2053657269616C000000B3
:10057000566F6C756D6520436F6E74726F6C20538F
:100580006F757263653A205243000000566F6C75B8
:100590006D6520436F6E74726F6C20536F7572635C
:1005A000653A204B6E6F6200446576696365206D25
:1005B0006F64653A20524320696E707574000000C4
:1005C000446576696365206D6F64653A2053657292
:1005D00069616C20696E707574000000556E61620F
:1005E0006C6520746F206163636573732074686544
:1005F0002053442063617264202D20636865636B1F
:1006000020616E64207265626F6F74206465766924
:1006100063650000496E692066696C6520280000EA
:100620002920646F6573206E6F7420657869737418
:100630000000000029206E6F742076616C69643AB6
:1006400020000000496E692066696C652065786944
:10065000737473202D2053657474696E6773204C16
:100660006F616465643A0000284F6E6C7920757381
:10067000656420696E205243206D6F646529000017
:100680002F6F70736F756E642E696E6900FFFFFFC8
:10069000E803350583060807E803E204DC05D6060F
:1006A000080700006E6F206572726F720000000014
:1006B00066696C65206E6F7420666F756E640000ED
:1006C00066696C65206E6F74206F70656E00000047
:1006D00062756666657220746F6F20736D616C6CF5
:1006E000000000007365656B206572726F72000018
:1006F00073656374696F6E206E6F7420666F756EBC
:10070000640000006B6579206E6F7420666F756EF3
:1007100064000000656E64206F662066696C650089
:10072000756E6B6E6F776E206572726F720000006F
:10073000756E6B6E6F776E206572726F7220766168
:100740006C75650074727565000000007965730052
:100750003100000066616C73650000006E6F000080
:100760003000FFFF0000010004000B0013001E001A
:100770002C003C004E0063007B009500B100D000CF
:10078000F10014013A0163018E01BB01EA011D026F
:1007900051028802C102FC023A037B03BD0302043A
:1007A00049049304DF042D057D05D00524067C064D
:1007B000D50630078E07EE075008B4081A098309DA
:1007C000ED095A0AC90A390BAC0B210C980C100D13
:1007D0008B0D080E860E070F890F0D1093101B113D
:1007E000A5113112BE124D13DE13701404159A15A3
:1007F0003216CB16651701189F183E19DF19811A9A
:10080000251BCA1B711C181DC21D6C1E181FC51F7D
:1008100073202321D42186223923ED23A2245825B5
:100820000F26C82681273B28F628B2296F2A2D2BB0
:10083000EC2BAB2C6B2D2C2EED2EAF2F72303531D7
:10084000F931BD32823348340E35D4359B366237A8
:100850002938F138B939813A493B123CDB3CA43D97
:100860006D3E363FFF3FC84091415A422343EB4320
:10087000B4447C4545460C47D4479C486349294AC3
:10088000F04AB64B7B4C404D044EC84E8C4F4E50F8
:100890001051D251935253531254D0548E554B563B
:1008A0000757C2577C583659EE59A55A5C5B115C04
:1008B000C55C785D2A5EDB5E8A5F3960E6609161C7
:1008C0003C62E5628D633364D9647C651E66BF66F5
:1008D0005F67FC6798683369CC69646AF96A8E6BF4
:1008E000206CB16C406DCD6D596EE26E6A6FF06F29
:1008F0007570F7707871F6717372EE726673DD73EE
:100900005274C5743675A47511767B76E4764A7791
:10091000AE7710787078CE7829798379DA792F7A62
:10092000817AD27A207B6C7BB57BFC7B417C847C9A
:10093000C47C027D3E7D777DAE7DE27D147E447E6B
:10094000717E9C7EC47EEA7E0E7F2F7F4E7F6A7F03
:10095000847F9B7FB07FC37FD37FE17FEC7FF47F79
:10096000FB7FFE7FFF7F0000000000000000000012
:10097000A57400000000000000000000000000005E
:100980002D760000000000000000000000000000C4
:1009900011770000000000000000000000000000CF
:1009A000F97F0000000000000000000000000000CF
:1009B0006D81000000000000000000000000000049
:1009C000AD8D0000C58D0000D58D00009D8F00000D
:1009D000BD8F0000F18D000000000000000000004D
:1009E000759C0000799D0000B99C0000CD9C000022
:1009F000F99C0000B59C0000050E08090D0C0607C7
:100A00000F0400130393050E08090D0C06070F04CD
:100A1000FFFFC585848687C4FFFF001303931A92E6
:100A2000170000004008FE4340A004404408FE4375
:100A300044A004400018FE4300C004403000FE43C0
:100A4000309004403400FE43349004401C18FE43B0
:100A50001CC004401018FE4310C004400818FE4398
:100A600008C004400C18FE430CC004400C10FE43A8
:100A70000CB004401010FE4310B004401810FE43A8
:100A800018B004401C10FE431CB004401410FE4378
:100A900014B004400418FE4304C004400010FE4398
:100AA00000B004400008FE4300A004400408FE43D8
:100AB00004A004400C08FE430CA004400808FE43B8
:100AC00008A004401418FE4314C004401818FE4344
:100AD00018C004400410FE4304B004400810FE4354
:100AE00008B004401400FE43149004404C08FE4338
:100AF0004CA004400420FE4304D004402410FE43D4
:100B000024B004402010FE4320B004402810FE43CF
:100B100028B004402C10FE432CB004400020FE43BB
:100B200000D004404808FE4348A004401000FE43A3
:100B3000109004400D0A00006E616E00696E660040
:100B40006F766600FFFFFFFF00000000000000005E
:100B50007DC4000089C4000055C400005DC40000CD
:100B600065C400006DC4000075C4000000000000F2
:100B700000151915000100009CA6FF1F12000000BF
:100B800000020000C8A6FF1F430000000003000091
:100B900024A7FF1F0000000001030904B0A6FF1FE7
:100BA00000000000020309040CA7FF1F0000000062
:100BB0000303090428A7FF1F000000000000000035
:100BC0000000000000000000000000000000000025
:100BD0000DD3000025D30000DDD20000EDD20000CF
:100BE000E5D20000F5D2000059D2000071D2000019
:100BF00091D2000099D20000A5D20000B1D200002D
:100C0000BDD20000CDD20000FDD2000005D300000F
:100C100029D2000035D2000041D200004DD20000A0
:100C200035D3000019D300000000000000000000D0
:100C300051D4000069D4000021D4000031D4000058
:100C400029D4000039D400009DD30000B5D30000A2
:100C5000D5D30000DDD30000E9D30000F5D30000B8
:100C600001D4000011D4000041D4000049D4000098
:100C70006DD3000079D3000085D3000091D300002C
:100C800079D400005DD400000000000000000000E6
:100C900095D50000ADD5000065D5000075D50000E4
:100CA0006DD500007DD50000E1D40000F9D400002E
:100CB00019D5000021D500002DD5000039D5000040
:100CC00045D5000055D5000085D500008DD5000024
:100CD000B1D40000BDD40000C9D40000D5D40000B8
:100CE000BDD50000A1D5000040A7FF1F0020202097
:100CF00020202020202028282828282020202020CC
:100D0000202020202020202020202020208810109B
:100D100010101010101010101010101010040404F7
:100D200004040404040404101010101010104141B5
:100D300041414141010101010101010101010101A3
:100D400001010101010101011010101010104242B7
:100D50004242424202020202020202020202020273
:100D60000202020202020202101010102000000013
:100D70000000000000000000000000000000000073
:100D80000000000000000000000000000000000063
:100D90000000000000000000000000000000000053
:100DA0000000000000000000000000000000000043
:100DB0000000000000000000000000000000000033
:100DC0000000000000000000000000000000000023
:100DD0000000000000000000000000000000000013
:100DE0000000000000000000000000000000000003
:100DF000F8B500BFF8BC08BC9E467047EDF800008F
:100E0000350400006D630000AD750000C975000079
:100E1000F5750000117600007579000091790000E9
:100E2000AD790000C9790000E5790000017A000081
:100E30006195000085950000FD9E000099C40000AA
:0C0E400051D3000095D40000D9D500006B
:040E4C00F8B500BF36
:100E500038B5084B1C681C6054B1074D94FAA4F3D4
:100E6000B3FA83F355F823309847631E1C40F5D13D
:100E700038BD00BFA0D0044088A6FF1F38B5084B7E
:100E80001C681C6054B1074D94FAA4F3B3FA83F3C1
:100E900055F823309847631E1C40F5D138BD00BF7C
:100EA000A0C0044068A6FF1F38B5084B1C681C6032
:100EB00054B1074D94FAA4F3B3FA83F355F82330F1
:100EC0009847631E1C40F5D138BD00BFA0B0044058
:100ED00038A6FF1F38B5084B1C681C6054B1074D7D
:100EE00094FAA4F3B3FA83F355F823309847631EBA
:100EF0001C40F5D138BD00BFA0A00440E8A5FF1FED
:100F000038B5084B1C681C6054B1074D94FAA4F323
:100F1000B3FA83F355F823309847631E1C40F5D18C
:100F200038BD00BFA0900440B0A5FF1F0000000026
:100F30000000803F0000803F0000803F0000000074
:100F400075736572312E7761760000000000000035
:100F5000000000000400000075736572322E776196
:100F60007600000000000000000000000400000007
:100F700075736572332E7761760000000000000003
:100F8000000000000400000075736572342E776164
:100F900076000000000000000000000004000000D7
:100FA00075736572352E77617600000000000000D1
:100FB000000000000400000075736572362E776132
:100FC00076000000000000000000000004000000A7
:100FD00075736572372E776176000000000000009F
:100FE000000000000400000075736572382E776100
:100FF0007600000000000000000000000400000077
:1010000075736572392E776176000000000000006C
:1010100000000000040000007573657231302E7707
:1010200061760000000000000000000004000000E5
:101030007573657231312E77617600000000000013
:1010400000000000040000007573657231322E77D5
:1010500061760000000000000000000004000000B5
:101060007573657231332E776176000000000000E1
:1010700000000000040000007573657231342E77A3
:101080006176000000000000000000000400000085
:101090007573657231352E776176000000000000AF
:1010A00000000000040000007573657231362E7771
:1010B0006176000000000000000000000400000055
:1010C0007573657231372E7761760000000000007D
:1010D00000000000040000007573657231382E773F
:1010E0006176000000000000000000000400000025
:1010F0007573657231392E7761760000000000004B
:1011000000000000040000007573657232302E7715
:1011100061760000000000000000000004000000F4
:1011200002016401656E7374617274322E776176A8
:101130000000000000000000010000000000FF00AF
:1011400080060100D0070000656E6163636C312E7C
:101150007761760000000000000000000100000040
:10116000656E6163636C322E77617600000000006B
:101170000000000001000000656E6163636C332EA7
:101180007761760000000000000000000100000010
:10119000656E6163636C342E776176000000000039
:1011A0000000000001000000656E6163636C352E75
:1011B00077617600000000000000000001000000E0
:1011C000625F62616E6B312E776176000000000015
:1011D0000000000004000000625F62616E6B322E4E
:1011E00077617600000000000000000004000000AD
:1011F000625F62616E6B332E7761760000000000E3
:101200000000000004000000625F62616E6B342E1B
:10121000776176000000000000000000040000007C
:10122000625F62616E6B352E7761760000000000B0
:101230000000000004000000625F62616E6B362EE9
:10124000776176000000000000000000040000004C
:10125000625F62616E6B372E77617600000000007E
:101260000000000004000000625F62616E6B382EB7
:10127000776176000000000000000000040000001C
:10128000625F62616E6B392E77617600000000004C
:101290000000000004000000625F62616E6B31308C
:1012A0002E776176000000000000000004000000BE
:1012B000625F62616E6B31312E77617600000000F3
:1012C0000000000004000000625F62616E6B31325A
:1012D0002E7761760000000000000000040000008E
:1012E000625F62616E6B31332E77617600000000C1
:1012F0000000000004000000625F62616E6B313428
:101300002E7761760000000000000000040000005D
:10131000625F62616E6B31352E776176000000008E
:101320000000000004000000625F62616E6B3136F5
:101330002E7761760000000000000000040000002D
:10134000625F62616E6B31372E776176000000005C
:101350000000000004000000625F62616E6B3138C3
:101360002E776176000000000000000004000000FD
:10137000625F62616E6B31392E776176000000002A
:101380000000000004000000625F62616E6B32309A
:101390002E776176000000000000000004000000CD
:1013A000656E73746F702E77617600000000000028
:1013B000000000000100000001050C020F00000009
:1013C0000000FF00FFFF0F19656E6465636C312E2E
:1013D00077617600000000000000000001000000BE
:1013E000656E6465636C322E7761760000000000E4
:1013F0000000000001000000656E6465636C332E20
:10140000776176000000000000000000010000008D
:10141000656E6465636C342E7761760000000000B1
:101420000000000001000000656E6465636C352EED
:10143000776176000000000000000000010000005D
:1014400001000000615F62616E6B312E7761760092
:10145000000000000000000004000000615F626105
:101460006E6B322E776176000000000000000000F5
:1014700004000000615F62616E6B332E776176005D
:10148000000000000000000004000000615F6261D5
:101490006E6B342E776176000000000000000000C3
:1014A00004000000615F62616E6B352E776176002B
:1014B000000000000000000004000000615F6261A5
:1014C0006E6B362E77617600000000000000000091
:1014D00004000000615F62616E6B372E77617600F9
:1014E000000000000000000004000000615F626175
:1014F0006E6B382E7761760000000000000000005F
:1015000004000000615F62616E6B392E77617600C6
:10151000000000000000000004000000615F626144
:101520006E6B31302E776176000000000000000005
:1015300004000000615F62616E6B31312E7761766D
:10154000000000000000000004000000615F626114
:101550006E6B31322E7761760000000000000000D3
:1015600004000000615F62616E6B31332E7761763B
:10157000000000000000000004000000615F6261E4
:101580006E6B31342E7761760000000000000000A1
:1015900004000000615F62616E6B31352E77617609
:1015A000000000000000000004000000615F6261B4
:1015B0006E6B31362E77617600000000000000006F
:1015C00004000000615F62616E6B31372E776176D7
:1015D000000000000000000004000000615F626184
:1015E0006E6B31382E77617600000000000000003D
:1015F00004000000615F62616E6B31392E776176A5
:10160000000000000000000004000000615F626153
:101610006E6B32302E776176000000000000000013
:101620000400000074725F73746172742E776176C7
:1016300000000000000000000100000074757272DC
:1016400065742E7761760000000000000000000045
:101650000100000074725F73746F702E7761760002
:1016600000000000000000000100000074725F73C1
:101670007472746D2E776176000000000000000027
:10168000010000007475727265745F6D2E7761766B
:1016900000000000000000000100000074725F7391
:1016A000746F706D2E7761760000000000000000FE
:1016B0000100000062725F73746172742E7761764C
:1016C0000000000000000000010000006261727272
:1016D000656C2E77617600000000000000000000BD
:1016E0000100000062725F73746F702E7761760084
:1016F0000000000000000000010000006D675F7343
:10170000746172742E7761760000000000000000A2
:10171000030000006D672E77617600000000000076
:101720000000000000000000030000006D675F7310
:10173000746F702E776176000000000000000000DA
:10174000030000006D673273746172742E776176E6
:101750000000000000000000030000006D67322E52
:10176000776176000000000000000000000000002B
:10177000030000006D673273746F702E776176001E
:101780000000000000000000030000006D673373DC
:10179000746172742E776176000000000000000012
:1017A000030000006D67332E7761760000000000B3
:1017B0000000000000000000030000006D673373AC
:1017C000746F702E7761760000000000000000004A
:1017D0000300000063616E6E6F6E662E77617600A7
:1017E00000000000000000000100000063616E6E58
:1017F0006F6E66322E7761760000000000000000F8
:101800000100000063616E6E6F6E66332E77617645
:1018100000000000000000000100000063616E6E27
:101820006F6E682E776176000000000000000000F7
:101830000100000072656C6F616465642E776176EB
:101840000000000000000000010000006D676869F2
:10185000742E776176000000000000000000000098
:101860000100000064657374726F792E77617600F1
:101870000000000000000000010000006C696768C3
:1018800074312E7761760000000000000000000037
:10189000010000006C69676874322E776176000081
:1018A0000000000000000000010000006C69676893
:1018B00074332E7761760000000000000000000005
:1018C000010000007265706169722E776176000018
:1018D000000000000000000001000000626565706B
:1018E0002E7761760000000000000000000000007C
:1018F000090000006272616B652E7761760000005E
:101900000000000000000000010000007478656E17
:10191000676167652E7761760000000000000000B7
:101920000100000074786465676167652E776176F1
:1019300000000000000000000100000073717565E8
:10194000616B312E7761760000000000000000001E
:101950000100000073717565616B322E776176004E
:1019600000000000000000000100000073717565B8
:10197000616B332E776176000000000000000000EC
:101980000100000073717565616B342E776176001C
:101990000000000000000000010000007371756588
:1019A000616B352E776176000000000000000000BA
:1019B0000100000073717565616B362E77617600EA
:1019C0000000000000000000010000000400000012
:1019D00074726B73746F702E776176000000000074
:1019E000000000000200000074726B737461727476
:1019F0002E77617600000000000000000200000069
:101A0000656E72756E312E77617600000000000001
:101A10000000000001000000656E72756E322E77C6
:101A200061760000000000000000000001000000DE
:101A3000656E72756E332E776176000000000000CF
:101A40000000000001000000656E72756E342E7794
:101A500061760000000000000000000001000000AE
:101A6000656E72756E352E7761760000000000009D
:101A70000000000001000000656E72756E362E7762
:101A8000617600000000000000000000010000007E
:101A9000656E72756E372E7761760000000000006B
:101AA0000000000001000000656E72756E382E7730
:101AB000617600000000000000000000010000004E
:101AC000656E72756E392E77617600000000000039
:101AD0000000000001000000656E72756E31302E4E
:101AE00077617600000000000000000001000000A7
:101AF000010D0000656E69646C655F642E77617628
:101B0000000000000000000001000000656E73741A
:101B1000617274312E7761760000000000000000D1
:101B200001000000656E69646C65312E7761760096
:101B3000000000000000000001000000656E696404
:101B40006C65322E77617600000000000000000016
:101B500001000000656E69646C65332E7761760064
:101B6000000000000000000001000000656E6964D4
:101B70006C65342E776176000000000000000000E4
:101B800001000000656E69646C65352E7761760032
:101B9000000000000000000001000000640A02FFD5
:101BA000E8030000747261636B73312E7761760015
:101BB000000000000000000001000000747261637A
:101BC0006B73322E77617600000000000000000089
:101BD00001000000747261636B73332E77617600CD
:101BE000000000000000000001000000747261634A
:101BF0006B73342E77617600000000000000000057
